:100000000C94AE110C940D830C94E2820C94B78284
:100010000C948C820C9461820C9436820C940B822A
:100020000C94E0810C94DF110C94DF110C94DF111F
:100030000C94DF110C94DF110C94DF110C94DF1180
:100040000C94DF110C94DF110C94DF110C94DF1170
:100050000C94DF110C94DF110C94DF110C9429AD7A
:100060000C94DF110C9464890C943A890C94DF1180
:100070000C94DF110C94DF110C94DF110C94DF1140
:100080000C94DF110C94DF110C94DF110C94DF1130
:100090000C94DF110C94DF110C94DF110C94B42834
:1000A0000C94DF110C94DF110C94DF110C94DF1110
:1000B0000C94DF110C94DF110C94DF110C94DF1100
:1000C0000C94DF110C94DF110C94DF110C94DF11F0
:1000D0000C94DF110C94DF110C94DF110C94DF11E0
:1000E0000C94DF1107634236B79BD8A71A396856BC
:1000F00018AEBAAB558C1D3CB7CC5763BD6DEDFD4A
:10010000753EF6177231BF000000803F0800000006
:10011000BE922449123EABAAAA2ABECDCCCC4C3EFC
:1001200000000080BEABAAAAAA3E00000000BF00EB
:100130000000803F0000000000084178D3BB4387E7
:10014000D1133D190E3CC3BD4282AD2B3E68EC82FB
:1001500076BED98FE1A93E4C80EFFFBE01C4FF7F80
:100160003F00000000000C9472360C9472150C9441
:10017000AE5E0C9489380C9466120C94F0540C9476
:10018000E25E0C940F5F0C94C4130C9467370C94CC
:10019000695A0C94BD1E0C9446210C944AB60C94DA
:1001A00025850C94847D0C94DFA20C94DB4A0C947E
:1001B000C8C30C94497B0C94FB130C94A3310C948E
:1001C00032600C94F0A20C9411120C94298B0C94B4
:1001D00027140C94011F0C9474A60C94FB4B0C94E4
:1001E000CB230C9491140C944F790C94E72D0C9420
:1001F0001E140C9483180C94A6BC0C9461180C94D7
:1002000029320C949C790C9426310C94354C0C9426
:1002100066400C9481270C9412A30C94FB190C9447
:1002200049540C94D57B0C94188B0C943D380C9449
:10023000111E0C9439230C94ECB90C9450220C949C
:100240001B170C9468590C94C81D0C9470400C94A6
:10025000553E0C94B7540C9499C30C94384C0C94A0
:10026000CC130C9476370C9407350C9485660C945B
:1002700070140C94DA5F0C94121A0C94FB370C94E3
:10028000E6A20C941F7B0C94AB200C94D2370C94F8
:10029000A0230C9464BE0C9493310C94FB110C9429
:1002A00014C60C946A150C942B160C94498B0C9460
:1002B0002D170C949BA80C9434330C94F2B90C9425
:1002C000411B0C94F7580C94E1110C94D0970C94AA
:1002D00065140C94944B0C9423400C947B130C9455
:1002E000C0360C94177A0C94A7C30C94285F0C9416
:1002F000B4150C94F2370C9482160C94893A0C9431
:10030000AD130C94654B0C9425C40C94BE150C9441
:10031000973F0C94752F0C942C190C9417790C940E
:10032000FB150C9476150C94A55F0C94454C0C941D
:100330000D320C94F27A0C9483300C94ED790C9479
:10034000EE970C943D1B0C9467120C94B0130C9414
:10035000DE8B0C94AB460C94D2150C940CA30C942D
:10036000199C0C9489170C94D7660C94F8340C944F
:10037000F1340C9435600C94F6A20C94D7A20C9432
:1003800004A30C943F1B0C947C320C944F4D0C94A2
:1003900038600C94D7160C94FB540C94107B0C947E
:1003A00041160C9410BF0C94B9780C94E16F0C9426
:1003B00001170C94FE540C9416A30C94DBA20C941D
:1003C000E3130C94A6370C94F69B0C94FC170C9436
:1003D000ECA20C940E7A0C94C8130C946EA60C9498
:1003E000EB130C944E340C941C120C94D2A70C9466
:1003F000FE340C94B7780C94E3450C94A7300C941D
:10040000CC150C94D26D0C94164C0C948C5F0C94FF
:1004100026750C9496370C94049C0C94E7130C945A
:10042000FF3F0C94FE1D0C94955E0C941A180C94CE
:100430005B7B0C9494150C940B9C0C94E3A20C9491
:100440006A5F0C944D4D0C94117A0C947E150C94AB
:100450009EA80C94F57B0C94A07A0C94A6A80C94FE
:1004600011400C94ED540C94BD1D0C94FAA20C9404
:10047000783B0C94AC130C9459600C944EC40C94BF
:1004800008230C94FEA20C94D5150C949E160C9483
:10049000AA360C94877A0C94938B0C9441A60C94F6
:1004A0008D360C94295E0C94EE580C9435180C94EF
:1004B00045140C94E8150C94B27C0C945C400C949C
:1004C0000D7C0C94F2310C948A140C94C0380C946A
:1004D00074370C948CC20C9453380C9457740C944D
:1004E000FD9B0C9427980C94F7110C94328B0C9470
:1004F0000D980C9465120C9411A30C94D1A20C9439
:10050000241E0C9472400C940C540C9498A80C94D7
:10051000A7360C9482150C94BC370C9465210C946E
:10052000F5780C94A3540C94EB4B0C9424170C9476
:10053000FD580C94B8780C9452380C945C6D0C9463
:1005400036140C941E4B0C94D1300C9441190C941D
:10055000BF300C942A370C944B370C943E140C94F7
:10056000B2450C94CE220C9435370C94316F0C9418
:100570007A150C9431380C94E1540C9472190C9443
:1005800090120C944FB40C946BA60C94A1A80C94EC
:10059000279C0C9423380C947B140C9442380C94B4
:1005A000E6780C94A5780C94D0150C9489120C94D0
:1005B0009C660C94E0380C94328D0C940B2B0C94AC
:1005C000547A0C9449400C9487380C94F63F0C9460
:1005D000D6130C9493C30C94B8160C94A58B0C945E
:1005E000209C0C94DB130C94BB130C9440C40C940F
:1005F000EA970C9409790C94CE4B0C94E5190C9461
:10060000CA540C9408A30C94BD120C9436400C945C
:10061000D7970C94D8130C9470230C948F160C94C9
:10062000A9130C9476120C9469460C940A550C94F8
:10063000A8130C9415380C9408400C946E150C9467
:10064000627B0C94077A0C94534D0C94DE460C9408
:10065000687C0C945F5E0C94CBA70C9416354E41CD
:100660004E494E495459494E46CDCCCC3D0AD7232C
:100670003C17B7D13877CC2B329595E6241FB14F74
:100680000A000020410000C84200401C4620BCBEB9
:100690004CCA1B0E5AAEC59D746364696E6F70734D
:1006A0007578585B00454F46002F00496E3A200090
:1006B0003D00494E3A003D004C45474143592049D1
:1006C0004E3A00000020002300260029002C002FB5
:1006D00000320000010000030106010901204E6FF5
:1006E00020656D69742064617461210020436F7519
:1006F0006E74657220747970652E2076616C3D0091
:10070000494E3A0020436F756E746572207479709B
:10071000652E20494E434F525245435420496E7432
:10072000657272757074206E756D6265722121211B
:10073000004952513A002D3E00200023002D3E007A
:10074000200050656E6465643A2023007261770072
:1007500076616C0074656D70007361740068756516
:100760000066616E0052474200485356006D6F6448
:100770006500536574436D643A0053746F72656429
:10078000204558543A00737566666978436F64650E
:100790003A0020666F7220286D73293A0043545244
:1007A0004C3A205363686564756C6520636D642002
:1007B00000206D73203A0041726D656420666F728F
:1007C00020002044697361726D656400584F4E00CB
:1007D00048414C54002074696D653A004354524CB2
:1007E0003A205265733A002054533A0020543A009C
:1007F0003D0050696E3A004354524C3A20436F6DAD
:100800006D616E6420626C6F636B65642062792039
:10081000647269766572206F72206368616E6E65BE
:100820006C2066726F7A656E004354524C3A204FCA
:100830004E3A416C726561647920416374697665F2
:100840000A004354524C3A2048414C543A416C728D
:100850006561647920496E6163746976650A004355
:1008600054524C3A20584F4E3A2044697361626C9E
:1008700065640A004354524C3A20584F4E3A416C3A
:100880007265616479204163746976650A00435436
:10089000524C3A20584F464620736B69707065641D
:1008A0002E205072657620636D643A004354524C9A
:1008B0003A205475726E6564206F66662066726FAA
:1008C0006D3A004354524C3A20526573746F72650E
:1008D000642066726F6D3A004354524C3A20496767
:1008E0006E6F7265642C206368616E6E656C206348
:1008F0006D643D0020457865633A004354524C3A9C
:10090000204163746976653A004354524C3A20485A
:10091000414C543A416C726561647920496E61635F
:10092000746976650A004354524C3A20584F4E3A47
:100930002044697361626C65640A004354524C3A06
:1009400020584F4E3A416C7265616479204163745E
:100950006976650A004354524C3A20584F46462067
:10096000736B69707065642E205072657620636DBC
:10097000643A004354524C3A205475726E656420B8
:100980006F66662066726F6D3A004354524C3A208F
:10099000526573746F7265642066726F6D3A0043BE
:1009A00054524C3A204E6F7420656E6F7567682004
:1009B0006D656D6F727920666F722067726F7570EA
:1009C000206F7065726174696F6E00496E76616C3C
:1009D00069642061726700496E76616C69642061A8
:1009E0007267004354524C3A20556E6B6E6F776EAF
:1009F0002073756666697800536B69707065642052
:100A0000686F6D69652073747566660020002053F9
:100A100075623D00204974656D3D004354524C3A67
:100A20002052414D3D004354524C3A204F75744F73
:100A3000664D656D6F72793A2000282D29200028B7
:100A40002B2920002076616C7565206973200020B9
:100A5000756E6B6E6F776E0A005D3D005B002069FE
:100A60006E76616C6964002000206F6B003A002094
:100A70006661696C6564003A005265747279696EEA
:100A80006720434D440A004354524C2F706F6C6CE6
:100A90003A204F75744F664D656D6F72793A20003C
:100AA000207365632072656D61696E696E670053BE
:100AB00074617475732064656666657265640A00A6
:100AC000444D58000000000000444D585247425722
:100AD0000000444D5852474200000050574D00005E
:100AE000000000004D42555344494D000054484514
:100AF000524D4F00000052454C4159000000004744
:100B0000524F555000000000564354454D500000D0
:100B1000004D42555356430000004143484149456A
:100B20005200005350494C45440000004D4F544F73
:100B300052000000005049440000000000004D42F7
:100B400055530000000000554152544252444700A2
:100B500052454C415950574D00444D585247425709
:100B6000570056454E545300000000454C45564131
:100B7000544F5200434F554E544552000048554D76
:100B80000000000000004D4552435552590000201E
:100B9000002D3E00436F6E76657274696E672000AB
:100BA0002D3E0057726F6E672041737369676E6DDB
:100BB000656E742000524742783A20004853562010
:100BC00064697361626C65640020764C6576656C5F
:100BD0003A0020436F6E76563A0020436F6E76538C
:100BE0003A0020486F743A00436F6C643A00204327
:100BF0006F6E76657274656420563A00436F6E7648
:100C0000657274656420533A002D3E0057726F6E12
:100C1000672041737369676E6D656E7420002D3EA9
:100C20000057726F6E672041737369676E6D656EF2
:100C300074200053617665643A0020537566663A05
:100C4000002041543A00206973200044656C6574AB
:100C5000696E6720636F6E662E2052414D2077616A
:100C6000733A0053746F70706564006E6F746869D6
:100C70006E6720746F2073746F700053746F7070A0
:100C8000696E67206368616E6E656C73202E2E2E10
:100C9000004E6F7420756E6C6F636B656420696EB7
:100CA00020313073202D20636F6E74696E7565205E
:100CB0002E2E2E00556E6C6F636B696E6720636F0E
:100CC0006E666967202E2E2E00436F6E6669672060
:100CD0006368616E676564206C6F63616C6C792C0E
:100CE00020706F7274616C2064697361626C6564FA
:100CF000002F636F6E6669672E6A736F6E00726590
:100D0000626F6F742000436D643A20002F636F6D33
:100D10006D616E642F002F72616D2F002F697465F5
:100D20006D2F002F6974656D2F004C6F63617469BE
:100D30006F6E3A20687474703A2F2F6C617A7968FC
:100D40006F6D652E72752F707761003F6D61633D29
:100D5000002669703D0026706F72743D00266E613A
:100D60006D653D002F002000436F6D706C657465EC
:100D70002E2052656D6F766520746F706963200058
:100D800024636F6D6D616E6400536B697070696E82
:100D9000672E2E00436C65616E557020726574611C
:100DA000696E656420746F70696320002200220000
:100DB0004F75744F664D656D6F727921005D20002F
:100DC0003A5B000A005D00456D7074793A205B0063
:100DD0000A003A004D41433A00554450205379737C
:100DE0006C6F6720696E697469616C697A65642EDD
:100DF0000A005379736C6F6720706172616D733A8A
:100E00000043757272656E74204C414E20636F6EA4
:100E10006669672869702C646E732C67772C73750C
:100E2000626E6574293A000A5573652074686573AB
:100E30006520636F6D6D616E64733A202768656C21
:100E40007027202D207468697320746578740A27D0
:100E50006D61632064653A61643A62653A65663A39
:100E600066653A3030272073657420616E642073A4
:100E7000746F7265204D41432D61646472657373B4
:100E800020696E20454550524F4D0A276970205BFE
:100E900069705B2C646E735B2C67775B2C73756277
:100EA0006E65745D5D5D5D27202D20736574207314
:100EB00074617469632049500A277361766527203D
:100EC0002D20736176652063757272656E74206380
:100ED0006F6E66696720696E204E5652414D3B2009
:100EE0004F4E7C4F4646202D20656E61626C652F0B
:100EF00064697361626C65206175746F7361766596
:100F00000A2767657427205B636F6E6669672061D7
:100F10006464725D27202D2067657420636F6E66A0
:100F200069672066726F6D207072652D636F6E66E3
:100F30006967757265642055524C20616E64207338
:100F4000746F726520616464722C204F4E7C4F4632
:100F500046202D20656E61626C652F646973616245
:100F60006C6520646F776E6C6F6164206F6E2073A8
:100F70007461727475700A276C6F616427202D206C
:100F80006C6F616420636F6E6669672066726F6D57
:100F9000204E5652414D0A2770776427202D206439
:100FA0006566696E6520616E642073746F7265207A
:100FB0004D5154542070617373776F72640A276FB8
:100FC000746170776427202D20646566696E6520E2
:100FD000616E642073746F726520485454502041D0
:100FE00050492070617373776F72640A276C6F6762
:100FF000205B73657269616C5F6C6F676C657665A9
:101000006C5D205B7564705F6C6F676C6576656C9A
:101010005D27202D20646566696E65206C6F6720F2
:101020006C6576656C2028302E2E37290A276B696F
:101030006C6C27202D20746573742077617463684D
:10104000646F670A27636C65617227202D20636CCB
:1010500065617220454550524F4D0A277365617294
:10106000636827202D2073656172636820312D77B6
:10107000697265206465760A277265626F6F7427EE
:10108000202D207265626F6F7420636F6E74726FB3
:101090006C6C657200536F6674207265626F6F745A
:1010A000696E672E2E2E00206E65770020697320F2
:1010B000003157543A003157543A205365617263F6
:1010C00068696E67206465760052414D3D000A53A1
:1010D00079736C6F6720000A312D77697265200083
:1010E0000A6D71747420000A696E70757473200043
:1010F0000A6974656D7320000A436F6E66696775CF
:101100007265643A003157543A20736574757020E3
:101110007265736F6C7574696F6E20003157543A45
:10112000204453323438322D313030206E6F7420E9
:1011300070726573656E74003157543A20445332AF
:101140003438322D31303020493243207265737487
:101150006F7265640009445332343832207265730B
:101160006574206572726F72000952657365742030
:10117000646F6E650009436865636B696E6720661E
:101180006F7220312D5769726520646576696365D9
:10119000732E2E2E003157543A20445332343832B5
:1011A0002D3130302070726573656E740045727237
:1011B0006F7220312D7720696E6974004672656503
:1011C0003A004453323438325F3130305F49324371
:1011D0005F544F5F31575F42524944474520696E23
:1011E0006974003B003D0050696E3A003B003D4C85
:1011F0004F5700546865726D6F3A004F6E652077E7
:101200006972652052656164790A004170706C7979
:10121000696E6720636F6E66696700436F6E66690B
:1012200067206175746F736176653A000A5379734C
:101230006C6F67206465627567206C6576656C3AD3
:101240000053657269616C206465627567206C6526
:1012500076656C3A0053617665640A0053657420C4
:1012600064796E616D69632049500A0045455052AA
:101270004F4D20636C65617265640A004D51545492
:101280002050617373776F72642075706461746548
:10129000640A004F54412050617373776F72642069
:1012A000757064617465640A00636F756C64206EA8
:1012B0006F742070617273653A20005570646174B8
:1012C00065640A004E6F2049502061647265737333
:1012D0000052656C656173696E6720736F636B653F
:1012E0007420616E64207265747279002053617697
:1012F0006564004C6F6164696E67204854545020E7
:10130000636F6E666967206F6E20737461727475A7
:10131000703A004F4646004F4E002B002D004554BA
:1013200061673A200047657420455441473A2000E0
:10133000485454502F312E310025733A2025730D17
:101340000A0020485454502F312E310D0A486F7333
:10135000743A2025730D0A4163636570743A202A3C
:101360002F2A0D0A436F6E6E656374696F6E3A20A3
:10137000636C6F73650D0A0025730020000D0A0071
:10138000474554006661696C656420746F20636F23
:101390006E6E6563740A004552524F523A2053658F
:1013A000727665722072657475726E656420004392
:1013B0006F6E666967206E6F74206368616E676523
:1013C000640A00446F6E652E0A00436F6E6669679B
:1013D0002070617273696E67206661696C65640A6A
:1013E00000676F7420436F6E6669670A00687474E3
:1013F0007020726574636F64652000667265652095
:1014000000436F6E666967205552493A20687474CC
:10141000703A2F2F002044656661756C7420636FED
:101420006E66696720736572766572207573656490
:101430003A20006C617A79686F6D652E7275000ACA
:10144000282D294D554C544956454E54000A282BF9
:101450002950574D5F52454C4159000A282D294DBE
:10146000444E53000A282D295541525442524944B2
:101470004745000A282B295359534C4F47000A2847
:101480002D29504944000A282D294D43503233302C
:101490003137000A282D294152544E4554000A285C
:1014A0002B294F5441000A282D29535049204C45DF
:1014B00044000A282D294D4F544F522043545200C6
:1014C0000A282D294143204841494552000A282D28
:1014D00029434353383131202620484443313038A2
:1014E00030000A282B29524553544152545F4C4135
:1014F0004E5F4F4E5F4D5154545F4552524F5253C1
:10150000000A282D294841524452455345542C2065
:101510007573696E6720736F6674000A282B294300
:101520004F554E544552000A282D29444854000A6C
:10153000282B294453323438322D313030000A28D8
:101540002B294F57495245000A282D2949504D4F04
:1015500044425553000A282D294D4F44425553000B
:101560000A282D29444D58000A282B2957697A6EDC
:10157000657435783030000A282B2946726565522B
:10158000616D207072696E74696E67000A282B297C
:101590005741544348444F47006C617A79686F6DF6
:1015A000652E7275000A436F6E66696720736572F7
:1015B0007665723A003230313130334C0020432BA3
:1015C0002B2076657273696F6E3A00326532313363
:1015D00036325F323032332D31312D3132000A4C08
:1015E000617A79686F6D652E7275204C69676874D1
:1015F00048756220636F6E74726F6C6C6572200048
:10160000204F464600204F4E002042595041535330
:1016100000757074696D65006672656568656170F6
:10162000002054696D65723A00204C6F636B733A09
:10163000002000204C6F636B733A000A52414D3D0D
:101640000020457870697265640A00202D7461720B
:10165000676574207A6F6E652D0020416C61726D34
:1016600020457870697265640A0020636D643A00F1
:10167000204375723A00205365743A0053617665D1
:101680006420746F20454550524F4D005361766978
:101690006E6720636F6E66696720746F20454550E2
:1016A000524F4D2E2E004C6F6164656420455441AD
:1016B000473A004E6F2073746F72656420636F6EDB
:1016C000666967004C6F616465642066726F6D20A7
:1016D000454550524F4D006C6F6164206661696CE6
:1016E0006564004A534F4E20646574656374656495
:1016F000004C6F6164696E6720436F6E6669672096
:1017000066726F6D20454550524F4D00556E6B6EA1
:101710006F776E207375666669782000556E6B6E04
:101720006F776E20636D642000436F756E74657211
:101730003A200020696E69740052656C61792D4F02
:1017400075742023002073746F700052656C61798A
:101750002D4F75742023003D3E003A0070756220C5
:10176000616374696F6E200069646C65006F666602
:101770000068656174696E670066616E0064727905
:10178000696E6700636F6F6C696E67002069732014
:10179000004F75742000556E6B6E6F776E207375F9
:1017A000666669782000556E6B6E6F776E20636D8C
:1017B000642000616374696F6E0072656C617943C7
:1017C00074723A20002072656164206572726F72D3
:1017D00020666F7220003E2000203C003157543AB2
:1017E000003157543A206E6F7420696E697400316D
:1017F00057543A206C6F7374204453323438322D6E
:10180000313030003157543A206572726F720031B6
:1018100057543A20312D776972652073686F72745E
:101820006564003157543A204453323438325F45AE
:1018300052524F525F434F4E464947003157543A38
:1018400020312D776972652073686F72746564004A
:101850005B305D3A2000202D202D202D20EFBBBFD6
:10186000003E003E31202D200020002E00696E0039
:10187000735F6F7574006D79686F6D6500435452C6
:101880004C2F657865633A204F75744F664D656DD2
:101890006F72793A2000202D3E2000456D69743A20
:1018A0002000202D3E20004974656D436D643A2070
:1018B00000202D3E20004974656D3A2000094453F4
:1018C00032343832207265736574206572726F72BB
:1018D0000009526573657420646F6E6500005EBC1C
:1018E000E2613FDD83C29C7E20A3FD1F419DC32199
:1018F0007FFCA2401E5F01E3BD3E6082DC237D9F32
:10190000C1421CFEA0E1BF5D0380DE3C62BEE0027E
:101910005CDF81633D7C22C09E1D43A1FF4618FA17
:10192000A427799BC584DA3866E5BB5907DB856750
:1019300039BAE406581947A5FB7826C49A653BD9FD
:1019400087045AB8E6A7F91B45C6987A24F8A64436
:101950001A99C7257B3A6486D85B05E7B98CD230E3
:101960006EEDB3510F4E10F2AC2F7193CD114FAD00
:10197000F3702ECC92D38D6F31B2EC0E50AFF113C9
:101980004DCE90722C6D33D18F0C52B0EE326C8EE6
:10199000D0530DEFB1F0AE4C1291CF2D73CA9476A7
:1019A00028ABF517490856B4EA6937D58B5709EBC8
:1019B000B536688AD495CB2977F4AA4816E9B75585
:1019C0000B88D6346A2B7597C94A14F6A8742AC8AE
:1019D00096154BA9F7B6E80A54D7896B353E3E20D9
:1019E00000496E76616C696420636F6D6D616E6431
:1019F000003E3E3E004E6F204D414320636F6E66B9
:101A00006967757265643A20736574206669726DE2
:101A1000776172652773204D41430A004545505256
:101A20004F4D207369676E6174757265206F6B002E
:101A3000496E697469616C697A696E6720454550C1
:101A4000524F4D2E00476F742049502061646472DC
:101A50006573733A00276970205B69705B2C646E54
:101A6000735B2C67775B2C7375626E65745D5D5D6F
:101A70005D27202D20736574207374617469632061
:101A800049500A004661696C656420746F20636F79
:101A90006E6669677572652045746865726E6574F7
:101AA000207573696E6720444843502E20596F7526
:101AB0002063616E20736574206970206D616E759E
:101AC000616C6C792100204D41534B3A00204757FF
:101AD0003A0020444E533A004C6F616465642066BE
:101AE000726F6D20666C6173682049503A000A7508
:101AF00073657320444843500A00537461727469DB
:101B00006E67206C616E0041424344454647484938
:101B10004A4B4C4D4E4F50515253545556575859AD
:101B20005A6162636465666768696A6B6C6D6E6F43
:101B3000707172737475767778797A3031323334A4
:101B400035363738392B2F3D0042617369632000E9
:101B500061726475696E6F3A004F544120696E6915
:101B60007469616C697A65640A0044454641554C64
:101B7000542070617373776F726420666F72204FA8
:101B80005441204150492E20557365206F74617077
:101B9000776420636F6D6D616E6420746F20736570
:101BA000740070617373776F726400546F6F206D8F
:101BB000616E79204D51545420636F6E6E6563746D
:101BC000696F6E206572726F72732E205265737426
:101BD000617274204C414E002074727920616761FB
:101BE000696E20696E2035207365636F6E647300C3
:101BF0006661696C65642C2072633D0041776169A0
:101C000074696E6720666F722072657461696E65B3
:101C10006420746F7069637300636F6E6E656374C4
:101C200065642061732000202E2E2E0020757365C0
:101C3000723A003A000A417474656D7074696E6797
:101C4000204D51545420636F6E6E656374696F6EDE
:101C500020746F2000646973636F6E6E65637465D2
:101C600064005573696E67204D5154542070617340
:101C700073776F72642066726F6D20636F6E666932
:101C80006700446576696365204E616D653A004181
:101C900074206C6561737420646576696365206E79
:101CA000616D6520616E642062726F6B65722049A0
:101CB00050206D75737420626520636F6E6669676E
:101CC0007572656400757074696D652C6672656502
:101CD0006865617000247374617473003265323119
:101CE0003336325F323032332D31312D3132004CC8
:101CF000696768744875622000246E616D650072C2
:101D00006561647900247374617465005265626969
:101D10006E6420737563636573732E204950206170
:101D20006464726573733A004572726F723A20721E
:101D30006562696E64206661696C0052656E6577E4
:101D4000656420737563636573732E204950206149
:101D50006464726573733A004572726F723A2072EE
:101D6000656E65776564206661696C000A4E6F2058
:101D70006C696E6B0033307320454550524F4D20D7
:101D80006973206E6F742072656C6F616465642E78
:101D9000205265626F6F7400416363657074696E91
:101DA0006720636F6D6D616E64732E2E2E0A004E78
:101DB0006F204D51545420636F6E6669677572656C
:101DC00064004C6F6164696E6720636F6E6669675B
:101DD0002066726F6D20706F7274616C206469731D
:101DE00061626C65642E2075736520676574204F91
:101DF0004E20746F20656E61626C6500436F6E6685
:101E000069672069732076616C696400436F6E7442
:101E1000696E756520776974682070726576696F80
:101E200075736C79206C6F6164656420636F6E6696
:101E300069670000002100240027002A002D0030DF
:101E400000330001010000040107010A0100002223
:101E500000250028002B002E003100340002010074
:101E600000050108010B010505050507050808081F
:101E700008020202020A0A0808040404040101011B
:101E80000101010101030303030303030304070723
:101E9000070C0C0C0C0C0C0C0C02020202060606C1
:101EA00006060606060B0B0B0B0B0B0B0B010210A9
:101EB0002020080810204010204080020102010864
:101EC0000402010102040810204080804020100814
:101ED000040201800402018040201008040201086D
:101EE00004020101020408102040800102040810CD
:101EF00020408000000A0B02090C0D0E08070304A5
:101F000001000000000000000000000000000000D0
:101F100000000000000000000000000000000012AF
:101F20001110000000000000000000000000000090
:101F30000000000000000000002F64617461002FA9
:101F4000736B65746368004163636573732D436FDE
:101F50006E74726F6C2D526571756573742D50724D
:101F600069766174652D4E6574776F726B3A207473
:101F7000727565004163636573732D436F6E747290
:101F80006F6C2D416C6C6F772D4865616465727361
:101F90003A202A004163636573732D436F6E747238
:101FA0006F6C2D416C6C6F772D4D6574686F647329
:101FB0003A20504F53542C4745542C4F5054494FBE
:101FC0004E53004163636573732D436F6E74726F7C
:101FD0006C2D416C6C6F772D43726564656E74690E
:101FE000616C733A2074727565004F5054494F4EBE
:101FF000530044454C455445005055540047455402
:1020000000504F535400617574686F72697A61743F
:10201000696F6E3A2000417574686F72697A6174F5
:10202000696F6E3A2000436F6E74656E742D4C6557
:102030006E6774683A20006F637465742F737472EE
:1020400065616D00696D6167652F6A70656700691C
:102050006D6167652F67696600746578742F6874B1
:102060006D6C006170706C69636174696F6E2F6A6A
:10207000736F6E00746578742F706C61696E0043C5
:102080006F6E74656E742D547970653A2000436FDD
:102090006E6E656374696F6E3A20636C6F73650072
:1020A0004163636573732D436F6E74726F6C2D4162
:1020B0006C6C6F772D4F726967696E3A202A0055F4
:1020C0006E6B6E6F776E004E6F74204D6F64696635
:1020D000696564004F4B004D6F76656420706572D2
:1020E0006D616E656E746C7900496E7465726E61B7
:1020F0006C20536572766572204572726F72005063
:1021000061796C6F616420546F6F204C61726765F8
:10211000004E6F7420666F756E64005757572D41DF
:10212000757468656E7469636174653A20426173A1
:102130006963207265616C6D3D22416363657373F1
:1021400020726573747269637465642200556E61F0
:102150007574686F72697A6564005061796C6F613B
:10216000642073697A652077726F6E6700426164DC
:10217000207265717565737400485454502F312E68
:1021800031200020000000000000000000004F4E41
:10219000000000000000004F464600000000000064
:1021A000524553540000000000544F47474C45002F
:1021B000000048414C540000000000584F4E000001
:1021C00000000000584F46460000000000494E4302
:1021D000524541534500444543524541534500450E
:1021E0004E41424C4500000044495341424C450099
:1021F00000554E465245455A4500465245455A45BA
:102200000000004155544F000000000046414E5F61
:102210004F4E4C59004849474800000000004D45CA
:102220004449554D0000004C4F570000000000008D
:10223000484541540000000000434F4F4C0000004F
:10224000000044525900000000000053544F500059
:1022500000000000524742000000000000485356B2
:1022600000000000000057726F6E67207061796C8B
:102270006164004354524C2F7478743A204F757443
:102280004F664D656D6F72793A2000202D3E2041DA
:10229000543A004368616E20747970653A004E6F5D
:1022A0002073746F7265642076616C756573202D80
:1022B0002064656661756C743A20002D3E0050758F
:1022C000623A20006374726C00454E41424C4500F6
:1022D000465245455A450044495341424C45002D1C
:1022E0003E005075623A2000636D640046414E5FC7
:1022F0004F4E4C590044525900434F4F4C004845F3
:102300004154004155544F002D3E005075623A2013
:10231000007365740064656C002D3E005075623A70
:1023200020002D3E005075623A2000556E6B6E6F96
:10233000776E20636D64200A004F4646004F4E00C2
:10234000536176656420455441473A0053657420D3
:10235000455441473A20000014C64FB411241FBE13
:10236000CFEFD1E2DEBFCDBF00E00CBF15E0A0E0B3
:10237000B2E0E6EFF5EB01E00BBF02C007900D9273
:10238000A63FB107D9F72BE0A6EFB5E001C01D923B
:10239000AB34B207E1F711E1CDEAD1E100E006C0CC
:1023A00021970109802FFE010E94CBD2CC3AD107A0
:1023B00080E00807A9F70E9461B40C94E9DA0C9454
:1023C0000000CF93DF931F92CDB7DEB76983DC01A6
:1023D000ED91FC910280F381E02D41E050E0BE01DF
:1023E0006F5F7F4F19950F90DF91CF910895FC019A
:1023F000818D928D0895CF93DF931F92CDB7DEB775
:102400006983DC01ED91FC910280F381E02D41E0D4
:1024100050E0BE016F5F7F4F19950F90DF91CF9114
:102420000895FC019485FB018485981303C081E025
:10243000983008F080E00895CF93DF931F92CDB7D6
:10244000DEB76983DC01ED91FC910280F381E02D20
:1024500041E050E0BE016F5F7F4F19950F90DF9113
:10246000CF910895FC01818191E09093A60880931B
:10247000C8081092A7081092C90808952091C706AD
:10248000260F3327331F21323105ECF42091A008A9
:10249000FC0190E080E0243069F082E00895A09192
:1024A000C7062191AC014955594FA40FB52FB11D55
:1024B0002C930196861798F38091C706680F609356
:1024C000C70680E0089581E0089508950895E09199
:1024D000790880917808E81730F4F0E0E651F94F78
:1024E000808190E008958FEF9FEF08959091790893
:1024F000809178082FEF3FEF981748F4E92FF0E02C
:10250000E651F94F208130E09F5F90937908C9012F
:1025100008958091780890917908891B990B089506
:10252000CF92DF92EF92FF920F931F93CF93DF939F
:102530007C01CB018A012091A608222389F0EB01BE
:102540006B01C40ED51ECC15DD0569F06991D7016C
:10255000ED91FC910190F081E02DC7011995F3CF29
:10256000642F0E943E12C801DF91CF911F910F91FD
:10257000FF90EF90DF90CF900895CF93DF931F925D
:10258000CDB7DEB769832091A6082223F9F0209108
:10259000C908203258F021E030E0FC013383228367
:1025A00090E080E00F90DF91CF9108958091A7088F
:1025B000E82FF0E0E855F74F998190838F5F809383
:1025C000A7088093C90881E090E0ECCF61E0CE01DC
:1025D00001960E943E12F7CF90E0FC01E959F14EBE
:1025E000E491F0E0EE0FFF1FE35BF14EA591B49193
:1025F0002C918355914EFC018491822391E009F442
:1026000090E0892F0895FC01DC018D918111FDCFAF
:1026100030E020E050E040E08AE09191992301F120
:10262000443051055CF59E3271F42F3F310509F0BD
:102630002CF5DB01A40FB51F12962C934F5F5F4F53
:1026400030E020E0EACF829FD001839FB00D1124BB
:10265000292F990F330B205331092A0F3B1FDDCF50
:102660002F3F310509F054F4443051053CF4640F18
:10267000751FFB01228381E090E0089590E080E0E7
:1026800008950097B1F1FC01DB01AC01405F5F4FA1
:1026900080E090812FE9290F263098F49755929584
:1026A000907F9C9321813FE9320F3630B0F427555B
:1026B000922B9D933296E417F50759F791E08927FD
:1026C00008952FEB290F263010F49753E8CF90533D
:1026D0009A3028F381E090E0E2CF3FEB320F3630C2
:1026E00010F42753E5CF20532A3010F381E020E087
:1026F000DFCF80E00895DC0115968D919C910097C5
:1027000039F0DC01ED91FC910680F781E02D199400
:1027100008950097D1F0DC011696ED91FC91309769
:10272000A1F080858F70843021F481859285009797
:1027300071F40680F781E02D309739F080858F7035
:10274000843019F481859285089590E080E00895A1
:10275000089583E090E00895089584E190E008955D
:10276000DC01ED91FC910684F785E02D60E0199580
:1027700081E090E008958FE090E0909316078093B9
:10278000150788EC90E00895FC01848195810895F7
:10279000FC01768765870895DC01ED91FC91068C3C
:1027A000F78DE02D199591E089270895862F0895DA
:1027B00081E08627089521E0FC018485883008F0B7
:1027C00020E0822F0895FC01848595850895FC0101
:1027D0008489958908952BED33E0FC0131832083B2
:1027E000FB014089518962897389FC0142835383CB
:1027F000648375830895DC01ED91FC91048CF58D63
:10280000E02D1994DC011196EC911197E295EF708F
:10281000E150EB3008F039C0F0E08827ED5EFB4E68
:102820008F4F0C94CBD23614361445141E141E143C
:1028300027143E143E143E141E141E1414966D915B
:102840007D918D919C9117970E94FDD008951496CB
:102850006D917D918D919C91179724E630E040E039
:1028600050E00E9462D2CA01B901EECF14966C9179
:1028700070E090E080E00E94FBD0089514966D9186
:102880007D918D919C911797089560E070E0CB0148
:102890000895DC011196EC911197E295EF70E150EB
:1028A000EB3008F03EC0F0E08827E65AFB4E8F4F31
:1028B0000C94CBD2701470149114651465148A149E
:1028C0007B147B147B146514651414962D913D9133
:1028D0004D915C911797A4E6B0E00E9481D20895D3
:1028E00014966C9184E6689FB0011124072E000CA9
:1028F000880B990B089520E030E048EC52E41496E0
:102900006D917D918D919C9117970E945CD10E9451
:10291000C8D3089514966D917D918D919C911797D0
:10292000089560E070E0CB010895FC01A7812A2F93
:102930002E7FD1F0818182958F7081508330A0F4F9
:10294000A695A150BB0B2BE531E00E94E2D224E614
:1029500030E040E050E00E9462D2DA01C9018756BF
:102960009F4FAF4FBF4F08958FEF9FEF0895DC014A
:10297000ED91FC91309729F090859F7081E0953022
:1029800009F080E00895FC01A481B581109721F140
:1029900018969C9118979F708EEF890F823010F0D7
:1029A00091111AC019964D935D936D937C931C976A
:1029B000A481B58118969C911897907F9260189683
:1029C0009C930480F581E02D8085982F907F903630
:1029D00019F48F70806A80870895DC0119968D91B3
:1029E0009C91009739F0DC01ED91FC910280F3811C
:1029F000E02D19940895FC01238130E090E080E0FF
:102A0000FC01EE0FFF1FE85DF94FA081B181A21715
:102A1000B30761F4880F991F880F991FFC01EC5EC2
:102A2000F94F40835183628373830895A081B181FC
:102A3000AB2B19F420813181EDCF019685309105C2
:102A4000F9F60895FC01238130E090E080E0FC017C
:102A5000EE0FFF1FE85DF94F408151814217530788
:102A600061F4880F991F880F991FFC01EC5EF94FE4
:102A70006081718182819381089540815181452BCC
:102A800089F431832083880F991F880F991FFC01D7
:102A9000EC5EF94F108211821282138260E070E0C6
:102AA000CB01089501968530910589F6F7CF880FFF
:102AB000991F880F991FFC01E450FA4F8081918182
:102AC000A281B3810196A11DB11D80839183A28350
:102AD000B383089585E090E00C94571584E090E06E
:102AE0000C94571583E090E00C94571582E090E029
:102AF0000C94571581E090E00C94571590E080E01D
:102B00000C945715CF93DF93EC01E881F98104848D
:102B1000F585E02D199529893A892F5F3F4F3A8B2A
:102B2000298BDF91CF910895CF93DF93EC018E85B0
:102B300081110DC081E090E049895A892C853D853D
:102B40004217530708F080E0DF91CF910895E881A4
:102B5000F9810484F585E02DCE0119958F3F91050B
:102B600049F780E090E0F0CFFC01848595856817F7
:102B7000790708F4CB01928B818B0895DC011E96B6
:102B80002C911E97222339F0ED91FC910190F08158
:102B9000E02D6FEF19940895FC01878590890895C1
:102BA00081E0089590E080E00895DC011296ED91B7
:102BB000FC91309761F00190F081E02D309739F071
:102BC000862F8295807F60856F70682B608708955F
:102BD000DC011296ED91FC91309751F00190F0815B
:102BE000E02D309729F0808582958F7090E00895D0
:102BF00090E080E00895CF93DF93CDB7DEB7609784
:102C00000FB6F894DEBF0FBECDBF19821A821B82A9
:102C10001C821D821E821F8218868A818F708061AD
:102C20008A836FEF3E819F81888529817A815B81CC
:102C30004C814C873E87888B372F452F5C857E855E
:102C4000892F988960960FB6F894DEBF0FBECDBF6E
:102C5000DF91CF9108950F931F93CF93DF9300D00F
:102C600000D01F921F92CDB7DEB781E028960FB635
:102C7000F894DEBF0FBECDBFDF91CF911F910F91B2
:102C80000895CF92DF92EF92FF920F931F93CF930D
:102C9000DF9300D000D0CDB7DEB78C016B017A0195
:102CA000FC01808D883010F40E94BE928BED93E081
:102CB0009A838983F60182819381A481B5818B8374
:102CC0009C83AD83BE83B701CE0101960E94CDA146
:102CD000F801808F8830A0F4F586E486128E118E7C
:102CE00081E026960FB6F894DEBF0FBECDBFDF9110
:102CF000CF911F910F91FF90EF90DF90CF900895AB
:102D000080E0EFCFCF93DF93EC01888D883020F403
:102D10000E94BE9288E0888FDF91CF910895FC01D8
:102D2000808D883040F4218D328D232B21F00E943C
:102D3000909190E008958FEF9FEF0895CF93DF93E8
:102D4000FC012485283028F08FEF9FEFDF91CF9191
:102D50000895EC010190F081E02D0084F185E02DD3
:102D60001995892B89F38C850E94909190E0EECF84
:102D7000CF93DF93FC01218D328D2115310529F48C
:102D80008FEF9FEFDF91CF910895EC01808D421777
:102D9000530708F0A9010E94DF911816190684F75D
:102DA000298D3A8D281B390B3A8F298FEBCF0F9342
:102DB0001F93CF93DF931F92CDB7DEB7FC01218D18
:102DC000328D232B41F48FEF9FEF0F90DF91CF9146
:102DD0001F910F9108958C0141E050E0BE016F5F9B
:102DE0007F4FFC01808D0E94DF91181619065CF759
:102DF000F801818D928D0197928F818F898190E06A
:102E0000E4CFCF93DF931F92CDB7DEB741E050E020
:102E1000BE016F5F7F4FFC0184850E94DF91181611
:102E2000190634F4898190E00F90DF91CF910895D5
:102E30008FEF9FEFF9CFFC018485883010F40C945C
:102E4000DF9190E080E00895FC018485883010F4E3
:102E50000C94B89190E080E008950F931F93CF9366
:102E6000DF9300D000D01F921F92CDB7DEB78C0148
:102E7000D80159964D915C915A974115510551F0E1
:102E8000ED91FC91048CF58DE02D70E060E0C801BF
:102E90001995EECFF801808D0E94B891892BB1F180
:102EA00048E050E0BE016F5F7F4FD80158968C918B
:102EB0000E94DF9118161906F4F4D801509684E0A8
:102EC000FE01319601900D928A95E1F78D8190E097
:102ED000982F88272E81820F911DF801958B848B66
:102EE0008F81282F30E0322F22278885820F932F61
:102EF000911D928F818F28960FB6F894DEBF0FBE7A
:102F0000CDBFDF91CF911F910F91089590E080E0A8
:102F1000F2CFCF92DF92EF92FF920F931F93CF9356
:102F2000DF93CDB7DEB7AF970FB6F894DEBF0FBE15
:102F3000CDBF7C016A010BED13E01A8309831C8667
:102F40001B8688EE93E0A0E0B0E08D879E87AF8778
:102F5000B88B81EB93E09A878987188F0F8B198E36
:102F60001A8E1B8E1C8E88E089A31BA70AA71CA69D
:102F70001DA61EA61FA68091F3089091F408A091AB
:102F8000F508B091F6088EA39FA3A8A7B9A78B83D5
:102F90009C83AD83BE8318861F82AE01465D5F4F62
:102FA000CE0101960E94C4AA81309105B1F4D701E7
:102FB000ED91FC910488F589E02D1DA30CA38CA54F
:102FC0009DA5AEA5BFA58EA39FA3A8A7B9A7A6013F
:102FD000BE016C5D7F4FC7011995AF960FB6F8948F
:102FE000DEBF0FBECDBFDF91CF911F910F91FF903C
:102FF000EF90DF90CF9008950F931F93CF93DF93BF
:10300000EC018B01888D883010F40E94BE92B801CB
:1030100082E00E940793888F883050F41D870C87C8
:103020001A8E198E81E0DF91CF911F910F91089533
:1030300080E0F9CF0F931F93CF93DF938C01EA01C8
:10304000FC018485883048F40E942E91892B39F444
:1030500081E090E0F80193838283D0E0C0E0CE016C
:10306000DF91CF911F910F910895EF92FF920F93EF
:103070001F93CF93DF937C0180916208D4E0833368
:1030800009F0D8E002E518E0C0E0F80121913191A3
:103090008F01F701848195812817390729F0CF5FC7
:1030A000DC13F3CF80E006C08C2F0E94CC928431D9
:1030B000B1F781E0DF91CF911F910F91FF90EF90D9
:1030C0000895CF93DF93EC018C858830D0F40E9473
:1030D000CC92843189F0882379F0883169F021E03D
:1030E0008C3159F4E881F9810084F185E02DCE011D
:1030F000199521E0892B09F420E0822FDF91CF91EF
:10310000089580E0FBCFCF92DF92EF92FF920F9372
:103110001F93CF93DF93CDB7DEB7AF970FB6F89479
:10312000DEBF0FBECDBF8C016B017A018BED93E04A
:103130009A8389831B821C821D821E821C861B86A9
:1031400048EE53E060E070E04D875E876F87788BD4
:1031500021EB33E03A872987988F8F8B198E1A8E4F
:103160001B8E1C8E28E029A39BA78AA71CA61DA640
:103170001EA61FA6D8011C968C91883060F40E9470
:10318000CC92882321F0F80184850E94B09288E0D7
:10319000D8011C968C938091F3089091F408A0912B
:1031A000F508B091F6088EA39FA3A8A7B9A78B83B3
:1031B0009C83AD83BE8318861F82AE01465D5F4F40
:1031C000B601CE0101960E94C4AA0097C1F0D801B1
:1031D000ED91FC910684F785E02D8BED93E09DA3A6
:1031E0008CA38CA59DA5AEA5BFA58EA39FA3A8A7C4
:1031F000B9A7A701BE016C5D7F4FC8011995AF96B5
:103200000FB6F894DEBF0FBECDBFDF91CF911F91F7
:103210000F91FF90EF90DF90CF9008950F931F9341
:10322000182F0E94ECA404C0969587957795679512
:103230001A95D2F78B019C0101501109210931091E
:103240000E3F1F4F2F4F3F4F20F061E070E080E0B6
:1032500090E01F910F910895CF93DF93EC018C853F
:10326000883060F40E94CC92873111F08C3131F4B7
:103270008C850E9411918115984088F3DF91CF9140
:103280000895FC018485883010F40C94119190E02D
:1032900080E00895CF93C62F0E94321261EE87EF2F
:1032A00098E00E94BD126C2F87EF98E00E94BD123B
:1032B000CF910C94B6A40E94321281E00E94C6A362
:1032C00091E0811190E0892F0895ECEBF0E080818E
:1032D0008A7B808360E084E10E941AA360E085E13C
:1032E0000C941AA3CF93DF93EC016BE477E187E3AF
:1032F0009AE00E94C9856C817D8187E39AE00E94F3
:10330000D19B65E477E187E39AE00E94C98587E372
:103310009AE00E94DA8360E08C810E9448A3E881F1
:10332000F9810684F785E02D60E0CE01199581E0F2
:1033300090E0DF91CF910895EF92FF921F93CF938A
:10334000DF93192F7B01C82FD92FD7FF03C0D19549
:10335000C195D10961E08C2F0E9448A382E0E81654
:10336000F10499F460E08C2F0E941AA369E076E1E1
:1033700087E39AE00E94C98587E39AE0DF91CF91C5
:103380001F91FF90EF900C94DA83612FEF2851F496
:103390006095661F6627661F8C2F0E941AA365E042
:1033A00076E1E6CF661F6627661F8C2F0E941AA360
:1033B00060E076E1DDCF6AE173E1811102C06CE18A
:1033C00073E186E899E00C94C98565E970E186E8C7
:1033D00099E00E94C985F0E0E0E0199584EF91E062
:1033E00008956FE37AE0811102C06AE37AE087E32F
:1033F0009AE00C94C985DC0155962C915597273796
:1034000081F4ED91FC91008CF18DE02D199565EA28
:1034100076E087E39AE00E94C98587E39AE00C94FE
:10342000DA8308954F925F926F927F92AF92BF922C
:10343000DF92EF92FF920F931F93CF93DF9300D011
:1034400000D0CDB7DEB77C01D62E8091A1068823AF
:1034500009F4BEC0D70114969C918091000289178F
:1034600008F4B6C080919F069091A006BAE06B1355
:10347000F0C0815B994FFC011082D70118960D9125
:103480001C910115110509F49FC0F8016185728531
:103490006115710591F44580568067807084809134
:1034A000ED089091EE08A091EF08B091F008481651
:1034B00059066A067B0609F487C0D8011B964D9110
:1034C0005C911C974115510509F47EC0F7012481D8
:1034D00053968C91539790E0322F377002C0959598
:1034E00087953A95E2F780FF6FC0A22EB12CC501F7
:1034F000887F9370892B39F451968D919C91887FA8
:103500009370A82AB92AD8018D919C91DC01ED9184
:10351000FC916115710509F486C00688F789E02DD4
:103520001995019709F050C06CE3F80180819181F1
:103530000E94F083A50170E060E02AE0D8018D913F
:103540009C910E948E83F80122818081918163E6A3
:1035500078E1222311F061E678E10E94C985D80163
:103560001D966D917C911E978D919C910E94638513
:1035700060E2F801808191810E94F083D8011F965A
:103580006D917C9150978D919C910E946385F8017B
:1035900022818081918166E578E1222311F060E546
:1035A00078E10E94C9856FE476E0D8018D919C9105
:1035B0000E946385F80180819181DC01ED91FC918D
:1035C000008CF18DE02D19951092A00610929F06A7
:1035D000D70115968D919C911697009771F01496CE
:1035E0003C9120910102231740F0DC01ED91FC9108
:1035F0000190F081E02D6D2D199581E090E02696E7
:103600000FB6F894DEBF0FBECDBFDF91CF911F91F3
:103610000F91FF90EF90DF90BF90AF907F906F90F1
:103620005F904F9008950488F589E02D2BED33E0ED
:103630003A832983D80115964D905D906D907C90CA
:1036400018974B825C826D827E82BE016F5F7F4FD6
:1036500067CF8F3491050CF0BBCFBDE06B1709F439
:10366000B7CF9C012F5F3F4F3093A00620939F065A
:10367000815B994FFC016083ABCF0C9464C90C94BF
:1036800064C9CF93C1E068EE73E080E090E00E94EF
:10369000B9A46C2F86E899E00E94CA9BCF5FC43121
:1036A00091F784EF91E0CF910895CF93DF93009746
:1036B00009F490C0FC012081222309F48BC0EC01A5
:1036C00061E173E20E9401CB892B09F45FC064ECD5
:1036D00072E2CE010E9401CB892B09F45AC068EE38
:1036E00072E2CE010E9401CB892B09F455C06DE630
:1036F00077E0CE010E9401CB892B09F450C069E626
:1037000077E0CE010E9401CB892B09F44BC065E61E
:1037100077E0CE010E9401CB892B09F446C061E617
:1037200077E0CE010E9401CB892B09F441C06DE501
:1037300077E0CE010E9401CB892BE9F169E577E0C2
:10374000CE010E9401CB892BC9F164E577E0CE015F
:103750000E9401CB892BA9F160E577E0CE010E94A0
:1037600001CB892B89F165E173E2CE010E9401CB87
:10377000892B69F16CE477E0CE010E9401CB892BA3
:1037800049F58DE090E0DF91CF91089582E090E0DF
:10379000FACF89E090E0F7CF81E090E0F4CF88E0C5
:1037A00090E0F1CF85E090E0EECF86E090E0EBCFC7
:1037B00087E090E0E8CF8AE090E0E5CF8BE090E012
:1037C000E2CF8CE090E0DFCF83E090E0DCCF84E0DC
:1037D00090E0D9CF90E080E0D6CFCF93DF9300D0B8
:1037E00000D01F921F92CDB7DEB7E0E7F9E0128A52
:1037F000118A80E090E19587848784E890E0948B3B
:10380000838B81E0868780E090E2908B878787E7D3
:10381000858B1C821B8281EA92E09A838983FE83D6
:10382000ED838FEF9FEF98878F836CE876E186E8D2
:1038300099E00E94C9856091450670914606CE01C7
:1038400001960E94F18A80E799E00E94FB196CE7DB
:1038500076E186E899E00E94C98586E899E00E94B1
:10386000DA830E94E2AD28960FB6F894DEBF0FBE51
:10387000CDBFDF91CF91089565E0FC0180819181FA
:103880000E94A297009749F0FC018085982F907FB5
:1038900021F082958F7090E0089590E080E0089587
:1038A000FC0186819781009799F0FC0120852F709B
:1038B000223029F4618572858385948508952530A9
:1038C00039F460E00E94A297009711F0FC01F2CF5A
:1038D00060E070E0CB0108950F931F93CF93DF93C7
:1038E000FC01C281D3812097C9F18B0188858F703B
:1038F000853021F5CE010E942E9C8017110671F1B2
:103900006CF1602FCE010E94A297FC01892B31F14E
:1039100080858F70823039F46185728583859485C6
:103920000E94FDD006C08330C9F46185728583850D
:103930009485DF91CF911F910F910895672B71F4BA
:10394000823029F469857A858B859C85E9CF83301F
:1039500029F469857A858B859C85EBCF60E070E0E2
:10396000CB01E7CFCF93C62F63E0FC01808191812B
:103970000E94A297FC01892B11F19085892F8D70EF
:10398000F1F4907F9260908781859285A385B485BC
:103990008827BB278C2B81879287A387B48762E710
:1039A00077E087E39AE00E94C9856C2F87E39AE06D
:1039B0000E94CA9B87E39AE0CF910C94DA83CF915F
:1039C000089563E0FC01808191810E94A297009795
:1039D00019F0FC01818508958FEF0895FF920F93F0
:1039E0001F93CF93DF93CDB7DEB764970FB6F894EC
:1039F000DEBF0FBECDBF8C01F62E8FE290E09A8322
:103A00008983FE01339688E0DF011D928A95E9F7EC
:103A1000F8016681FF2011F081E06827D801149633
:103A20008C910E941AA3F80187819085A185B285A7
:103A3000883E9340A105B10508F48BC061E977E1A8
:103A400087E39AE00E94C985D80114966D917C9114
:103A500087E39AE00E94D19B6CE877E187E39AE0E4
:103A60000E94C9856F2D70E087E39AE00E94D19B88
:103A700087E39AE00E94DA8363EB77E1CE01019657
:103A80000E94F6CAF801828193810E94E11CFF2006
:103A900009F46BC064E877E1843151F06DE777E1B8
:103AA000853131F061E777E18F3011F469E777E133
:103AB000CE010B960E940ACB6CE577E187E39AE092
:103AC0000E94C985D8011296ED91FC91139701903F
:103AD000F081E02D60817181ED91FC910488F58980
:103AE000E02D9E012F5F3F4FAE01455F5F4FC80144
:103AF0001995BC0187E39AE00E94D19B6AE577E1C2
:103B000087E39AE00E94C985D8011296ED91FC9155
:103B10000190F081E02D6081718187E39AE00E943D
:103B20006385BE016F5F7F4F87E39AE00E946385E4
:103B300067E577E187E39AE00E94C985BE01655F8A
:103B40007F4F87E39AE00E94638587E39AE00E94B3
:103B5000DA8364960FB6F894DEBF0FBECDBFDF9157
:103B6000CF911F910F91FF9008956DE677E182301C
:103B700009F49ECF68E677E19BCFDC01ED91FC91E3
:103B80000684F785E02D62E0199581E090E00895C4
:103B9000CF92DF92EF92FF920F931F93CF93DF9319
:103BA000CDB7DEB760970FB6F894DEBF0FBECDBFBE
:103BB0007C016B01CA01B9012AE0AE014F5F5F4F82
:103BC0000E94A5CBD701ED91FC910488F589E02DE9
:103BD0009801AE014F5F5F4FB601C701199560961E
:103BE0000FB6F894DEBF0FBECDBFDF91CF911F910E
:103BF0000F91FF90EF90DF90CF900895892B71F097
:103C0000FB01828193810E94499963E972E186E810
:103C100099E00E94C98588EC90E0089590E080E0EA
:103C2000F2CF892B71F0FB01828193810E94FB9876
:103C30006CE772E186E899E00E94C98588EC90E023
:103C4000089590E080E0F2CFEF92FF920F931F93E0
:103C5000CF93DF93CDB7DEB72C970FB6F894DEBFC6
:103C60000FBECDBF8C017B018BED93E09A838983DE
:103C70001B821C821D821E8298878F8319861A865A
:103C80001B861C8605301105ECF0BE01695F7F4F75
:103C9000F701808591850E940313892B99F0CE014D
:103CA00007960E94EC99BE01695F7F4FF7018681FC
:103CB00097810E940313892B61F0CE0107960E9421
:103CC000969A0EC0CE0101960E94EC99043011051F
:103CD00054F7CE0101960E94969A03301105A4F183
:103CE000BE01695F7F4FF701848195810E940313B4
:103CF000892B51F1CE0107960E94419ABE01695F5E
:103D00007F4FF701828193810E940313892B19F160
:103D1000CE0107960E94979965E572E186E899E0E1
:103D20000E94C98580E00E94809B88EC90E02C96E0
:103D30000FB6F894DEBF0FBECDBFDF91CF911F91BC
:103D40000F91FF90EF900895CE0101960E94419A45
:103D5000023011059CF6CE0101960E949799013020
:103D60001105D1F6CE0101960E9497996CE572E19A
:103D700086E899E00E94C985CFCF0F931F93CF9318
:103D8000DF938C01EB010297C4F08A819B810E9432
:103D900095CA8093010299270E94939B02301105D6
:103DA00049F08C819D810E9495CA809300029927D9
:103DB0000E949D9BC8ECD0E002C0C0E9D1E061E464
:103DC00072E186E899E00E94C9856091010286E867
:103DD00099E00E94CA9B6CE272E186E899E00E9439
:103DE000C9856091000286E899E00E94CA9B86E836
:103DF00099E00E94DA83CE01DF91CF911F910F915C
:103E00000895CF93DF93EB010297A4F167E173E18B
:103E10008A819B810E94E3CA892B29F40E94EB9A34
:103E20006F770E94309B63E173E18A819B810E94DE
:103E3000E3CA892B29F40E94EB9A60680E94309BA8
:103E40006BE172E186E899E00E94C9850E94EB9AD5
:103E50006095661F6627661F70E086E899E00E94FD
:103E6000D19B86E899E00E94DA8388EC90E0DF91AC
:103E7000CF9108950E94ED1BF8CFCF92DF92EF9281
:103E8000FF920F931F93CF93DF93EC016A017B01A5
:103E90008E819F81892BF1F4888199810E942E9CCB
:103EA000082F10E005301105ACF40E94FF8CFC01D6
:103EB000892B19F08085807F808780858F7080872F
:103EC000FF83EE83BF01888199810E94A99B0F5FC8
:103ED0001F4FE8CFEE81FF81309749F18085982F01
:103EE0009F7019F5807F82608087EE81FF81C18697
:103EF000D286E386F4866AE777E087E39AE00E9459
:103F0000C9852AE030E0B701A60187E39AE00E9464
:103F1000DD8487E39AE0DF91CF911F910F91FF90AD
:103F2000EF90DF90CF900C94DA839230F1F2DF9132
:103F3000CF911F910F91FF90EF90DF90CF90089558
:103F40008F929F92AF92BF92CF92DF92EF92FF92A9
:103F50000F931F93CF93DF93EC01888199810E9487
:103F60002E9C082F10E0043011059CF40E94FF8C59
:103F7000FC01892B19F08085807F808780858F7078
:103F80008087BF01888199810E94A99B0F5F1F4F85
:103F9000EACF60E0888199810E94A2977C01009716
:103FA00051F1FC0180858F70843039F5C184D28451
:103FB000C114D10401F1F60180818823E1F080EC85
:103FC000882E8AE0982EB12CA12C1A2DC4010E94B3
:103FD00011CBAC01B401C6010E942ACB892B09F494
:103FE00093C0FFEFAF1ABF0A89E0880E911CE7E18A
:103FF000AE16B10451F71FEF03C08230E1F711850F
:104000001887E880F98061E0C7010E94A2979B832E
:104010008A8362E0C7010E94A2979D838C8364E03B
:10402000C7010E94A2979F838E83103181F01431C3
:1040300009F45CC0DF91CF911F910F91FF90EF9039
:10404000DF90CF90BF90AF909F908F9008958BE0BE
:1040500090E00E94C8C88C01FC01D383C28384E530
:1040600092E0918380831682CE010E943E9C97FD50
:104070002AC0F80195838483F80184819581009793
:1040800019F0863491052CF080E290E0F8019583D8
:10409000848361E070E0CE010E946C1C20E030E07F
:1040A0004AE754E40E945CD10E94CFD361157105A8
:1040B0008105910589F0F801678370878187928770
:1040C0001A870987B7CF919581959109F801958352
:1040D000848381E08683D0CF88E893E1A0E0B0E0DC
:1040E000F80187839087A187B287EACF84E090E0C8
:1040F0000E94C8C8FC01D383C2832EE232E0318320
:1041000020839A87898796CFC6010E947F8A8A2D4D
:1041100090E0B0E0A0E0F70181879287A387B487A1
:104120008085807F826080876BCFCF93DF93EC01A7
:10413000798368831A8619861B861C8E1B8E0E94C3
:10414000B714882329F0CE01DF91CF910C94A01FE2
:10415000DF91CF9108952F923F924F925F926F928D
:104160007F928F929F92AF92BF92CF92DF92EF9207
:10417000FF920F931F93CF93DF93CDB7DEB7629774
:104180000FB6F894DEBF0FBECDBF5C014B01290115
:104190003A01CA01B9010E94C8D31B013F926F9333
:1041A00084E394E09F938F93CE0101967C019F93CB
:1041B0008F930E94B1D70F900F900F900F900F9098
:1041C0000F9020E030E0A901C301B2010E94FED3AC
:1041D000181624F077FA709477F87094F70101902C
:1041E0000020E9F731976F01CE18DF088EE2808357
:1041F000A2E0B0E0AC0FBD1FAC0DBD1DBA8BA98B0A
:10420000B10137FE03C0719561957109072E000C4D
:10421000880B990B0E94FDD09B01AC01C301B20138
:104220000E94E9D220E030E040E251E40E945CD1FB
:104230000E94C8D3605DE989FA896083FE01EC0DB4
:10424000FD1D1382D501ED91FC910488F589E02DC7
:104250009801A701B401C501199562960FB6F894AB
:10426000DEBF0FBECDBFDF91CF911F910F91FF90A9
:10427000EF90DF90CF90BF90AF909F908F907F9006
:104280006F905F904F903F902F9008951F93CF9322
:10429000DF93FC01162FC389D489818992899C01FF
:1042A0002F5F3F4F328B218BC80FD91FCE010E9449
:1042B0001AD2181721F0612FCE010E9422D281E07C
:1042C00090E0DF91CF911F910895FC01818992893F
:1042D000248535858217930740F423893489820F1A
:1042E000931F0E941AD290E008958FEF9FEF0895D8
:1042F000DA01E0910A07F0E0FE2FEE27E60FF71F44
:1043000090E0982F8827A901BD018E0F9F1F0C9464
:10431000838ECF93DF931F92CDB7DEB720910A072C
:1043200030E0322F2227260F371F90E0982F882762
:10433000498341E050E0BE016F5F7F4F820F931FC2
:104340000E94838E0F90DF91CF910895CF93DF93DA
:104350001F92CDB7DEB741E050E0BE016F5F7F4FE7
:104360000E94F88D89810F90DF91CF91089520915F
:104370000A0730E0322F2227620F731F90E0982F38
:104380008827860F971F0C94A62163E070E00C9499
:10439000B7219F92AF92BF92CF92DF92EF92FF929E
:1043A0000F931F93CF93DF93EC017B018091620801
:1043B000811121C01B821A8288EE93E0A0E0B0E058
:1043C0008C839D83AE83BF8389E593E09983888343
:1043D00088E08C8788EE93E09E878D87CE01DF9101
:1043E000CF911F910F91FF90EF90DF90CF90BF90F2
:1043F000AF909F90089534E0932E833311F028E01E
:10440000922E82E5C82E88E0D82E10E098E0B92ED2
:10441000A12CD6012D913D916D01F70184819581EB
:104420002817390791F4812F0E94CC92082F8731E9
:1044300011F08C3139F5812F0E94B891892B59F5F3
:104440000C3119F4812F0E94B0921F5F9112E1CFBD
:10445000A11008C0D701ED91FC910084F185E02DF9
:10446000C70119951B821A8288EE93E0A0E0B0E0A4
:104470008C839D83AE83BF8389E593E09983888392
:10448000BC86A8CF843149F08111DFCFF601329785
:1044900011821082DACFB12ED8CFAA24A394D5CF1F
:1044A0008F929F92AF92BF92CF92DF92EF92FF9244
:1044B0000F931F93CF93DF93CDB7DEB72F970FB630
:1044C000F894DEBF0FBECDBF5C014B017A01809135
:1044D00062088823C9F104E0833309F008E0B501DC
:1044E000CE0101960E94C92182E5C82E88E0D82E0F
:1044F00010E0F601219131916F01F50184819581E0
:104500002817390751F4812F0E94CC92873129F462
:10451000A701B401812F0E942E911F5F0113E9CFE3
:10452000C7012F960FB6F894DEBF0FBECDBFDF9147
:10453000CF911F910F91FF90EF90DF90CF90BF90A0
:10454000AF909F908F900895F12CE12CE9CFDA0184
:10455000E0910A07F0E0FE2FEE27E60FF71F90E04C
:10456000982F8827A901BD018E0F9F1F0C94F88DED
:1045700044E050E0BC018FE090E00C94838E44E076
:1045800050E0BC0185E090E00C94838E44E050E064
:10459000BC0181E090E00C94838E08959F92AF92CD
:1045A000BF92CF92DF92EF92FF920F931F93CF9320
:1045B000DF938C015B01942EE52EFC01C688D78821
:1045C000F08C80E591E00E941EA08F2D0E94D49077
:1045D000C92DDE2D8C179D0708F4EC019E01A50165
:1045E000B6018F2D0E945190F801868997898C0F12
:1045F0009D1F978B868BCE01DF91CF911F910F91DD
:10460000FF90EF90DF90CF90BF90AF909F90089574
:10461000CF93FC01C08D80E591E00E941EA060E276
:1046200070E08C2F0E94E88D62E070E08C2F0E9479
:10463000B72184FD16C062E070E08C2F0E94B72184
:1046400083FF0AC048E162E070E08C2F0E9489215C
:1046500080E090E0CF91089580E591E00E941EA057
:10466000E3CF40E162E070E08C2F0E94892181E07D
:10467000F0CFFF920F931F93CF93DF93EB01FC01D9
:10468000178A168A2A81211109C02B81211106C09F
:104690002C81211103C02D81222301F141155105E7
:1046A000E9F08A01FC01F08C80E591E00E941EA0F7
:1046B000AE014E5F5F4F24E030E06CE070E08F2D84
:1046C0000E947821B8018F2D0E94DB9281E090E05A
:1046D000DF91CF911F910F91FF90089580E0F7CF68
:1046E0000F931F93CF938C01FC016481758181E24C
:1046F0000E940793C82F8830F8F480E591E00E946B
:104700001EA08C2F0E94C521833131F08C2FCF91B8
:104710001F910F910C94B09262E070E08C2F0E9478
:10472000E88DF80184819581EC2FF0E0EE0FFF1FFA
:10473000EE5AF74F91838083CF911F910F91089587
:104740000F931F93CF93DF931F921F92CDB7DEB7C6
:10475000FC0124852830E0F48C0180E591E00E9482
:104760001EA022E030E0AE014F5F5F4F60E170E0DD
:10477000F80184850E94A72289819A819827892738
:1047800098270F900F90DF91CF911F910F9108956F
:1047900090E080E0F6CF0F931F93CF93DF931F92AB
:1047A0001F92CDB7DEB7FC0124852830E0F48C01E0
:1047B00080E591E00E941EA022E030E0AE014F5F54
:1047C0005F4F64E070E0F80184850E94A722898130
:1047D0009A819827892798270F900F90DF91CF9182
:1047E0001F910F91089590E080E0F6CFCF93DF9373
:1047F000EC018BED93E0998388831A821B821C82E3
:104800001D8280E591E00E941EA0BE016E5F7F4F79
:1048100044E050E08FE090E00E94F88DCE01DF91FF
:10482000CF9108950E94448F882331F080916208CF
:10483000843329F0873381F090E080E0089580E5AB
:1048400091E00E941EA085E390E00E94A62185FDD4
:104850000DC082E090E0089580E591E00E941EA0E6
:104860008EE290E00E94A62180FFF3CF81E090E0ED
:1048700008951092A00881E080939F0810927A0812
:1048800061E084E10E941AA361E085E10E941AA31D
:10489000E9EBF0E080818E7F808380818D7F808353
:1048A00088E48093B80085E48093BC000895CF939A
:1048B000DF9391E09093A606882361F0C091B80041
:1048C000D091BA000E9465190E943924D093BA0091
:1048D000C093B800DF91CF910895CF92DF92EF920D
:1048E000FF920F931F93CF93FC01C1810E94A1A35C
:1048F0006B017C018091A008811164C081E08093EC
:10490000A00880939F089FEF90939E0810929D08A7
:1049100010929C0880937B0880917B08CC0FC82B59
:10492000C0937B0880917A08813009F081C0109291
:104930007A080E94A1A36B017C0180917B0880937F
:10494000BB008091A2089091A308A091A408B09107
:10495000A508892B8A2B8B2BA1F00E94A1A3009183
:10496000A2081091A3082091A4083091A5086C1901
:104970007D098E099F09061717072807390708F4CC
:1049800042C08091BC0083FDD8CF85EC8093BC00F1
:104990000E94A1A36B017C018091A008813009F4E1
:1049A00049C080919D08811167C080919D08ECE706
:1049B000F8E0AAEEB6E090E0981751F121912D931E
:1049C0009F5FFACF8091A2089091A308A091A408BC
:1049D000B091A508892B8A2B8B2B09F48BCF0E94D1
:1049E000A1A30091A2081091A3082091A4083091DE
:1049F000A5086C197D098E099F0906171707280756
:104A0000390708F077CF8091A1080E94572480E0F1
:104A1000109279088093780887EF98E00E947612C8
:104A2000CF911F910F91FF90EF90DF90CF9008955D
:104A300085EEACCF8091A2089091A308A091A40824
:104A4000B091A508892B8A2B8B2B09F4A5CF0E9446
:104A5000A1A30091A2081091A3082091A40830916D
:104A6000A5086C197D098E099F09061717072807E5
:104A7000390708F091CFC7CF81E099CFAF92BF92AD
:104A8000CF92DF92EF92FF921F93CF93DF93EC01CF
:104A90000E94ECA46B017C0128EEC20E23E0D21E22
:104AA000E11CF11C10E08BE4A82EB12C0E94ECA4B8
:104AB0006C157D058E059F0598F4ED85FE85309774
:104AC00009F0199560EFCE010E944A19CE010E94AB
:104AD0006D24182F80FF06C0C5010197F1F7E6CFBE
:104AE00081E08A83812FDF91CF911F91FF90EF901A
:104AF000DF90CF90BF90AF9008951F93CF93DF9337
:104B0000EC01162F0E943E25CE010E94321262ED6A
:104B100087EF98E00E94BD12612F70E0609570955C
:104B200084E0660F771F8A95E1F7612B87EF98E0A5
:104B30000E94BD120E94B6A4CE010E946D2481176E
:104B400011F084E08A83DF91CF911F910895CF9374
:104B5000DF93EC0163EC0E944A19CE01DF91CF9103
:104B60000C946D240F931F93CF93DF93EC01162FBA
:104B7000042F0E943E25002341F0CE010E94A7256C
:104B8000682F6460CE010E947D25CE010E94321202
:104B900065EA87EF98E00E94BD12612F87EF98E0E9
:104BA0000E94BD12DF91CF911F910F910C94B6A47A
:104BB000EF92FF920F931F93CF93DF938C017B01B2
:104BC00040E065E50E94B225E70188E0E80EF11CAF
:104BD000699140E0C8010E94B225CE15DF05C1F7FA
:104BE000DF91CF911F910F91FF90EF900895CF9398
:104BF000DF93EC010E94321240E060EFCE010E9490
:104C0000B225DF91CF910C94B6A40F931F93CF934D
:104C1000DF93EC010E943E2580FD36C0CE010E944C
:104C2000A72560E0CE010E947D25CE010E943E2591
:104C3000CE010E94321264EB87EF98E00E94BD1211
:104C40000E94B6A4CE010E943E25082F10E082FFEC
:104C500016C082E08A838881882341F0CE010E94B9
:104C6000A725682F6160CE010E947D2515950795C7
:104C7000802F8170DF91CF911F910F9108958A81CC
:104C8000823049F71A82E7CF80E0F4CFCF92DF92EB
:104C9000EF92FF920F931F93CF93DF938C01EB0161
:104CA0007A01FC01858196810E9405268823C1F145
:104CB000BE01F801858196810E94D82540E06EEB07
:104CC000F801858196810E94B225E7016701F9E02C
:104CD000CF0ED11CF801E580F680C7010E943E2569
:104CE000C7010E94321266E987EF98E00E94BD1268
:104CF0000E94B6A4C7010E943E2561EEC7010E9432
:104D00004A19C7010E946D248993CC16DD0611F75C
:104D1000F801858196810E94052691E0813009F095
:104D200090E0892FDF91CF911F910F91FF90EF902D
:104D3000DF90CF900895CF93DF93EA010E9446263B
:104D4000882381F0DE0189E090E0815039F0ED9117
:104D5000E927F0E0E352F74E9491F7CF81E0288500
:104D6000291380E0DF91CF910895CF93DF9300D096
:104D700000D000D0CDB7DEB7AE014F5F5F4F0E94CD
:104D80009B26882331F08D818F33A9F020F48F3159
:104D9000A1F080E007C08F3521F08F37D1F78CE08C
:104DA00001C08BE029960FB6F894DEBF0FBECDBFD1
:104DB000DF91CF9108958AE0F5CF89E0F3CF6F922C
:104DC0007F928F929F92AF92BF92CF92DF92EF929B
:104DD000FF920F931F93CF93DF93FC012485211142
:104DE0008CC0872E762EEC010E940526882309F4BC
:104DF00086C0CE010E943E2540E060EFCE010E94B9
:104E0000B22510E000E066246A94AA24A394B12C91
:104E1000E02EE694E694E694F12C802F87706501ED
:104E200001C0CC0C8A95EAF78B85082E000C990BF3
:104E30000817190734F5FE01EE0DFF1D93809C2025
:104E4000CE010E943E25CE010E94321268E787EF14
:104E500098E00E94BD12992011F080E8982E692DEB
:104E600087EF98E00E94BD120E94B6A4CE010E9476
:104E70003E25982F907485FF0BC0992369F08EEF23
:104E80002AC09924939408171907D1F2912CD8CFEE
:104E9000911102C087FF602EFE01EE0DFF1D938170
:104EA00087FF28C0C92AC3820F5F1F4F0034110536
:104EB00009F0AECF6B86FFEF6F1202C081E08C87E6
:104EC0002396E72DF82DCF01089629912193E81715
:104ED000F907D9F781E0DF91CF911F910F91FF90F2
:104EE000EF90DF90CF90BF90AF909F908F907F908A
:104EF0006F900895C094C922D6CF80E0ECCF8FEF99
:104F0000EACFCF92DF92EF92FF920F931F93CF934E
:104F1000DF93CDB7DEB769970FB6F894DEBF0FBE4B
:104F2000CDBFE091A406F091A506309709F483C0A7
:104F30008091190790911A07892B09F47CC08FEF93
:104F40008387148613821482158216821782108634
:104F50001186128666EB70E186E899E00E94C985A9
:104F600086E899E00E94DA838E010F5E1F4FBE0132
:104F70006E5E7F4F8091A4069091A5060E94DF2669
:104F800018160CF058C0A895DE0111969E012E5EF1
:104F90003F4F7D01F90141919F01842F90E054E042
:104FA000959587955A95E1F78A589D4FFC01808128
:104FB0008C93E42FEF70F0E0EA58FD4F808111965A
:104FC0008C9311971296A017B10721F7198AB70190
:104FD0008091190790911A070E942A976C0161EB42
:104FE00070E186E899E00E94C985B70186E899E0FA
:104FF0000E946385C114D104B9F0C6010E948913CF
:105000007C01892B09F4B3CF6CEA70E186E899E062
:105010000E94C985B70186E899E00E94638586E809
:1050200099E00E94DA83A3CF67EA70E186E899E00D
:105030000E94C985F4CF88EC90E069960FB6F89489
:10504000DEBF0FBECDBFDF91CF911F910F91FF90BB
:10505000EF90DF90CF9008950F931F93CF93DF933E
:105060006DED73E087E39AE00E94DE8381E00E94A9
:10507000C6A30E94651961E085E10E9448A360E033
:1050800084E10E9448A3C4E1D0E010E001E0612F78
:1050900085E10E941AA310276AE070E080E090E0AA
:1050A0000E94B9A4219799F70E94E99FC091A40694
:1050B000D091A5062097D1F0CE010E945B198823DC
:1050C000A9F0CE010E94F7258091A4069091A50633
:1050D000FC0100830E94052661ED78E1811102C088
:1050E0006DEB78E187E39AE00E94ED8581E0DF9146
:1050F000CF911F910F91089585ED8093BC00809111
:10510000A2089091A308A091A408B091A5080796C1
:10511000A11DB11D23E0B695A795979587952A9572
:10512000D1F72091BC0024FD03C01092A00808957F
:105130004091A2085091A3086091A4087091A5081D
:10514000452B462B472B69F30097A105B10541F08C
:1051500025E32A95F1F700000197A109B109E1CFF4
:105160008091A1080C9457241F920F920FB60F92B2
:1051700011240BB60F922F933F934F935F936F932E
:105180007F938F939F93AF93BF93EF93FF93809100
:10519000B900887F803609F44DC008F040C08832DD
:1051A00009F4A9C028F5803109F49DC0C8F488230A
:1051B00009F4FBC0883009F496C0FF91EF91BF91CC
:1051C000AF919F918F917F916F915F914F913F919F
:1051D0002F910F900BBE0F900FBE0F901F90189540
:1051E000883109F488C0803241F780939E0814C04A
:1051F000803409F49DC040F48033B9F38833E9F674
:1052000080939E0885ECB0C0803509F485C0883550
:1052100009F496C0883489F60E947C28CECF88395C
:1052200009F48CC038F5883729F050F4883611F02D
:10523000803719F683E08093A0081092E90657C0E2
:10524000883809F47BC0803919F0803809F0B5CF6F
:105250008091E906803208F071C0E091E90681E0B2
:105260008E0F8093E9068091BB00F0E0E753F94F81
:1052700080833DC0803B39F0E0F4803A09F479C086
:10528000883A09F09ACF84E08093A0081092C8066B
:105290001092C706E0917608F091770819958091F1
:1052A000C70681110FC081E08093C7061092A70640
:1052B00009C0803C09F4A6CF883C09F4A3CF883B01
:1052C00009F07BCFE091C80681E08E0F8093C8067D
:1052D000F0E0E955F94F80818093BB009091C806BA
:1052E0008091C70629C080917B088093BB0085EC24
:1052F0008093BC0062CF90919D0880919C08981784
:1053000058F5E0919D0881E08E0F80939D08F0E0B4
:10531000E458F74F8081E9CFE0919D0881E08E0F3E
:1053200080939D088091BB00F0E0E458F74F8083A4
:1053300090919D0880919C089817C8F285E8D8CF75
:10534000E0919D0881E08E0F80939D088091BB00C5
:10535000F0E0E458F74F808380919F0881115CCF83
:1053600081E080937A0884EA8093BC001092A008C0
:1053700024CF85EC8093BC001092A0088091E906B0
:10538000803230F4E091E906F0E0E753F94F108203
:105390006091E90670E0E0917408F091750889EC7D
:1053A00096E019951092E90608CF10929E0834CF26
:1053B0004F925F926F927F92AF92BF92CF92DF92A5
:1053C000EF92FF920F931F93CF93DF9300D01F9222
:1053D000CDB7DEB72B013C0129833A834B835C8335
:1053E000A6019501C801B701640D751D861D971DA5
:1053F000211531054105510511F00E9440D2298146
:105400003A814B815C816217730784079507D0F45A
:10541000241535054605570530F521E0822F0F90FC
:105420000F900F900F90DF91CF911F910F91FF90F0
:10543000EF90DF90CF90BF90AF907F906F905F9094
:105440004F900895461657066806790650F421E0F5
:1054500089819A81AB81BC8184159505A605B70524
:10546000E8F220E0DBCF21E0461657066806790611
:10547000A8F2F7CF8F929F92AF92BF92CF92DF9216
:10548000EF92FF920F931F93CF93DF937C014A011A
:105490005901C091A206D091A306062F660F110BE9
:1054A000209709F45CC088858F70863009F055C05C
:1054B00067EE73E0CE010E942A976C0182E08816A5
:1054C000910449F06CEE73E0E3E08E16910429F04C
:1054D000D0E0C0E006C060EF73E0CE010E942A97E2
:1054E000EC01C114D104D9F1F60180858F708430AC
:1054F000B1F561857285A801C7010E945AD7A8013C
:1055000065EF73E0C7010E943CD7209779F1888549
:105510008F70843059F569857A85A801C7010E948A
:105520003CD7A80165EF73E0C7010E943CD7A114E6
:10553000B10429F0A801B501C7010E943CD7C701F9
:10554000DF91CF911F910F91FF90EF90DF90CF905F
:10555000BF90AF909F908F900895D0E0C0E0A801D9
:1055600066E778E1C7010E9438CBC9CFF2E08F1619
:10557000910481F083E08816910429F060910B0773
:1055800070910C07CACFA80160E778E1C7010E94BB
:105590001ACBC7CFA8016DE678E1F8CFCF92DF92A2
:1055A000EF92FF920F931F93CF93DF93CDB7DEB7A8
:1055B000C154D1090FB6F894DEBF0FBECDBF6C0148
:1055C000AB0130E020E060E4CE0101967C010E9456
:1055D0003A2AF70101900020E9F731978F010E195F
:1055E0001F09A801B701C6010E944CD7892B11F0F1
:1055F00010E000E0C801CF5BDF4F0FB6F894DEBFCC
:105600000FBECDBFDF91CF911F910F91FF90EF9013
:10561000DF90CF900895CF92DF92EF92FF920F9399
:105620001F93CF93DF93CDB7DEB7C054D1090FB628
:10563000F894DEBF0FBECDBF80911507909116077D
:10564000059709F449C06115710509F445C0690160
:105650007A018B0140E450E0CE0101960E945AD7B6
:105660006FE270E0CE0101960E9421D7892B41F4B0
:10567000980143E050E060E4CE0101960E943A2A8E
:105680004FE350E0B601CE0101960E943CD70E9444
:105690004897882309F1809115079091160706977E
:1056A000D9F48091CA08811117C0B701CE010196C3
:1056B0000E94BAA581E090E0C05CDF4F0FB6F8947D
:1056C000DEBF0FBECDBFDF91CF911F910F91FF9035
:1056D000EF90DF90CF90089590E080E0EDCFEF92D3
:1056E000FF920F931F93CF937C018C01C0E0C330D6
:1056F000E1F0F801428150E070E060E02AE030E043
:1057000086E899E00E94DD846BE678E186E899E01E
:105710000E94C985CF5F0F5F1F4FC43041F7CF9103
:105720001F910F91FF90EF900895F701458150E090
:1057300070E060E02AE030E086E899E00E94DD84D5
:1057400069E678E1E3CFCF93DF931F921F92CDB745
:10575000DEB780913F0B9091400B009711F48BE4E2
:105760009BE0BE016F5F7F4F681B790B072E000C1B
:10577000880B990B0F900F90DF91CF9108954F9266
:105780005F926F927F928F929F92AF92BF92DF92C1
:10579000EF92FF920F931F93CF93DF93CDB7DEB7B6
:1057A00060970FB6F894DEBF0FBECDBFFC0119861F
:1057B0001A861B861C869A859F7090669A87A081A0
:1057C000B181109709F4F7C08C91882309F4F3C0D4
:1057D00000811181D8019C91992309F443C09D3225
:1057E00009F4EDC090539A3028F00F5F1F4F1183DA
:1057F0000083EECFC801D12CDC017D01E81AF90A43
:105800002D91022E000C330B205331092A30310523
:10581000A0F35F016EE270E0C8010E9421D7FC0195
:10582000009709F448C0DC014D018E1A9F0A1196B9
:105830008C911197082E000C990BC09711960A971E
:1058400098F38181282F082E000C330B2053310947
:105850002A30310518F480330CF06EC020E030E0BF
:10586000A90108C0D12CF12CE12CD3CF29E030E0E4
:1058700040E050E0AAE0B0E00E9481D22B013C0160
:105880002281822F022E000C990BC0978A3091053D
:1058900070F420330CF458C02A330CF059C0092E90
:1058A000000CAA0BBB0B480E591E6A1E7B1E8114EE
:1058B000910409F052C0C8010E94B3CA2A852F7012
:1058C000206A2A872B013C016CE270E0D5018D91A2
:1058D0009C910E9421D7009709F068C0F5011182C0
:1058E00010824D865E866F86788A88E0FE01399642
:1058F000DE01119601900D928A95E1F729813A8196
:105900004B815C816D817E818F81988560960FB619
:10591000F894DEBF0FBECDBFDF91CF911F910F91E5
:10592000FF90EF90DF90BF90AF909F908F907F900F
:105930006F905F904F9008958A330CF097CF032EAD
:10594000000C440B550B96CF80E090E0DC01ABCF10
:1059500089E090E0A0E0B0E0A6CFC801B3E08B16EC
:105960009104DCF4E8E0EE16F104BCF40E94B3CA42
:105970009B01AC01A4E6B0E00E9481D2DD2041F0A1
:105980007094609450944094411C511C611C711C93
:10599000460E571E681E791E97CF0E9491CA2B0192
:1059A0003C018A858F7080678A878ECF0196D501EA
:1059B0008D939C9396CF412C512C320192CFC801EC
:1059C0000196DD24D39418CFCF92DF92EF92FF920D
:1059D0000F931F93CF93DF93EC01A881B9811097A8
:1059E00081F18C91882369F108811981F8019081F6
:1059F000992351F09D3241F090539A3028F00F5F77
:105A00001F4F19830883F0CFC8010E94B3CA6B01EE
:105A10007C016CE270E0C8010E9421D7009769F414
:105A200019821882C701B601DF91CF911F910F91A2
:105A3000FF90EF90DF90CF9008950196998388832F
:105A4000F1CFC12CD12C7601EDCF6EED75E186E85A
:105A500099E00E94C9856BEC75E186E899E00E94A7
:105A6000C9856DEB75E186E899E00E94C98565EB13
:105A700075E186E899E00E94C98586E899E00E9470
:105A8000DA8365EA75E186E899E00E94C98569E9EB
:105A900075E186E899E00E94C9856CE875E186E8C1
:105AA00099E00E94C98567E775E186E899E00E9460
:105AB000C98568E675E186E899E00E94C98560E6D7
:105AC00075E186E899E00E94C98565E575E186E89B
:105AD00099E00E94C98568E475E186E899E00E9432
:105AE000C9856EE375E186E899E00E94C9856FE299
:105AF00075E186E899E00E94C98567E275E186E86C
:105B000099E00E94C9856BE175E186E899E00E9401
:105B1000C98561E075E186E899E00E94C98562EE79
:105B200074E186E899E00E94C9856DEC74E186E82D
:105B300099E00E94C98560EC74E186E899E00E94D2
:105B4000C98562EB74E186E899E00E94C98566EA3E
:105B500074E186E899E00E94C9856EE974E186E8FF
:105B600099E00E94C98563E974E186E899E00E94A2
:105B7000C98566E874E186E899E00E94C9856EE708
:105B800074E186E899E00E94C98563E774E186E8DC
:105B900099E00E94C98564E674E186E899E00E9474
:105BA000C9856BE574E186E899E00E94C9856DE4DA
:105BB00074E186E899E00E94C9856FE374E186E8A4
:105BC00099E00E94C98586E899E00C94DA830F93E6
:105BD0001F93CF93DF9300D000D0CDB7DEB70E94E4
:105BE000252D61E07EE086E899E00E94C985CE011E
:105BF00001960E94F623CE0101960E946F2B0BEDB9
:105C000013E01A8309838091F3089091F408A0911E
:105C1000F508B091F6088B839C83AD83BE83CE01DB
:105C200001960E946F2B1A8309831B821C821D829E
:105C30001E8280E591E00E941EA044E050E0BE017B
:105C40006D5F7F4F81E090E00E94F88DCE0101965C
:105C50000E946F2B1A8309831B821C821D821E8265
:105C600080E591E00E941EA044E050E0BE016D5F1F
:105C70007F4F85E090E00E94F88DCE0101960E9452
:105C80006F2B67E27EE086E899E00E94C98588EC88
:105C900090E026960FB6F894DEBF0FBECDBFDF9121
:105CA000CF911F910F910895009789F0FC012085F5
:105CB0002F70253061F40E94A297009741F0FC01FB
:105CC00020852F70243019F481859285089590E005
:105CD00080E00895CF92DF92EF92FF920F931F938F
:105CE000CF93DF9300D000D0CDB7DEB78091A1066F
:105CF00081119AC0809115079091160702970CF4B4
:105D000093C08091450690914606009709F48CC097
:105D100069EF73E00E942A978C01009709F484C010
:105D20000E942E9CE82EF12CE114F10409F47CC0B1
:105D300070E060E0C8010E94542E6C01EA94EF28E4
:105D400009F481C061E0C8010E94A297FC010185AD
:105D50001285CE0101960E94F623CE0101960E9483
:105D600021A062EF7DE086E899E00E94C985B60136
:105D700086E899E00E94638566E674E086E899E02B
:105D80000E946385B80186E899E00E94D19B66E68F
:105D900074E086E899E00E94638563E678E086E82F
:105DA00099E00E94638586E899E00E94DA8362E0C8
:105DB00072E085E59AE00E94FC17D0924B0AC092EF
:105DC0004A0A10934D0A00934C0A83E698E0892B07
:105DD000E9F587EF93E090934F0A80934E0A809104
:105DE0000D0790910E07009741F070E060E00E946F
:105DF000542E90930C0780930B0780910B07909182
:105E00000C07009731F19093510A8093500A109239
:105E1000530A1092520A81E08093A10669ED7DE059
:105E200086E899E00E94C98526960FB6F894DEBFF1
:105E30000FBECDBFDF91CF911F910F91FF90EF90DB
:105E4000DF90CF90089502E012E083CF83E698E0E0
:105E5000C2CF86EC92E0892B19F487EF93E0D3CF81
:105E600086EC92E0D0CF0F931F93CF9364ED7DE04B
:105E700086E899E00E94C9850AE619E0C0E0F801C9
:105E800081918F01803130F460E074E086E899E020
:105E90000E946385C530C9F0F8013197408150E018
:105EA00070E060E020E130E086E899E00E94DD8467
:105EB00062ED7DE086E899E00E94C985CF5FC6303B
:105EC000F1F6CF911F910F91089540916F0950E025
:105ED00070E060E020E130E086E899E00E94DD8437
:105EE00086E899E00E94DA83E9CFEF92FF920F9360
:105EF0001F93CF93DF9300D000D01F92CDB7DEB7B2
:105F00007B01CE0107969F938F9301979F938F9369
:105F100001979F938F9301979F938F9301979F93DF
:105F20008F9301979F938F938E010F5F1F4F1F9346
:105F30000F9382E094E09F938F93DB0113968C91F3
:105F400013978F9312968C918F930E94E1D70FB67F
:105F5000F894DEBF0FBECDBF0697ECF469EA72E19C
:105F600080E999E00E94C985D70112966D917C91D4
:105F700080E999E00E94638580E991E027960FB659
:105F8000F894DEBF0FBECDBFDF91CF911F910F916F
:105F9000FF90EF9008958091620990916309892B99
:105FA000A9F10E948C98882389F182E70E94779852
:105FB0008091620990916309DC01ED91FC91008868
:105FC000F189E02D64E070E019958091620990916B
:105FD0006309DC01ED91FC910280F381E02D46E044
:105FE00050E0B801199586E0F801AAE6B9E0019001
:105FF0000D928A95E1F78091620990916309DC0125
:10600000ED91FC910488F589E02D19950E94332FBC
:106010006BEB72E186E899E00E94C98588EC90E01C
:10602000ADCF2F923F924F925F926F927F928F925D
:106030009F92AF92BF92CF92DF92EF92FF920F9317
:10604000CF93DF9300D01F92CDB7DEB77C017A8368
:1060500069835C834B83DB011C92FC0160816623B6
:1060600009F44EC030FF4CC0F9E06F9FB00111241D
:106070006B577E4DCD010E9438CBD70111968C9184
:10608000807F41F04B815C8161E574E089819A8178
:106090000E943CD7E981FA8101900020E9F731970D
:1060A00029813A81E21BF30B19012E0E3F1E4B8111
:1060B0005C814E1B5F0B415051095C834B83D701C0
:1060C0001196EC9111978E2F807F09F4F7C0E2951D
:1060D000EF70E150EC3008F0F1C0F0E08827EC58A8
:1060E000FF4C8F4F0C94CBD2833026319331F23159
:1060F0000D32D130A331A331A331BF30A7302932C3
:1061000029803A80DCCFF7018481282F30E050E0ED
:1061100040E0002359F030E0A4E6B0E00E9494D2C1
:106120002FEF30E040E050E00E9462D25F934F9347
:106130003F932F9386E194E09F938F93FC81FF938D
:106140002B812F933F922F920E9474D7B2C0179643
:106150008C9117978F9316968C9116978F9315960F
:106160008C9115978F9314968C918F9389E194E07D
:106170009F938F93BC81BF93EB81EF93E3CF1796EF
:106180008C9117978F9316968C9116978F931596DF
:106190008C9115978F9314968C918F938DE194E049
:1061A000E7CF1496CD90DD90ED90FC901797F7FE19
:1061B00034C084E6882E912CA12CB12CC701B601E5
:1061C000A50194010E9462D29B01AC018827992706
:1061D000DC01821B930BA40BB50BBF93AF939F9372
:1061E0008F9366277727CB016C197D098E099F094C
:1061F000A50194010E9462D25F934F933F932F9326
:1062000081E294E09F938F933C813F934B814F9326
:106210003F922F920E9474D74CC0C701B60124E66A
:1062200030E040E050E00E9462D29F938F937F93D2
:106230006F935F934F933F932F9382E294E09F93EA
:106240008F939C819F93AB81AF93E2CFC7010E9454
:106250009514BC01D7011696CC9016971796DC9032
:106260001797D0FADD24D0F814969C9114971596C0
:10627000FC90EB80BC80292F30E050E040E077FDBF
:1062800035C0011135C07F936F931F921F921F92EB
:106290009F931F92FF92DF92CF928BE294E09F93A5
:1062A0008F93FC81FF932B812F933F922F920E941B
:1062B00074D70FB6F894DEBF0FBECDBF89819A8127
:1062C0000F900F900F900F90DF91CF910F91FF9053
:1062D000EF90DF90CF90BF90AF909F908F907F9086
:1062E0006F905F904F903F902F900895002361F042
:1062F000292F30E0A4E6B0E00E9494D22FEF30E0E6
:1063000040E050E00E9462D25F934F933F932F93FF
:106310001F92FF92DF92CF928EE294E09F938F9331
:10632000BF92EF9275CF15968C9115971F928F9310
:1063300016969C91169717968C9181708F939F93C8
:1063400081E394E015CF14968D909D90AD90BC9014
:10635000179720E030E0A901C501B4010E94F6D0F2
:106360002401350187FF04C077FA709477F87094A0
:10637000C301B2010E94C8D36B01072E000C880B29
:10638000990B0E94FDD09B01AC01C301B2010E9498
:10639000E9D220E030E04AE754E40E945CD10E9458
:1063A00053D40E94C8D3062F772E20E030E0A901F5
:1063B000C501B4010E94F6D087FF07C07F920F93FA
:1063C000DF92CF9287E394E0D3CE7F920F93DF9258
:1063D000CF9288E394E09F938F933C813F934B81CE
:1063E0004F93B0CE14968C9114971F928F9315965D
:1063F0008C9115971F928F9316968C911F928F9365
:106400008EE294E09F938F93BC81BF93EB81EF93D7
:106410003F922F920E9474D74CCF17968C9117976A
:106420001F928F9314968C9114971F928F931596A9
:106430008C9115971F928F9316968C911F928F9324
:106440008BE294E09F938F93BC81BF93EB81EF939A
:10645000DFCE14966D917C914B815C81C1010E94CD
:106460005AD72CCFEF92FF920F93CF93DF93CDB7F4
:10647000DEB7A0970FB6F894DEBF0FBECDBF7C018C
:1064800000E020E033E040E250E0BE016F5F7F4F6C
:106490000E941130BE016F5F7F4F87E39AE00E9438
:1064A000638561E47CE087E39AE00E94C985F70197
:1064B000618162956F7087E39AE00E94CA9B6AE3EC
:1064C0007CE087E39AE00E94C985F70161816F70E3
:1064D00087E39AE00E94CA9B87E39AE00E94DA83EE
:1064E000A0960FB6F894DEBF0FBECDBFDF91CF915F
:1064F0000F91FF90EF900895AF92BF92CF92EF92DD
:10650000FF920F931F93CF93DF9300D000D01F9281
:106510001F92CDB7DEB75C0109831A832B833C83BE
:106520004D835E836F8378876AEB77E187E39AE038
:106530000E94C985CE0101960E943232E114F10415
:1065400039F063EB77E1C7010E9401CB009721F19D
:10655000F5010281138101151105E1F08981811195
:1065600059C08A818F70813009F45CC038F1823063
:1065700019F1082F10E066E977E187E39AE00E94BD
:10658000C985B80187E39AE00E94D19B87E39AE02E
:106590000E94DA8390E080E028960FB6F894DEBF80
:1065A0000FBECDBFDF91CF911F910F91FF90EF9064
:1065B000CF90BF90AF900895CC20B9F0CE01019656
:1065C0000E94B197892B09F444C0C8010E94501C55
:1065D000672B682B692BD9F480E00E940E19AB0160
:1065E000BC01C8010E943D1F12C0C8010E94E11CED
:1065F0008E3019F048F4813051F4CE0101960E949A
:10660000B197892B21F0E1CF83518330B0F381E042
:1066100090E0C2CF8031C0F48E30B8F68130A9F25C
:106620008230B9F066EA77E187E39AE00E94C98593
:10663000698187E39AE00E94CA9B87E39AE00E94FF
:10664000DA8301E010E097CF8351833008F4BDCFA7
:10665000E9CF40E050E0BA01C8010E943D1F60E070
:10666000C5010E94EE1CD3CFCF92EF92FF920F9301
:106670001F93CF93DF9300D000D01F921F92CDB70E
:10668000DEB77C0109831A832B833C834D835E83B1
:106690006F83788769E277E187E39AE00E94C98592
:1066A000CE0101960E9432328981811129C00A816E
:1066B0000F70013069F128F010E00230D1F5CC20E4
:1066C000E1F0CE0101960E94B197F701028113819A
:1066D000892B69F0C8010E94501C672B682B692B1D
:1066E00061F480E00E940E19AB01BC0103C040E0E0
:1066F00050E0BA01C8010E943D1F81E090E02AC02D
:106700008031B0F58E30B8F58130A9F18230B9F121
:106710006CE177E187E39AE00E94C985698187E3AC
:106720009AE00E94CA9B87E39AE00E94DA8301E024
:1067300010E06CE077E187E39AE00E94C985B80138
:1067400087E39AE00E94D19B87E39AE00E94DA8374
:1067500090E080E028960FB6F894DEBF0FBECDBF64
:10676000DF91CF911F910F91FF90EF90CF900895FF
:106770008351833068F6F70102811381ABCF40E08B
:1067800050E0BA01F70182819381B5CFCF92DF92B9
:10679000EF92FF920F931F93CF93DF9361157105D3
:1067A00009F458C06A017B018C01CB010E94B71427
:1067B000D82F882371F1D70114968D919C91009761
:1067C000E9F1FC01C0852C2F2F703EEF320F3230E3
:1067D00010F0211128C0C295CF70D0FE59C0C7015A
:1067E0000E94E11CF8018083CC2351F1C295C07F47
:1067F00081818F70C82BC183D7011496ED91FC91D4
:1068000081859285A385B485F80184839583A683C9
:10681000B7838D2FDF91CF911F910F91FF90EF9054
:10682000DF90CF900895253049F460E00E94A29750
:10683000009721F0DC011896CC91CDCFC0E0CDCFF0
:10684000D7011496ED91FC9180858F70823021F0F4
:10685000833081F0D0E0DDCF41855285638574853A
:10686000F80181818F70806A8183448355836683B8
:106870007783CFCF4185528563857485F801818107
:106880008F70806781834483558366837783C1CF0C
:10689000CC23B1F2C295C07FF801AACF0F931F930A
:1068A000CF93DF9300D000D01F921F92CDB7DEB7F9
:1068B00019821A821B821C821D821E821F821886E8
:1068C0002A812F702A83FC0102811381C8010E9452
:1068D000E11C813041F020F0823011F0853081F4EC
:1068E00090E080E002C081E090E028960FB6F89436
:1068F000DEBF0FBECDBFDF91CF911F910F910895E5
:1069000040E052E0B801CE0101960E94C633CE01AC
:1069100001960E94B197E9CFCF93DF9300D000D0CA
:106920001F921F92CDB7DEB7FC01862F8F70618159
:10693000607F682B618388E0DE01119601900D92E3
:106940008A95E1F729813A814B815C816D817E8155
:106950008F81988528960FB6F894DEBF0FBECDBF05
:10696000DF91CF910895CF93DF9300D000D01F9295
:106970001F92CDB7DEB7FC01608398E0DE0111966F
:1069800001900D929A95E1F729813A814B815C81C2
:106990006D817E818F81988528960FB6F894DEBF31
:1069A0000FBECDBFDF91CF910895DC011196EC9120
:1069B0001197E295EF70E150EB3008F037C0F0E04E
:1069C0008827EA51FB4C8F4F0C94CBD2F834F83423
:1069D0001635F134F1340735FE34FE34FE34F1342B
:1069E000F13414966D917D918D919C911797089536
:1069F00014966C9170E090E080E0089514966D918B
:106A00007D918D919C9117970E94C8D308951496FB
:106A10006D917D918D919C91179724E630E040E037
:106A200050E00E9462D2CA01B901089560E070E0AE
:106A3000CB0108958F929F92AF92BF92CF92DF9237
:106A4000EF920F931F93CF93DF9300D000D01F924C
:106A50001F92CDB7DEB709831A832B833C834D8306
:106A60005E836F837887FC01208131812115310598
:106A7000A1F490E080E028960FB6F894DEBF0FBE38
:106A8000CDBFDF91CF911F910F91EF90DF90CF900D
:106A9000BF90AF909F908F9008958C01C9010E9484
:106AA0002E9CC82ED12CF6E0CF16D104ACF40E9457
:106AB000FF8CFC01892B19F08085807F8087808581
:106AC0008F708087BF01F801808191810E94A99B0E
:106AD000FFEFCF1ADF0AE7CF65E0F80180819181EF
:106AE0000E94A2978C01892B21F28981803108F6BE
:106AF000CE0101960E94D5341616170618061906FF
:106B000044F4F8018085982F9D70A1F08F70873034
:106B100089F0F80180858F70808762EC77E087E3E9
:106B20009AE00E94C98587E39AE00E94DA8381E0B7
:106B300090E0A1CF0E94ECA44B015C01CE01019634
:106B40000E94D534860E971EA81EB91EF8018186B4
:106B50009286A386B48682E0E11087E099819295BF
:106B6000907F892BF801808767EB77E087E39AE0D5
:106B70000E94C985CE0101960E94D534AB01BC01AB
:106B80002AE030E087E39AE00E94DD8461EB77E061
:106B900087E39AE00E94C985F801418552856385A3
:106BA00074852AE030E087E39AE00E94DD84BBCF61
:106BB000CF93DF93EC016115710539F48F818170FA
:106BC0008F8381E0DF91CF9108958981982F9295ED
:106BD0009F7029F180E09430A8F79B01770F440B58
:106BE000550B2959310941095109A4E6B0E00E9429
:106BF00081D22BE531E040E050E00E9462D237FFC5
:106C000002C030E020E02536310514F024E630E003
:106C10002F5F220F8F818170282B2F83D2CF8F700F
:106C200080628983DACF2F923F924F925F926F9268
:106C30007F928F929F92AF92BF92CF92DF92EF920C
:106C4000FF920F931F93CF93DF93CDB7DEB76A9771
:106C50000FB6F894DEBF0FBECDBF1C0109871A879F
:106C60002B873C874D875E876F87788B22E1E21602
:106C7000F10408F035C0F701EA52FD4F30813D8B39
:106C8000CE0109960E94951497FD04C0BC01C10174
:106C90000E94D8359A85892F8F70D1011196EC9179
:106CA0001197E07FE82B1196EC93119789858C93CF
:106CB000E295EF70EC3008F063C0F0E08827EC5903
:106CC000F94C8F4F0C94CBD253388D368D36F2372A
:106CD00072368738BC37FB37FB37FB37BC37BC37DE
:106CE0001D8ACECF10E092959F709D3008F011C4A0
:106CF000E92FF0E08827E058F94C8F4F0C94CBD265
:106D0000C036C038E038C03889388938C038C03813
:106D1000893A893AC038C038963792959F709D302D
:106D200008F014C1E92FF0E08827E656F94C8F4FA0
:106D30000C94CBD2C036743767372A37AA36A736B9
:106D40004B377637A637A6373537353796378889A4
:106D5000F10187838F85D10116968C9316978E85C6
:106D600015968C9315978D8514968C931497929500
:106D7000907F11968C9111978F70982B11969C9300
:106D8000FD89FF2309F463C0D10111968C9182958E
:106D90008F702F2F30E08217130609F458C064E972
:106DA0007BE087E39AE00E94C985F10161816295E9
:106DB0006F7087E39AE00E94CA9B61E97BE087E3FA
:106DC0009AE00E94C9856D8987E39AE00E94CA9B78
:106DD0006FE87BE087E39AE00E94C985D1010C91BE
:106DE00019821A821B821C821D821E821F821886B3
:106DF0008D898295807F9A819F70892B8A830983F0
:106E0000EE24EA94FE2C11961C91119712962C9167
:106E1000129713963C91139714964C9114971596CC
:106E20005C91159716966C91169717967C91CE01EA
:106E300001960E941336F1012083318342835383EC
:106E40006483758386839783C1010E94323288E010
:106E5000F1016FC18F859889F1018683878190FB4D
:106E600080F987838E8585838BCF8D859E85AF85C1
:106E7000B889B7FD0EC08F3F9105A105B10529F076
:106E800024F08FEF90E0A0E0B0E0D10114968C9355
:106E900077CF80E0FACF6D857E858F85988920E059
:106EA0006D39BFEF7B078B079B076CF02FEF6115E8
:106EB000E4E67E078105910534F424E630E040E005
:106EC00050E00E9462D2D10114962C9359CF8F8545
:106ED0009889F1018683878190FB80F987838E856D
:106EE00085838D8584834CCF8D85CFCFCD84DE8403
:106EF000EF84F88820E030E0A901C701B6010E94C4
:106F0000F6D060E087FD0FC020E030E04FE753E4AB
:106F1000C701B6010E94FED36FEF181624F0C70117
:106F2000B6010E94CFD3F10164832ACFD10111961B
:106F30008C9111978F70806C11968C9311978D8521
:106F40009E8515969C938E9314971ACF61E27CE0F0
:106F500087E39AE00E94C9856A8562956F7087E32E
:106F60009AE00E94CA9B6EE17CE087E39AE00E946F
:106F7000C985F1016181C0C092959F70933091F0F5
:106F80009C30A1F24D855E856F857889F10144833F
:106F90005583668377839295907F81818F70982B3C
:106FA0009183EECEC1010E94B197D10114968C93CA
:106FB00014978F85988916968C93169717968C91AF
:106FC000179790FB80F917968C9317978E851596D7
:106FD0008C93159711968C9111978F7080621196F2
:106FE0008C93CECECE0109960E94B197D101149612
:106FF0008C931497EFCF92959F709D3008F066C0E8
:10700000E92FF0E08827E85FF74C8F4F0C94CBD244
:10701000C03623385238D2375238523815384238B1
:107020004238423831383D3896378D859E85AF8558
:10703000B889F10184839583A683B78381818F709A
:10704000806681839DCE6D8570E090E080E00E9437
:10705000FBD0D10114966D937D938D939C931797DC
:107060008FCE6D857E858F8598890E94FDD0F10138
:10707000648375838683978383CE6D857E858F85B4
:107080009889E5CF9295907FF10181818F70982B3F
:1070900091838D859E85AF85B88984839583A683EA
:1070A000B7836ECE9295907FD10111968C911197F6
:1070B0008F70982B11969C938D859E85AF85B8898E
:1070C000F10184839583A683B7835ACE6CE07CE07C
:1070D00087E39AE00E94C9856A8562956F7087E3AD
:1070E0009AE00E94CA9B69E07CE087E39AE00E94F4
:1070F000C985D10111966C9162956F7087E39AE012
:107100000E94CA9B87E39AE00E94DA8339CE11E09D
:10711000EACD4D855E856F857889F101448355837D
:10712000668377839295907F81818F70982B91836E
:1071300088E0DE01119601900D928A95E1F7298190
:107140003A814B815C816D817E818F8198856A96C1
:107150000FB6F894DEBF0FBECDBFDF91CF911F9168
:107160000F91FF90EF90DF90CF90BF90AF909F90E6
:107170008F907F906F905F904F903F902F900895E9
:10718000963009F4C1C048F46D85913071F06FEF0D
:1071900070E0933051F060E008C0973009F4C0C04F
:1071A0009A506D857E859230B0F784E68F87888906
:1071B0008E7F888B1E868A858F7080628A876D8716
:1071C0002E8530E0AFEFB0E00E9494D2C12CD12CDC
:1071D0007601CA946115F4E67F078105910544F4B0
:1071E00024E630E040E050E00E9462D269017A017A
:1071F000112309F475C0DA8AC98A2D852E8B022FD6
:1072000010E088898695A82FA150BB0BB88FAF8B53
:10721000119609F0A4C09601203831050CF087C002
:107220008FE790E08C199D09809FD001819FB00D60
:10723000909FB00D11242FEF30E00E94E2D221E8A0
:107240003EE740E050E00E9462D2D10117962C93B5
:10725000ABE9B0E0A70196010E9481D23FE7432E3F
:10726000512C612C712CA30192010E9462D22C59E5
:107270003F4F4F4F5F4F5901AEEFB1E0A70196016D
:107280000E9481D2A30192010E9462D2D8010E9481
:1072900081D22FEF30E040E050E00E9462D28901BD
:1072A0002F3F310519F014F00FEF10E06CEF7BE089
:1072B00087E39AE00E94C985B50187E39AE00E94BE
:1072C000D19B6EEE7BE087E39AE00E94C985B8010E
:1072D00087E39AE00E94D19B87E39AE00E94DA83D9
:1072E0006CEB7BE087E39AE00E94C98587E39AE034
:1072F0000E94DA8365EB7BE087E39AE00E94C98510
:10730000C1010E9432323CCD6D857E858F85988982
:1073100024E630E040E050E00E9462D2B90145CF5F
:107320006D857E858F8598890E94C8D33ECFA70141
:107330002058310941095109ABE9B0E00E9481D2DE
:107340002FE730E040E050E00E9462D22C593F4FDE
:107350004F4F5F4F5901D10117961C92A7CF2F892C
:10736000388DAAEBBFEF0E94DAD224E6822E912C50
:10737000A12CB12CA50194010E9462D229013A01ED
:10738000B4E64B0E511C611C711C26E430E0AF8941
:10739000B88D0E94E2D2A50194010E9462D24901F7
:1073A0005A01EEE18E0E911CA11CB11C29893A896B
:1073B000203831050CF094C08FE790E0821B930BCE
:1073C000809FD001819FB00D909FB00D1124A50129
:1073D00094010E948CD29B01AC01AFEFB0E00E94FF
:1073E00081D224E63AE640E050E00E9462D2D10128
:1073F00017962C93A7019601240D351D461D571D88
:10740000AEEFB1E00E9481D223EE30E040E050E0E8
:107410000E9462D2298B3A8B4B8B5C8BE989FA896B
:10742000FA8FE98FAFEFB0E0A70196010E9481D2F9
:107430002FE730E040E050E00E9462D27901FE89FF
:10744000AF2FB0E029893A894B895C890E9481D2AB
:107450002FEF30E040E050E00E9462D289012F3FE0
:10746000310519F014F00FEF10E068EE7BE087E3D0
:107470009AE00E94C9852AE030E0B301A20187E3C7
:107480009AE00E94DD8462EE7BE087E39AE00E944E
:10749000C9852AE030E0B501A40187E39AE00E94A3
:1074A000DD846AED7BE087E39AE00E94C985B7013D
:1074B00087E39AE00E94D19B62ED7BE087E39AE04C
:1074C0000E94C985B80187E39AE00E94D19B69ECCC
:1074D0007BE087E39AE00E94C985698D7A8DF8CEBA
:1074E000A70196012058310941095109ABE9B0E0E3
:1074F0000E9481D22FE730E040E050E00E9462D24B
:107500002C593F4F4F4F5F4F7901D10117961C9275
:10751000ACCF63EA7BE087E39AE00E94C9856A8585
:1075200062956F7087E39AE00E94CA9B60EA7BE0F5
:107530001CCDFC019181892F82958F7021F08230C2
:1075400029F080E008959F70906291839B0177FFFE
:1075500002C030E020E02E3681E0380714F02DE63E
:1075600031E02683878130FB80F9878381E00895AD
:107570000F931F93CF93DF938C01FC01C081D181C6
:107580006FE270E0CE010E9469D70097D9F0FC014C
:107590001192CF010E94551BEC0166E877E087E36A
:1075A0009AE00E94C985BE0187E39AE00E94D19BC0
:1075B00087E39AE00E94DA83CE01DF91CF911F9199
:1075C0000F910895CE010E94551BEC01892BA1F368
:1075D000F80111821082F0CF8F929F92AF92BF92EA
:1075E000CF92DF92EF92FF920F931F93CF93DF938F
:1075F000CDB7DEB767970FB6F894DEBF0FBECDBF2D
:107600008C017B014C018BE0880E911C9F8A8E8A35
:10761000F801128611861386148E138E672B09F4D7
:1076200063C0A0901707B0901807A114B10409F423
:107630005BC06FE270E0C7010E9421D76C01892B0B
:1076400009F44AC0F701DE01119690E080E0BD0127
:107650002191222341F02F3231F08431910519F02C
:107660002D930196F5CF860F971FFC011082C5015F
:107670000E942A97F80191838083B6016F5F7F4F44
:107680004FE050E0C4010E945AD7CE0146960E94B6
:10769000B83AF801948F838F8E899F89892B09F4DA
:1076A0001386C8010E94B714882319F0C8010E94EC
:1076B000A01F67960FB6F894DEBF0FBECDBFDF9157
:1076C000CF911F910F91FF90EF90DF90CF90BF90DF
:1076D000AF909F908F900895B701C5010E942A979F
:1076E000F80191838083DDCFF80111821082D9CF18
:1076F0008F929F92AF92BF92CF92DF92EF92FF92C2
:107700000F931F93CF93DF93CDB7DEB7CD55D1093C
:107710000FB6F894DEBF0FBECDBF8C016B016115B3
:10772000710519F041155105D1F460ED7DE087E355
:107730009AE00E94C98567EC7DE087E39AE00E94A9
:10774000C985B80187E39AE00E94638565EC7DE016
:1077500087E39AE00E94C98587E39AE030C0460F2C
:10776000571FDA011C920E94A32B4B0163EC7DE0B2
:1077700087E39AE00E94C985B40187E39AE00E94FA
:10778000D19B60EC7DE087E39AE00E94C985B80157
:1077900087E39AE00E9463856DEB7DE087E39AE0E2
:1077A0000E94C985BAE38B16B1E09B06F4F460EB46
:1077B0007DE080E999E00E94C98580E999E00E9416
:1077C000DA83C35ADF4F0FB6F894DEBF0FBECDBFCA
:1077D000DF91CF911F910F91FF90EF90DF90CF90AD
:1077E000BF90AF909F908F9008956EEA7DE087E301
:1077F0009AE00E94C985B60187E39AE00E946385FA
:107800006CEA7DE087E39AE00E94C98587E39AE00D
:107810000E94DA831A821982FE0133968EE3DF0119
:107820001D928A95E9F780911507909116070597A3
:1078300091F563E070E0C8010E94CE2A7C01892B9B
:10784000E9F5E0910909F0910A09808180FFB9CF3B
:1078500061E070E0C8010E94CE2A892B09F4B1CF03
:1078600064E270E0C8010E9469D7892B09F0A9CFB2
:1078700064E97DE087E39AE00E94C985B80187E367
:107880009AE00E94638587E39AE00E94DA83C80148
:107890000E9484A196CF61E070E0C8010E94CE2AC8
:1078A0007C01892B21F562E070E0C8010E94CE2A9C
:1078B0007C0169E87DE0892B09F44ACFE00EF11ED6
:1078C00060E87DE0C7010E9401CB892BC1F4F6017D
:1078D00001900020E9F73197EC19FD09329778F013
:1078E000C8010E9484A1C6010E94C8896ACF4FE3E3
:1078F00050E0B801CE0101960E945AD7DFCF64E272
:1079000070E0C8010E9469D7892B09F05ACFB701EE
:10791000CE018F5B9F4F0E94EC3ACE018F5B9F4F51
:107920000E94B714882339F1B601CE018F5B9F4FB7
:107930000E94F39C18161906F4F489818823D9F063
:1079400080911507909116070597A9F068E67DE0EC
:1079500087E39AE00E94C985BE016F5F7F4F87E38E
:107960009AE00E94638587E39AE00E94DA83CE0161
:1079700001960E9484A1CE018F5B9F4F0E94ED145F
:1079800020CFCF92DF92EF92FF926A017B0163E0FA
:10799000FC01808191810E94A297FC01892BA9F0B2
:1079A00080858D7091F4C094D094E094F094CC24B0
:1079B000CA9481859285A385B4858C219D21AE21B1
:1079C000BF2181879287A387B487FF90EF90DF90D4
:1079D000CF900895CF92DF92EF92FF926A017B01E0
:1079E00063E0FC01808191810E94A297FC01892BB8
:1079F000A9F09085892F8D7089F4907F926090878F
:107A0000CC24FF2441855285638574854C295D29EA
:107A10006E297F294187528763877487FF90EF9093
:107A2000DF90CF900895CF92DF92FF920F931F9334
:107A3000CF93DF93F12C6115710509F499C06A01A8
:107A4000EB018C01CB010E94B714F82E882309F4B6
:107A50008FC0D2FE09C0D8018C918B3009F44BC085
:107A6000E8F58A3009F44CC0D0FE09C0F801608105
:107A700086EF860F843018F0CE010E94B21CD1FE32
:107A80006EC0D80114964D915D916D917C911797C0
:107A900011968C9182958F70873038F0893008F478
:107AA0003EC08A50823008F46CC0CE010E94C314DC
:107AB000EC81FD81309709F452C080858F709EEF74
:107AC000980F923010F081114AC0D80111969C9104
:107AD000907F80858F70892B808741C08C30B9F072
:107AE00040E050E062E070E08D3009F0BDCFCE01A3
:107AF0000E94EA3CB9CF40E050E061E070E0F7CF8F
:107B000040E050E061E070E0CE010E94C13C40E006
:107B100050E062E070E0CE010E94C13CA5CFEC8154
:107B2000FD813097E1F080858F709EEF980F923045
:107B300010F0811114C04187528763877487EC81EC
:107B4000FD818085807F83608087EC81FD818085D9
:107B5000982F907F8F708067903609F4BDCF63E3D4
:107B60007CE087E39AE00E94C985C8010E94323216
:107B70008F2DDF91CF911F910F91FF90DF90CF90CC
:107B80000895CE010E94C314EACFCF92DF92EF9204
:107B9000FF926A017B0163E0FC01808191810E9478
:107BA000A297009791F0FC0120852F70223069F494
:107BB00061857285838594856C217D218E219F212D
:107BC000FF90EF90DF90CF90089560E070E0CB01E0
:107BD000F7CFCF92DF92EF92FF920F931F93CF9345
:107BE000DF9300D000D01F921F92CDB7DEB76C019B
:107BF0007B0160FF03C0E894E0F8F4F8F4FC0DC0EA
:107C00000E94A32B663971058105910530F08091A2
:107C1000150790911607059709F5A7014427577096
:107C2000052E000C660B770BC6010E94EA3C6FEA3A
:107C30007AE087E39AE00E94C9858FEF9FEF28964C
:107C40000FB6F894DEBF0FBECDBFDF91CF911F916D
:107C50000F91FF90EF90DF90CF90089519821A82D4
:107C60001B821C821D821E821F8218868A818F7051
:107C70008A8340E053E0B601CE0101960E94C633EC
:107C800040E057E060E070E0C6010E94C53DE62A92
:107C9000F72A09811A812B813C814D815E816F8198
:107CA0007885C6010E94D5A5CACF4F925F926F9288
:107CB0007F928F929F92AF92BF92CF92DF92EF927C
:107CC000FF920F931F93CF93DF93CDB7DEB72C971F
:107CD0000FB6F894DEBF0FBECDBF6D7F613071056A
:107CE00009F4BAC0DC011296ED90FC90E114F104A5
:107CF00009F4B2C04C01C7010E94501C2B013C0189
:107D000061E070E0C7010E946C1C411451046104E1
:107D1000710409F4A1C020E030E04AE754E40E9475
:107D20005CD10E94CFD369877A878B879C87672B2A
:107D3000682B692B09F490C00E94ECA49B01AC0154
:107D4000A12CB12C6501E984FA840B851C85C30143
:107D5000B2010E94D829882309F47EC0F401628010
:107D6000738070E060E0C3010E946C1C20E030E092
:107D700048EC52E40E945CD10E94CFD36B017C019D
:107D800080E00E940E19AB01BC01C3010E943D1F9F
:107D900019821A821B821C821D821E821F821886F3
:107DA0008A818F708A83D40112966D917C9140E014
:107DB00053E0CE0101960E94C633CE0101960E9487
:107DC00049142B013C0160E474E087E39AE00E94CF
:107DD0006385B301A20187E39AE00E94C79B6FE429
:107DE00074E087E39AE00E946385B701A60187E308
:107DF0009AE00E94C79B87E39AE00E94DA83C40C52
:107E0000D51CE61CF71C8A818F7080668A83CD8220
:107E1000DE82EF82F886F4016281738140E052E0F5
:107E2000CE0101960E94133D63E574E087E39AE07A
:107E30000E946385B701A60187E39AE00E94C79B71
:107E400087E39AE00E94DA8360E072E0D401129640
:107E50008D919C910E94E93D90E080E02C960FB6B8
:107E6000F894DEBF0FBECDBFDF91CF911F910F9170
:107E7000FF90EF90DF90CF90BF90AF909F908F904A
:107E80007F906F905F904F900895AF92BF92CF9286
:107E9000EF920F931F93CF93DF93CDB7DEB7C85602
:107EA000D1090FB6F894DEBF0FBECDBF5C01A2961C
:107EB0000FAFA297A3961FAFA397A4962FAFA49737
:107EC000A5963FAFA597A6964FAFA697A7965FAF8B
:107ED000A797A8966FAFA897A9967FAFA9979E2D51
:107EE00028E0FE01EF59FF4FDE01A75ABF4F019076
:107EF0000D922A95E1F7A296EFADA297E150ED30F1
:107F000008F0F0C0EC2CF0E08827E657F04C8F4FDB
:107F10000C94CBD2FF3F0840664070405C40973FD6
:107F2000F63F724072401140234049403640992349
:107F300031F0C5010E943C1C009709F447C067E07E
:107F4000CE01875A9F4F0E94B3346DE977E087E3F3
:107F50009AE00E94C9856A966FAD6A9787E39AE0B6
:107F60000E94CA9B62E977E087E39AE00E94C98594
:107F7000CE01875A9F4F0E94D534AB01BC012AE045
:107F800030E087E39AE00E94DD8487E39AE00E9474
:107F9000DA836A960FAD6A976B961FAD6B976C96F6
:107FA0002FAD6C976D963FAD6D976E964FAD6E97FA
:107FB0006F965FAD6F97A0966FADA097A1967FADBE
:107FC000A197C5010E941A3581E090E0C859DF4FA2
:107FD0000FB6F894DEBF0FBECDBFDF91CF911F91DA
:107FE0000F91EF90CF90BF90AF900895911105C081
:107FF000C5010E943C1C009749F366E0A1CF99237C
:1080000029F0C5010E943C1C009701F362E098CF63
:10801000911105C0C5010E943C1C0097B9F261E0B6
:108020008FCF40E050E061E070E0C5010E94C53DA7
:10803000672B682B692B29F4C5010E943C1C009713
:1080400029F26BE07DCF40E050E061E070E0C501D7
:108050000E94C53D672B682B692B31F0C5010E943A
:108060003C1C009709F4B2CF6AE06ACF40E050E0D0
:1080700062E070E0C5010E94C53D672B682B692B4B
:1080800031F0C5010E943C1C009709F49FCF6CE0C1
:1080900057CF40E050E062E070E0C5010E94C53D6E
:1080A000672B682B692B31F4C5010E943C1C00979B
:1080B00009F48CCF6DE044CF911106C0C5010E9438
:1080C0003C1C009709F482CF63E03ACF992331F04A
:1080D000C5010E943C1C009709F478CF65E030CFC1
:1080E00064E02ECF90E080E071CF2F923F924F92CC
:1080F0005F926F927F928F929F92AF92BF92CF9238
:10810000DF92EF92FF920F931F93CF93DF93CDB740
:10811000DEB7C35CD1090FB6F894DEBF0FBECDBF8A
:108120003C01C755DF4F0883C95AD040C655DF4FC1
:108130001883CA5AD040C555DF4F2883CB5AD04048
:10814000C455DF4F3883CC5AD040C355DF4F4883E6
:10815000CD5AD040C255DF4F5883CE5AD040C1557A
:10816000DF4F6883CF5AD040C055DF4F7883C05B64
:10817000D040CF54DF4FF982E882C15BD040CB546E
:10818000DF4FC882C55BD040C354DF4FA882CD5BB0
:10819000D0400E94A32B6B01CD54DF4F79836883BD
:1081A000C35BD040683C7105A4F466E27AE080E9E4
:1081B00099E00E94C985B60180E999E00E94D19BAF
:1081C00080E999E00E94DA83AA24AA94BA2C0C943C
:1081D0002E4A0E94ECA4C054DF4F688379838A83BF
:1081E0009B83C05CD040C655DF4F8881CA5AD040BF
:1081F0008F70282E312C2091150730911607C2540C
:10820000DF4F39832883CE5BD040CF54DF4FE881E6
:10821000F981C15BD040309721F0808181110C94AD
:10822000084ED3011B968C91882341F0C3010B9615
:10823000CF54DF4F99838883C15BD0402114310430
:1082400011F00C94514ECF54DF4FE881F981C15B9E
:10825000D040309711F00C940C4EF301238C348CE9
:108260002114310411F40C94514EC655DF4F88810E
:10827000CA5AD0408F7011F00C94514E622DCE012D
:1082800087559F4F0E948C34C756DF4F2883C959AA
:10829000D040C656DF4F3883CA59D040C556DF4F4D
:1082A0004883CB59D040C456DF4F5883CC59D04077
:1082B000C356DF4F6883CD59D040C256DF4F788315
:1082C000CE59D040C156DF4F8883CF59D040C056D9
:1082D000DF4F9883C05AD0400C94514ED3018D91FA
:1082E0009C91892B09F470CFB4E02B16310499F5D9
:1082F000C354DF4FE880CD5BD040C755DF4F0881C6
:10830000C95AD040C655DF4F1881CA5AD040C5550A
:10831000DF4F2881CB5AD040C455DF4F3881CC5A2B
:10832000D040C355DF4F4881CD5AD040C255DF4FB2
:108330005881CE5AD040C155DF4F6881CF5AD040C6
:10834000C055DF4F7881C05BD040C3010E941A3511
:108350005C010C942E4AC755DF4F1881C95AD04092
:10836000143009F4E5C248F4112309F467C0912CD4
:10837000812CAA24AA94BA2C52C388EF810F823090
:10838000B0F788E0FE01E755FF4FDE01119601903E
:108390000D928A95E1F7C655DF4F8881CA5AD040C1
:1083A000807F09F447C3CE0187559F4F0E9449142F
:1083B0006B017C01C114D104E104F10409F43AC356
:1083C000193041F4F094E094D094C094C11CD11CB5
:1083D000E11CF11CB301CE0187559F4F0E94609CA8
:1083E00060E0CE0187559F4F0E94B3346A962FAF4D
:1083F0006A976B963FAF6B976C964FAF6C976D9685
:108400005FAF6D976E966FAF6E976F967FAF6F97FA
:10841000A0968FAFA097A1969FAFA19722E02216BA
:10842000310409F45EC30CF00BC3442443942114BB
:10843000310409F457C3912C812C2CC519821A825E
:108440001B821C821D821E821F8218868A818F7069
:108450008A83C655DF4F8881CA5AD040807F09F48D
:1084600086CF0AE02016310409F41EC25CF4211400
:10847000310459F122E02216310409F4D4C0912CC0
:10848000812C0DC23BE02316310409F4B9C18CE004
:1084900028163104A1F7B301CE0101960E94609C19
:1084A000CE0187559F4F0E949514BC01CE010196C5
:1084B0000E94D83588E0FE013196DE01A755BF4FF6
:1084C00001900D928A95E1F7E7C1EF2B59F063EE29
:1084D00079E087E39AE00E94C98587E39AE00E94E9
:1084E000DA83CDCFC3010E9467588C0161E070E050
:1084F0001816190614F070E060E087E39AE00E9415
:10850000D19B61E574E087E39AE00E946385CE0128
:1085100087559F4F0E94D534AB01BC012AE030E063
:1085200087E39AE00E94DD8487E39AE00E94DA8381
:10853000CE0187559F4F1016110614F00C94FC4D78
:108540000E94D534912C812C672B682B692B89F5DF
:1085500062E0CE0187559F4F0E94B334CF56DF4F64
:108560002883C159D040CE56DF4F3883C259D040FE
:10857000CD56DF4F4883C359D040CC56DF4F588388
:10858000C459D040CB56DF4F6883C559D040CA5636
:10859000DF4F7883C659D040C956DF4F8883C7590B
:1085A000D040C856DF4F9883C859D0408824839460
:1085B000982C44244394DD24D3943AC061E0CE0146
:1085C00087559F4F0E94B334C757DF4F2883C95840
:1085D000D040C657DF4F3883CA58D040C557DF4F09
:1085E0004883CB58D040C457DF4F5883CC58D04035
:1085F000C357DF4F6883CD58D040C257DF4F7883D1
:10860000CE58D040C157DF4F8883CF58D040C05795
:10861000DF4F9883C059D04088248394982C4424F9
:108620004394D12C05C0912C812C412CDD24DA946B
:10863000B301CE0101960E94609C8A81982F929589
:108640009F70945F9F70923060F4C655DF4F9881A1
:10865000CA5AD04092959F70923019F48F70806200
:108660008A83D30118969C91973071F4C655DF4FD9
:108670008881CA5AD040807E803211F0803421F443
:108680008A818F7080628A83F301A185B285892FE8
:1086900090E0109741F0ED91FC911197068CF78DC9
:1086A000E02DCD0119957C01C755DF4F0881C95ACE
:1086B000D040C655DF4F1881CA5AD040C555DF4F4C
:1086C0002881CB5AD040C455DF4F3881CC5AD04096
:1086D000C355DF4F4881CD5AD040C255DF4F588136
:1086E000CE5AD040C155DF4F6881CF5AD040C055D7
:1086F000DF4F7881C05BD040CE0101960E941336D7
:10870000CF57DF4F2883C158D040CE57DF4F388333
:10871000C258D040CD57DF4F4883C358D040CC57C4
:10872000DF4F5883C458D040CB57DF4F6883C558BC
:10873000D040CA57DF4F7883C658D040C957DF4F63
:108740008883C758D040C857DF4F9883C858D04057
:10875000CE0101960E943232442051F1C655DF4FBE
:108760008881CA5AD04082958F709FE0980F9F7081
:10877000923020F08A5F8F708230D0F48A818295A7
:108780008F7081508230A0F42D8130E0AFEFB0E0E7
:108790000E9494D22FEF6115F4E67F0781059105C1
:1087A00034F424E630E040E050E00E9462D22D83B1
:1087B00088E0FE013196DE01A755BF4F01900D9272
:1087C0008A95E1F702E1902A512CAA24AA94BA2CA6
:1087D000D30118968C911897873009F070C5CD5445
:1087E000DF4FE881F981C35BD040EE35F1400CF0FA
:1087F0007AC36FE979E080E999E00E94C985E0CC0D
:10880000B301CE0101960E94609CC255DF4F888162
:10881000CE5AD0409A8192959F7039F0923049F0AB
:10882000912C812C552453943BC09A819F70906267
:108830009A8390E08536910514F084E690E08E836B
:1088400088E0FE013196DE01A755BF4F01900D92E1
:108850008A95E1F762E0CE0187559F4F0E948C34E4
:10886000EA962FAFEA97EB963FAFEB97EC964FAFB8
:10887000EC97ED965FAFED97EE966FAFEE97EF96B4
:108880007FAFEF97C158DF4F8883CF57D040C05894
:10889000DF4F9883C058D040812CE2E19E2E512CAE
:1088A000412CDD24DA9491CFB301CE0101960E94D0
:1088B000609CC155DF4F6881CF5AD040C055DF4F13
:1088C0007881C05BD0407170CE0101960E94993AC8
:1088D000482E912C812C55245394882311F388E041
:1088E000FE013196DE01A755BF4F01900D928A958A
:1088F000E1F762E0CE0187559F4F0E948C34E296EB
:108900002FAFE297E3963FAFE397E4964FAFE4973C
:10891000E5965FAFE597E6966FAFE697E7967FAF90
:10892000E797E8968FAFE897E9969FAFE997B4CFBE
:1089300019E02116310409F459C0C3010E94675897
:108940001816190654F562E0CE0187559F4F0E9414
:10895000B334AA962FAFAA97AB963FAFAB97AC961E
:108960004FAFAC97AD965FAFAD97AE966FAFAE978A
:10897000AF967FAFAF97E0968FAFE097E1969FAF4E
:10898000E19788248394982CAA24AA94BA2C512C79
:1089900044244394DD24D3941BCF61E0CE0187555A
:1089A0009F4F0E94B334A2962FAFA297A3963FAFDA
:1089B000A397A4964FAFA497A5965FAFA597A69649
:1089C0006FAFA697A7967FAFA797A8968FAFA897E8
:1089D000A9969FAFA99788248394982CAA24AA9437
:1089E000BA2C512C44244394D12CF2CE40E050E0D8
:1089F00061E070E0C3010E94C53D672B682B692BC5
:108A000089F040E050E061E070E0C3010E94C13CA9
:108A10008824839494E0992EAA24A394B12C512CF9
:108A2000412CCEC040E050E061E070E0C3010E9404
:108A3000EA3CEECF85E0C82ED12CE12CF12CC0CC45
:108A40008AE02816310409F4C8C19BE029163104D4
:108A500009F0F1CCC655DF4F8881CA5AD0408295C3
:108A60008F70823009F032C2C701B60124E630E0CF
:108A700040E050E00E9462D2C255DF4F8881CE5A5A
:108A8000D04090E0280F391F37FF02C030E020E0CF
:108A90002536310514F024E630E0C255DF4F288337
:108AA000CE5AD04062E0CE0187559F4F0E948C3451
:108AB0002A962FAF2A972B963FAF2B972C964FAF26
:108AC0002C972D965FAF2D972E966FAF2E972F96E2
:108AD0007FAF2F9760968FAF609761969FAF61973A
:108AE000D6C1412CD30119968D919C911A9700976C
:108AF00089F518968C9190E010E5812E912CA12C8F
:108B0000B12C8530910549F0812C912C540144976A
:108B100021F0812C912C54018A94C655DF4FE881B5
:108B2000CA5AD040E295EF70E150EB3008F046C1F0
:108B3000F0E08827E156FA4B8F4F0C94CBD2B24528
:108B4000B245DE46DE46DE46AB46694669466946C4
:108B5000E345E345DC01ED91FC91068CF78DE02DBA
:108B60001995CACFC355DF4F1881CD5AD040C701E0
:108B7000B60124E630E040E050E00E9462D2DA0123
:108B8000C901810F911DA11DB11DB7FF03C080E078
:108B900090E0DC018F3F9105A105B10529F024F09B
:108BA0008FEF90E0A0E0B0E0C355DF4F8883CD5A4F
:108BB000D040812CB2E19B2E512CAA24AA94BA2C2D
:108BC000DD24DA9405CEC355DF4F088119812A814F
:108BD0003B81CD5AD040C754DF4F088319832A8385
:108BE0003B83C95BD04014E6C116D104E104F10413
:108BF0000CF041C0A4E6B0E0C754DF4F28813981B2
:108C00004A815B81C95BD0400E9481D2C60ED71ECB
:108C1000E81EF91E81149104A104B104B9F0A50164
:108C200094010E9481D2362F272FB701A60177FF2A
:108C300003C040E050E0BA01C32ED22E7C014C1597
:108C40005D056E057F0514F46A017B01C355DF4F96
:108C5000C882D982EA82FB82CD5AD040C655DF4F06
:108C60008881CA5AD0408F708066C655DF4F88838E
:108C7000CA5AD0409ECFC701B60124E630E040E09A
:108C800050E00E9462D2C754DF4F88819981AA8147
:108C9000BB81C95BD040280F391F4A1F5B1F81145D
:108CA0009104A104B10461F057FF03C020E030E05B
:108CB000A90182169306A406B50614F4A501940131
:108CC000C355DF4F288339834A835B83CD5AD04015
:108CD00070CFC355DF4F688179818A819B81CD5ADE
:108CE000D0400E94C8D3C754DF4F688379838A83FA
:108CF0009B83C95BD040C701B60124E630E040E069
:108D000050E00E9462D2C754DF4F688179818A8126
:108D10009B81C95BD040620F731F841F951F811414
:108D20009104A104B10461F097FF03C060E070E01A
:108D3000CB0186169706A806B90614F4C501B4013E
:108D40000E94FDD0C355DF4F688379838A839B835C
:108D5000CD5AD0402ECFC355DF4F88819981AA814B
:108D6000BB81CD5AD040C80ED91EEA1EFB1E81140D
:108D70009104A104B104C9F0A4E6B0E0A5019401F6
:108D80000E9481D2362F272FB701A60177FF03C09B
:108D900040E050E0BA01C32ED22E7C014C155D0597
:108DA0006E057F0514F46A017B01C355DF4FC8824D
:108DB000D982EA82FB82CD5AD040FBCE88E0FE0108
:108DC0003196DE01A755BF4F01900D928A95E1F7CC
:108DD000912C812C55245394F0CEC655DF4F8881B9
:108DE000CA5AD04082958F70823009F055C0C701B1
:108DF000B60124E630E040E050E00E9462D2C15566
:108E0000DF4F8881CF5AD040C055DF4F6881C05BAB
:108E1000D040962F9170280F391F2E3691E03907D8
:108E20002CF437FF05C02DE631E002C030E020E031
:108E3000C155DF4F2883CF5AD040C055DF4F8881BE
:108E4000C05BD04030FB80F9C055DF4F8883C05BEA
:108E5000D04062E0CE0187559F4F0E948C346296CD
:108E60002FAF629763963FAF639764964FAF649757
:108E700065965FAF659766966FAF669767967FAFAB
:108E8000679768968FAF689769969FAF6997812CAF
:108E9000A2E19A2E512C18C088E0FE013196DE0125
:108EA000A755BF4F01900D928A95E1F767ED79E0E4
:108EB00080E999E00E94C98580E999E00E94DA83FF
:108EC000912C812C55245394412C77CE88E0FE01BF
:108ED0003196DE01A755BF4F01900D928A95E1F7BB
:108EE0006BEC79E0E5CFCB54DF4F1881C55BD04008
:108EF000112309F467C01296ED91FC9180858F7063
:108F0000853009F070C0C254DF4FE881F981CE5B33
:108F1000D040359709F467C0C3010E94675821E02B
:108F2000181619060CF020E0D22ECF54DF4F4881DE
:108F30005981C15BD040C354DF4F2881CD5BD04005
:108F4000BE0167557F4FD30112968D919C910E946F
:108F5000A057B1E02B16310409F045C0C655DF4FCC
:108F60001881CA5AD040812F807FE9F1C354DF4F66
:108F7000C880CD5BD040ED2CC755DF4F0881C95A62
:108F8000D040C555DF4F2881CB5AD040C455DF4F64
:108F90003881CC5AD040C355DF4F4881CD5AD0409C
:108FA000C255DF4F5881CE5AD040C155DF4F68813E
:108FB000CF5AD040C055DF4F7881C05BD040C3014D
:108FC0000E94453FC755DF4F8881C95AD040853040
:108FD00009F444C170F48330C9F1CD54DF4F1882D5
:108FE000C35BD040B8C0CB54DF4F1882C55BD040C4
:108FF000E9CF863009F47CC0873079F7C3010E943D
:10900000E11C182F863009F062C063E779E087E33E
:109010009AE00E94C98566E070E087E39AE00E94CA
:10902000D19B87E39AE00E94DA8362E0CE01875504
:109030009F4F0E94B33429AF3AAF4BAF5CAF6DAFD7
:109040007EAF8FAF21969FAF21973DC0C3010E9495
:10905000E11C853021F093E0A92EB12CFFC16AE814
:1090600079E087E39AE00E94C98565E070E087E3D4
:109070009AE00E94D19B87E39AE00E94DA83B301D1
:10908000CE0187559F4F0E94609C61E0CE018755BD
:109090009F4F0E94B33422962FAF229723963FAF63
:1090A000239724964FAF249725965FAF2597269652
:1090B0006FAF269727967FAF279728968FAF289771
:1090C00029969FAF2997689480F890F886CF65E538
:1090D00079E087E39AE00E94C985612F70E087E319
:1090E0009AE00E94D19B87E39AE00E94DA83B3CF93
:1090F00040E050E061E070E0C3010E94C53D672B95
:10910000682B692B09F0A7C0EFEFDE129AC0C301EC
:109110000E946758181619060CF496C0B301CE01C8
:1091200087559F4F0E94609C61E0CE0187559F4FFD
:109130000E94B33429AB3AAB4BAB5CAB6DAB7EABAF
:109140008FAB98AF689480F890F8F6E0CD54DF4F7D
:10915000F883C35BD04084010160C655DF4F88812E
:10916000CA5AD040982F9F70923050F4C755DF4FA5
:109170009881C95AD040992319F084010160116087
:10918000807F09F491C01260CB54DF4F2881C55B0A
:10919000D04021111D7FA801B301CE0187559F4FFB
:1091A0000E94133D4801AA24A394B12C5110C7C5B5
:1091B000D30119968D919C91009709F06FC340E0FF
:1091C00050E062E070E0C3010E94C53D672B682B50
:1091D000692B09F495C367EF77E080E999E00E9475
:1091E000C98580E999E00E94DA8392FCF0C46CEDB5
:1091F00077E087E39AE00E94C985B50187E39AE0AA
:109200000E94D19B65ED77E087E39AE00E94C985D3
:109210000E94ECA4AB01BC01C054DF4F088119814E
:109220002A813B81C05CD040401B510B620B730B09
:1092300087E39AE00E94C79B87E39AE00E94DA8363
:109240000DC1DD2009F46ACF6BE379E087E39AE092
:109250000E94C98500CF66E279E0F8CF0FEFD01207
:1092600009C0C3010E946758181619062CF069E05E
:1092700079E0ECCFDD20D9F362E0CE0187559F4F36
:109280000E94B33429A73AA74BA75CA76DA77EA776
:109290008FA798AB689480F890F815E0CD54DF4F15
:1092A0001883C35BD04057CF40E052E0B301CE01FA
:1092B00087559F4F0E94C633811165CF65CF3FEF21
:1092C000D312E7C0C3010E946758DD24D394181657
:1092D00019060CF4E1C0D12C6BEF78E087E39AE03B
:1092E0000E94C9850D2D0D2C000C110BC754DF4FAA
:1092F00019830883C95BD040B80187E39AE00E94D4
:10930000D19B64EF78E087E39AE00E94C985642DE1
:1093100070E087E39AE00E94D19B87E39AE00E9485
:10932000DA83CF54DF4FE880F980C15BD040E1148D
:10933000F10409F4BAC06DE373E2C7010E9401CBE6
:1093400001E010E0892B09F44BC069E373E2C70127
:109350000E9401CB02E010E0892B09F441C060EDCE
:1093600077E0C7010E9401CB05E010E0892BC1F135
:109370006CEC77E0C7010E9401CB06E010E0892B7E
:1093800079F16EEF72E2C7010E9401CB03E110E0B8
:10939000892B31F169EF72E2C7010E9401CB04E130
:1093A00010E0892BE9F063E073E2C7010E9401CB72
:1093B0000EE010E0892BA1F06CEE72E2C7010E9472
:1093C00001CB0FE010E0892B59F065EF72E2C70185
:1093D0000E9401CB10E000E0892B11F405E110E0C0
:1093E000C3010E94E11C282F30E0CD54DF4F3983A8
:1093F0002883C35BD040232B61F4C754DF4F88819F
:109400009981C95BD040CD54DF4F99838883C35B7A
:10941000D0400115110509F491C0CD54DF4FA8814A
:10942000B981C35BD040A017B107C9F168ED78E0FE
:1094300087E39AE00E94C985CD54DF4F6881798126
:10944000C35BD04087E39AE00E94D19B87E39AE018
:109450000E94DA836DEFA62EBB24BA94C501CD53CA
:10946000DF4F0FB6F894DEBF0FBECDBFDF91CF91B7
:109470001F910F91FF90EF90DF90CF90BF90AF9032
:109480009F908F907F906F905F904F903F902F9024
:109490000895DD2009F420CF442443941DCFCF54F8
:1094A000DF4F19821882C15BD040B1E02B16310426
:1094B000A9F4CB54DF4FE881C55BD040EE2399F08F
:1094C000C655DF4F8881CA5AD040807FF1E0CB5427
:1094D000DF4FF883C55BD040811105C0CB54DF4F0F
:1094E0001882C55BD040C755DF4F0881C95AD040AC
:1094F000CD54DF4F0883C35BD040063108F0B8C1BC
:10950000E02FF0E08827E857F54B8F4F0C94CBD233
:10951000DB4AFB4BEB4B1E4BDB4ACE4B944B654B74
:10952000DB4ADB4A354C354C454C454C164C164C09
:10953000384C384C384C164C164C164CF30181857F
:109540009285009709F4B1CFDC01ED91FC9106887A
:10955000F789E02DC354DF4FA880CD5BD040C42CE9
:10956000C755DF4F0881C95AD040C655DF4F188113
:10957000CA5AD040C555DF4F2881CB5AD040C45578
:10958000DF4F3881CC5AD040C355DF4F4881CD5A88
:10959000D040C255DF4F5881CE5AD040C155DF4F21
:1095A0006881CF5AD040C055DF4F7881C05BD04032
:1095B00019950C94A841CD54DF4F1882C35BD0405D
:1095C000CB54DF4F2881C55BD040222309F4EECD78
:1095D0003D2D3170E32EC354DF4FC880CD5BD040AA
:1095E000C755DF4F0881C95AD040C655DF4F188193
:1095F000CA5AD040C555DF4F2881CB5AD040C455F8
:10960000DF4F3881CC5AD040C355DF4F4881CD5A07
:10961000D040C255DF4F5881CE5AD040C155DF4FA0
:109620006881CF5AD040C055DF4F7881C05BD040B1
:10963000C3010E94453FE89491F8B8CDC3010E9450
:10964000E11C853009F007CD63EC78E087E39AE010
:109650000E94C98565E070E087E39AE00E94D19B93
:1096600087E39AE00E94DA83B301CE0187559F4FCA
:109670000E94609CD30118968C918530B9F46EE0FD
:10968000CE0187559F4F0E94B33429A33AA34BA321
:109690005CA36DA37EA38FA398A7689480F890F82D
:1096A000CD54DF4F1882C35BD0406FC061E0CE0164
:1096B00087559F4F0E94B334298F3A8F4B8F5C8F11
:1096C0006D8F7E8F8F8F98A3E8CFC3010E94E11C1E
:1096D000182F863031F56CEA78E087E39AE00E9433
:1096E000C98566E070E087E39AE00E94D19B87E33A
:1096F0009AE00E94DA8362E0CE0187559F4F0E9474
:10970000B334298B3A8B4B8B5C8B6D8B7E8B8F8B21
:10971000988F40E050E068E070E0C3010E94C13CD7
:10972000BCCF6EE878E0D5CC40E050E061E070E07E
:10973000C3010E94C53D672B682B692B61F5D110D1
:1097400027C0B301CE0187559F4F0E94609C61E006
:10975000CE0187559F4F0E94B33429873A874B87A4
:109760005C876D877E878F87988B40E050E068E04C
:1097700070E0C3010E94EA3C689480F890F8B6E07B
:10978000CD54DF4FB883C35BD0404424439418CFFB
:1097900064E778E05BCD6FE578E058CDDD20C1F07F
:1097A00062E0CE0187559F4F0E94B33429833A83EC
:1097B0004B835C836D837E838F839887689480F866
:1097C00090F8E5E0CD54DF4FE883C35BD040DDCFB8
:1097D00062E478E03BCDC655DF4F8881CA5AD0405D
:1097E0008F70823008F05CCFC3010E94E11C85308D
:1097F00009F053CF30CCC655DF4F8881CA5AD040CC
:109800008F70823008F04CCFDD2081F069E278E083
:1098100087E39AE00E94C98561E0C3010E94B21CFF
:1098200060E071E1C3010E94E93D15CCC655DF4FF0
:109830008881CA5AD040982F9F70923008F030CF5C
:10984000CD54DF4FF881C35BD040FF2309F49DCF97
:10985000807F31F4B301CE0187559F4F0E94609CF9
:10986000689480F803E0902A1BCF689492F818CF90
:10987000C655DF4F8881CA5AD040807F19F468945A
:1098800090F80ECF13E0912A0BCFCD54DF4F188202
:10989000C35BD040812C54E0952E77CFDC01ED9155
:1098A000FC91028CF38DE02DC755DF4F0881C95A1A
:1098B000D040C655DF4F1881CA5AD040C555DF4F3A
:1098C0002881CB5AD040C455DF4F3881CC5AD04084
:1098D000C355DF4F4881CD5AD040C255DF4F588124
:1098E000CE5AD040C155DF4F6881CF5AD040C055C5
:1098F000DF4F7881C05BD0401995811160CC6BCC73
:10990000F30181859285892B09F473C08114910438
:1099100039F0A401B301CE0187559F4F0E94133D3A
:10992000D30119968D919C91CF54DF4FE880F98037
:10993000C15BD040DC01ED91FC910688F789E02DF8
:10994000C354DF4FA880CD5BD040C42CC755DF4F38
:109950000881C95AD040C655DF4F1881CA5AD04035
:10996000C555DF4F2881CB5AD040C455DF4F3881D1
:10997000CC5AD040C355DF4F4881CD5AD040C25554
:10998000DF4F5881CE5AD040C155DF4F6881CF5A42
:10999000D040C055DF4F7881C05BD04019955C0145
:1099A000F30181859285DC01ED91FC91068CF78DA8
:1099B000E02D1995059711F4689480F892FCFFC08A
:1099C000CD54DF4FB881C35BD040BB2321F06B2F58
:1099D000C3010E94B21CC254DF4FE881F981CE5B03
:1099E000D040B401359709F402CCC3010E94E93D8F
:1099F000FECB8085853009F474C0863009F7C755E1
:109A0000DF4FD880C95AD040DD2009F46AC0C301B5
:109A10000E943E9C8C018114910439F0A401B30191
:109A2000CE0187559F4F0E94133D0115110541F24C
:109A3000F12CE12C17FF06C0119501951109EE24B8
:109A4000E394F12CC80101978634910508F0B8CF52
:109A5000C02E61E0802F0E9448A3EFEFED0DE531AD
:109A600010F5F0E08827E85CF24B8F4F0C94CBD2D6
:109A70004D4D4F4D534D534D4F4D4D4D4F4D534DFE
:109A8000534D534D534D534D534D4D4D4D4D534DE2
:109A9000534D534D534D4D4D4D4DF1E0EF266E2D31
:109AA0008C2D0E941AA362EF77E087E39AE00E9470
:109AB000C985B80187E39AE00E94D19B60EF77E007
:109AC00087E39AE00E94C985B70187E39AE00E9484
:109AD000D19B87E39AE00E94DA83689480F890F83B
:109AE0006EC08114910439F0A401B301CE018755F1
:109AF0009F4F0E94133D02E02016310409F463C019
:109B000013E02116310429F02A94232809F058CFB4
:109B1000E4CFC3010E94501C892B49F4D301ED917D
:109B2000FC916081718188E694E00E94BAA8CE0120
:109B300087559F4F0E94021420E030E048EC52E429
:109B40000E945CD10E94C8D3CB54DF4F68837983D5
:109B50008A839B83C55BD040CB54DF4FC880D980BC
:109B6000C55BD04088E00E940E191B012C016CEEF1
:109B700077E087E39AE00E94C985CB54DF4F688184
:109B80007981C55BD04087E39AE00E94D19B67EE64
:109B900077E087E39AE00E94C985B201A1016627B8
:109BA00077272AE087E39AE00E948E8387E39AE092
:109BB0000E94DA83B101A601C3010E943D1FAA24BD
:109BC000A394B12CFDCE689480F891F8F8CFC254DC
:109BD000DF4F08811981CE5BD0400530110509F4B3
:109BE00006CB40E054E0B301CE0187559F4F0E9461
:109BF000133D60E074E0F9CE0E94D534672B682BEA
:109C0000692B11F00C94DE42912C812C0C940F43A3
:109C10002114310409F045C08081882311F40C948B
:109C20002D41CE018F549F4F0E94B83A1C01C6555A
:109C3000DF4F8881CA5AD0408F7071F5622DCE01F6
:109C400087559F4F0E948C34CF55DF4F2883C15AD0
:109C5000D040CE55DF4F3883C25AD040CD55DF4F6C
:109C60004883C35AD040CC55DF4F5883C45AD040A4
:109C7000CB55DF4F6883C55AD040CA55DF4F788334
:109C8000C65AD040C955DF4F8883C75AD040C855FF
:109C9000DF4F9883C85AD0402114310411F40C943A
:109CA0002D416BE17AE087E39AE00E94C985B60115
:109CB00087E39AE00E94D19B64E17AE087E39AE02F
:109CC0000E94C985D301ED91FC916081718187E388
:109CD0009AE00E9463856EE07AE087E39AE00E9452
:109CE000C985CF54DF4F68817981C15BD04087E35C
:109CF0009AE00E9463856CE07AE087E39AE00E9434
:109D0000C985CE0187559F4F0E943232CF54DF4F15
:109D1000E881F981C15BD040309711F40C946E4119
:109D20008081843211F00C946E4168EF79E087E312
:109D30009AE00E94C98587E39AE00E94DA838CEF5B
:109D4000A82EBB24BA948ACB2F923F924F925F9257
:109D50006F927F928F929F92AF92BF92CF92DF923B
:109D6000EF92FF920F931F93CF93DF93CDB7DEB7A0
:109D7000C955D1090FB6F894DEBF0FBECDBF3C0167
:109D8000562E6296EFAE62976396FFAE6397649627
:109D90000FAF649765961FAF659766962FAF66976E
:109DA00067963FAF679768964FAF689769965FAFC2
:109DB00069976A96CFAE6A972D2C4A2C3B2C009758
:109DC00009F464C1FC0180858F70843009F449C1B5
:109DD00028F4882309F44EC180E02DC0853009F4B1
:109DE00044C08630C9F767E774E0C3010E942A9730
:109DF0004C01009709F46FC0B12CA12CD12CC12CBF
:109E00006296EFAC62976396FFAC639764960FAD72
:109E1000649765961FAD659766962FAD66976796B2
:109E20003FAD679768964FAD689769965FAD699744
:109E3000652D0E94A44EC75ADF4F0FB6F894DEBFBF
:109E40000FBECDBFDF91CF911F910F91FF90EF908B
:109E5000DF90CF90BF90AF909F908F907F906F904A
:109E60005F904F903F902F900895809111078F5FE2
:109E700080931107868097808114910431F1A42C7E
:109E8000B32C6A96CFAC6A97D22C6296EFAC6297ED
:109E90006396FFAC639764960FAD649765961FADAC
:109EA000659766962FAD669767963FAD67976896FC
:109EB0004FAD689769965FAD6997652DC4010E94A3
:109EC000A44EF40182809380D7CF809111078150F6
:109ED0008093110781CF6BE774E0C3010E942A973A
:109EE0007C0160E874E0C3010E942A976C01552050
:109EF00039F0F1E05F1609F495C010E000E00CC005
:109F000065E874E0C3010E942A974C016AE874E096
:109F1000C3010E942A978C018114910409F4430122
:109F20000115110509F48301E114F10421F46A9685
:109F3000EFAC6A97F22CC114D10411F4C42CD32CC9
:109F40008114910409F49FC0F40180858F708430DE
:109F500009F099C0818492840115110509F49EC00D
:109F6000F80180858F70843009F098C001851285D2
:109F7000E114F10409F4E0C08114910409F49DC0D6
:109F800066EB78E187E39AE00E94C985F701618575
:109F9000728587E39AE00E94638561EB78E187E34D
:109FA0009AE00E94C985B40187E39AE00E94638524
:109FB00087E39AE00E94DA83CE018F5A9F4F0E9476
:109FC0003232C114D10409F0C0C0F70180858F700E
:109FD000843009F00CC161857285CE0101960E9422
:109FE000EC3ACE0101960E94B7148823B1F00E948A
:109FF000A32B6B01683C71050CF073C06DE778E131
:10A0000080E999E00E94C985B60180E999E00E9443
:10A01000D19B80E999E00E94DA83CE0101960E94EB
:10A02000ED14E5C06FE874E0C3010E942A974C016B
:10A0300064E974E0C3010E942A978C0181149104A1
:10A0400009F0D7C065E874E0C3010E942A974C016B
:10A050000115110509F45ACF892B09F065CF430189
:10A0600063CF10E000E0912C812CD12CC12CF12C7D
:10A07000E12C52CF10E000E0912C812CD12CC12C8E
:10A08000F12CE12C51CF912C812C66CFCA2CDB2CEA
:10A090006A96EFAC6A97F22C912C812C00E020E0BC
:10A0A00033E040E150E0BE016F5B7F4FCE018F5A3D
:10A0B0009F4F0E9411308C015BCF67EA78E187E304
:10A0C0009AE00E94C985F7016185728587E39AE06D
:10A0D0000E94638562EA78E187E39AE00E94C9857D
:10A0E0006BCF8114910431F0B401CE0101960E942E
:10A0F000F39C93CFA12CCC24C394F12CE12C629639
:10A100000FAD629763961FAD639764962FAD64970A
:10A1100065963FAD659766964FAD669767965FAD5E
:10A12000679768966FAD689769967FAD6997CE011E
:10A1300001960E94754071CFC114D10409F457C033
:10A140000115110509F453C004C00115110509F4E6
:10A150003CCFF60180858F70843009F044C06BE9F4
:10A1600078E187E39AE00E94C985F60161857285EE
:10A1700087E39AE00E94638566E978E187E39AE0E5
:10A180000E94C985B80187E39AE00E94638587E34E
:10A190009AE00E94DA83F6016185728540E450E01E
:10A1A000CE0101960E945AD70E9448978823D9F081
:10A1B0008091CA08811117C06FE270E0CE0101964C
:10A1C0000E9421D7892B51F4F6012185328543E085
:10A1D00050E060E4CE0101960E943A2AB801CE0117
:10A1E00001960E94BAA5E114F10409F0EECE81E0D7
:10A1F00022CE892B09F098CE89CE4F925F926F9232
:10A200007F928F929F92AF92BF92CF92DF92EF9206
:10A21000FF920F931F93CF93DF93CDB7DEB769976C
:10A220000FB6F894DEBF0FBECDBF0E94ECA49B0119
:10A23000AC0160914B0670914C0680914D06909157
:10A240004E06A12CB12C650118E8E12E13E1F12E88
:10A2500000E010E00E94D829882369F1E091A4066B
:10A26000F091A5069281913061F0E0F16CE378E124
:10A27000923049F063E278E1943029F064E078E1CB
:10A2800002C06FE078E180E999E00E94C98580E929
:10A2900099E00E94DA838091A4069091A5060E941D
:10A2A00005260E94ECA460934B0670934C068093A5
:10A2B0004D0690934E0669960FB6F894DEBF0FBE1A
:10A2C000CDBFDF91CF911F910F91FF90EF90DF9065
:10A2D000CF90BF90AF909F908F907F906F905F9046
:10A2E0004F900895CF010E945B19811108C06FEE55
:10A2F00077E186E899E00E94ED850E942C28E090A5
:10A300004906F0904A06E114F10431F0E091190792
:10A31000F0911A07309759F461EE77E180E999E0FE
:10A320000E94C98580E999E00E94DA83BACF8091C2
:10A33000470690914806892B61F480858F7086309E
:10A3400041F486819781009721F09093480680938D
:10A350004706E091A406F091A506309721F085E824
:10A3600096E696878587E0914706F09148063097F4
:10A3700009F448C1BE016E5E7F4F808191810E94C9
:10A380004113882309F43EC18A89883209F03AC111
:10A39000AE014F5F5F4FBE016E5E7F4FC7010E94EF
:10A3A0009B26811107C0C12CD12C2EEFE22E22EC6E
:10A3B000F22E3DC06A8170E0762F6627770F770F07
:10A3C000770F298148E0249F90011124262B372BF9
:10A3D0008A898031D1F4688570E08F81FB01E81BA8
:10A3E000F109CF019695982F8827979587950E9418
:10A3F000B7D2CB014097B90153E0660F771F5A954A
:10A40000E1F760789C01260F371F2138F4EE3F07F3
:10A4100054F2B901330F880B990B0E94FDD020E054
:10A4200030E040E05CE30E945CD16B017C018090F5
:10A430004706909048068114910409F480C08091E9
:10A44000190790911A07892B09F479C0C4010E9459
:10A4500089135C0187E39AE00E94DA836CED77E16F
:10A4600087E39AE00E94C98522E0B701A60187E34D
:10A470009AE00E94F78369ED77E187E39AE00E9412
:10A48000C985F4016081718187E39AE00E94638548
:10A4900066ED77E187E39AE00E94C98520E030E02D
:10A4A0004EEF52ECC701B6010E94F6D0882309F4A2
:10A4B000B4C020E030E04AEA52E4C701B6010E948D
:10A4C000F6D0882309F4A9C020E030E0A901C70133
:10A4D000B6010E94F6D0882309F49FC0A114B104EC
:10A4E00029F0B50187E39AE00E94638587E39AE04B
:10A4F0000E94DA8319821A821B821C828A818F70E1
:10A5000080678A83CD82DE82EF82F88663E0CE01A7
:10A5100001960E948C342A873B874C875D876E8723
:10A520007F87888B998BB12CA12CD12CC12C7901E0
:10A530008A019B01AC016FEFC4010E94A44EE09020
:10A540004906F0904A068A89803109F47AC0BE0132
:10A550006E5E7F4FC7010E94B526182F882309F42D
:10A5600051C0F701858196810E940526882309F450
:10A5700049C0BE016E5E7F4FF701858196810E94C2
:10A58000D825F701408164E4858196810E94B22537
:10A59000F70182818823B1F119508EEE882E82E076
:10A5A000982E133040F4E12FF0E0EE0FFF1FED5432
:10A5B000FD4F80809180F7018381882309F443C097
:10A5C0008081811140C00E94ECA42B013C01092C28
:10A5D000000CAA08BB08AE014F5F5F4FBE016E5E64
:10A5E0007F4FC7010E944626898181110BC00E94BE
:10A5F000ECA4681979098A099B0964157505860513
:10A60000970548F3E0914706F091480682819381CF
:10A61000909348068093470644CEA114B10409F4F0
:10A620008ECF65EC77E187E39AE00E94C985B5019A
:10A6300087E39AE00E94638587E39AE00E94DA83C9
:10A640007ECF1CE08ECFB401990C880B990B0E9431
:10A65000B9A4D8CF6F927F928F929F92AF92BF9200
:10A66000CF92DF92EF92FF920F931F93CF93DF93DE
:10A67000CDB7DEB7A0970FB6F894DEBF0FBECDBF43
:10A680008C01862E7A01DC018D919C911197892B8A
:10A6900009F460C01496ED91FC91309709F45AC00A
:10A6A00080818071BFEF6B1357C0B1F481E0A09639
:10A6B0000FB6F894DEBF0FBECDBFDF91CF911F91D3
:10A6C0000F91FF90EF90DF90CF90BF90AF909F9051
:10A6D0008F907F906F9008954330510539F38180BA
:10A6E00082942FE0822262E477E087E39AE00E947E
:10A6F000C985D80113966C9187E39AE00E94CA9BA2
:10A7000060E477E087E39AE00E94C985D801149657
:10A71000ED91FC9161816F7087E39AE00E94CA9B82
:10A720006DE377E087E39AE00E94C985682D87E3AF
:10A730009AE00E94CA9B87E39AE00E94DA83D801DC
:10A740001496ED91FC9181818F70881207C08081F1
:10A750008F7E808380E0ABCF8111FCCF198E1A8E63
:10A760001B8E1C8E1D8E1E8E1F8E18A28A8D8F70C2
:10A770008A8FD8011496ED91FC9181818F70881594
:10A7800079F1B3E0EB16F10459F16BE377E087E37D
:10A790009AE00E94C985F801638187E39AE00E94EC
:10A7A000CA9B69E377E087E39AE00E94C985D801F4
:10A7B0001496ED91FC9161816F7087E39AE00E949D
:10A7C000CA9B66E377E087E39AE00E94C985682D1B
:10A7D00087E39AE00E94CA9B87E39AE00E94DA83AB
:10A7E000F80120813181FCE0F81508F416C1E82D4C
:10A7F000F0E08827E150FC4A8F4F0C94CBD20C54E8
:10A800004954CA54E154ED54CA54A354CA54F054A0
:10A81000FB54B754FE540A55D8011496CD90DC90E1
:10A82000F60181818F70853009F4F7C050F48230D1
:10A83000C1F067EA74E0C9010E942A973C01912C9B
:10A840004BC08730D1F08A30A1F760EA74E0C901CB
:10A850000E942A973C01D6019C9092FA992490F884
:10A860003BC06AE974E0C9010E942A973C01D60105
:10A870009C9090FA992490F82FC069E974E0C9017E
:10A880000E942A973C01F601908091FA992490F851
:10A8900023C06CEA74E0C9010E942A973C01D801E8
:10A8A0001496ED91FC91808180FB992490F8982F6B
:10A8B0009E7F80FF916090836114710469F461E070
:10A8C000CE0149960E94B334298B3A8B4B8B5C8B1B
:10A8D0006D8B7E8B8F8B988FF801A080B1806BE79A
:10A8E00074E0C5010E942A976C0160E874E0C5011C
:10A8F0000E942A975C01892B81F4C114D10469F468
:10A9000060E0CE0149960E94B33429833A834B8399
:10A910005C836D837E838F839887D8011496ED9135
:10A92000FC916114710409F07CC0898D811179C09A
:10A93000B82DBF708B2E8181807F882A8182808193
:10A940008F7E8083B3CE61EB74E0C9010E942A97A9
:10A950003C01D8011496ED91FC91808181FB9924F2
:10A9600090F8982F9D7F81FF92609083B5CF67EB21
:10A9700074E0C9010E942A973C01D8011496ED9118
:10A98000FC91808182FB992490F8982F9B7F82FF15
:10A990009460EBCF67EA74E0C9010E942A973C01FA
:10A9A000892B09F04CCF62E0CE0149960E94B33466
:10A9B00029873A874B875C876D877E878F87988B3F
:10A9C0003ECF6DEB74E0C9010E942A973C01D8018B
:10A9D0001496ED91FC9190804CCF62EC74E0F3CF33
:10A9E00068EC74E0C9010E942A973C01D8011496D2
:10A9F000ED91FC9149CF6EEC74E0F4CF65ED74E01D
:10AA0000C9010E942A973C01D8011496ED91FC914E
:10AA1000908023CF6BED74E0F3CF912C712C612CDF
:10AA20005BCF83E0E816F104B9F0982D9F70892E72
:10AA30008181807F882A818280818F7E8083E98CDA
:10AA4000FA8C0B8D1C8D2D8D3E8D4F8D58A1692D4F
:10AA5000C3010E94A44E2ACE81818F70881509F40B
:10AA600025CE829490EF8922882A8182808180611C
:10AA700068CF2F923F924F925F926F927F928F9208
:10AA80009F92AF92BF92CF92DF92EF92FF920F937D
:10AA90001F93CF93DF93CDB7DEB763970FB6F894CC
:10AAA000DEBF0FBECDBF4C013B0140E058E060E08F
:10AAB00070E00E94C53D672B682B692B09F45CC0D0
:10AAC00019821A821B821C821D821E821F82188696
:10AAD0008A818F708A8340E053E0B401CE010196F1
:10AAE0000E94C633D40119968D919C91892B09F44B
:10AAF00043C040E058E060E070E0C4010E94C13C07
:10AB000069E77AE087E39AE00E94C985F4018185CC
:10AB10009285DC01ED91FC910688F789E02DA12C4E
:10AB2000CC24C394F12CE12C09811A812B813C8126
:10AB30004D815E816F81788519958F3F9807E1F08F
:10AB4000D401ED91FC9160817181892B09F0B8C02D
:10AB500087E39AE00E94638567E77AE087E39AE0FB
:10AB60000E94C9856FE67AE087E39AE00E94C98572
:10AB700087E39AE00E94DA8365E0F40180819181A5
:10AB80000E94A2976C01009709F4D0C0DC011896CE
:10AB9000BC91B98BBB2EB2942FE0B222FC01218470
:10ABA0003284438454840E94ECA4BB2009F4BEC0C8
:10ABB000261A370A480A590A19861A861B861C86DD
:10ABC000B9861A851F70106A1A872D863E864F86B1
:10ABD000588AF4E06F16710439F5E12C90E2F92EF1
:10ABE0000B2D2B853C854D855E856F857889C4014D
:10ABF0000E94D5A5C201B10128EE33E040E050E04B
:10AC00000E9462D2BA01A9012AE030E087E39AE00B
:10AC10000E94DD8460EA7AE087E39AE00E94C985B9
:10AC200087E39AE00E94DA8357FE80C022E0221672
:10AC30003104410420E852060CF478C00E94A32B92
:10AC40001B017B8B6A8BE12C80E2F82E09851A852B
:10AC50002B853C854D855E856F857889C4010E9472
:10AC6000D5A58A899B89883C9105BCF567E87AE07F
:10AC700080E999E00E94C985B10180E999E00E94CC
:10AC8000D19B80E999E00E94DA838FEF9FEF639672
:10AC90000FB6F894DEBF0FBECDBFDF91CF911F91ED
:10ACA0000F91FF90EF90DF90CF90BF90AF909F906B
:10ACB0008F907F906F905F904F903F902F9008956E
:10ACC00087E39AE00E9463856DE67AE087E39AE085
:10ACD0000E94C98569E67AE047CFD60118968C9123
:10ACE00018978F7018968C9319821A821B821C8277
:10ACF0001D821E821F8218868A818F708A83B98284
:10AD000089898F70AA24A394873009F0A12CCC24C0
:10AD1000C394F12CE12C09811A812B813C814D8156
:10AD20005E816F817885C4010E947540B1E06B1629
:10AD30007104E9F440E053E060E070E0C4010E9477
:10AD4000C53D611571058105910589F020911507B3
:10AD5000309116072630310551F4C4010E94E93DB7
:10AD600040E053E060E070E0C4010E94C13CF401A7
:10AD700081859285009719F490E080E088CFDC010E
:10AD8000ED91FC910484F585E02D1995892BA1F3B3
:10AD9000F40181859285DC01ED91FC910480F581BF
:10ADA000E02DB301199573CFAF92BF92CF92DF928E
:10ADB000EF92FF920F931F93CF93DF93CDB7DEB740
:10ADC0006D970FB6F894DEBF0FBECDBF0E94ECA406
:10ADD0009B01AC016091410670914206809143064F
:10ADE00090914406A12CB12C650118EEE12E13E0E0
:10ADF000F12E00E010E00E94D829F82E882351F0AF
:10AE00000E94ECA46093410670934206809343062F
:10AE100090934406809111078F5F80931107E09112
:10AE20001707F09118070681178194E0C92ED12CDD
:10AE3000F11003C082E0C82ED12CA0901707B0906B
:10AE40001807A114B10429F10115110511F1F80138
:10AE500080858F708530A9F7C8010E942E9C8230B2
:10AE600080F3B801CE0101960E949520CE01019693
:10AE70000E94B714882329F0B601CE0101960E94E2
:10AE80003955F80102811381CE0101960E94ED141B
:10AE9000D4CF8091110781508093110780911507BD
:10AEA000909116070597D9F1FF20C9F110E0609144
:10AEB0003F06709140066115710589F111112FC08F
:10AEC000FB0180858F70853091F4CE0101960E9440
:10AED000952061E070E0CE0101960E94395511E0A5
:10AEE000892B09F410E0CE0101960E94ED14E09147
:10AEF0003F06F0914006309791F0828193819093C4
:10AF0000400680933F06892B91F6E0911707F09158
:10AF10001807868197819093400680933F066D962F
:10AF20000FB6F894DEBF0FBECDBFDF91CF911F915A
:10AF30000F91FF90EF90DF90CF90BF90AF9008956A
:10AF40002F923F924F925F926F927F928F929F9239
:10AF5000AF92CF92DF92EF92FF920F931F93CF9316
:10AF6000DF93CDB7DEB76D970FB6F894DEBF0FBE97
:10AF7000CDBF009709F4A9C0FC0130853F70353082
:10AF800009F0A3C0D22E1A014B0166807780809110
:10AF900011078F5F809311076114710409F490C049
:10AFA000F30180858F70843009F086C061857285D9
:10AFB00080911707909118070E942A972C010097FB
:10AFC00009F47AC0FC0180858F70853009F074C067
:10AFD000B201CE0101960E94952081149104B1F036
:10AFE000CE0101960E94B714882381F0AD2CC12CAC
:10AFF0007101F401008111812281338144815581E5
:10B0000066817781CE0101960E94754060E0C201A1
:10B010000E94A2970097E9F1FC0120852F70223051
:10B02000C1F581859285A385B4850797A105B105F2
:10B0300081F561E0C2010E94A2972D2DA101B4010A
:10B040000E94A0578114910499F5882389F1809179
:10B050001107815080931107CE0101960E94ED14D3
:10B0600081E06D960FB6F894DEBF0FBECDBFDF91C5
:10B07000CF911F910F91FF90EF90DF90CF90AF9005
:10B080009F908F907F906F905F904F903F902F9008
:10B0900008958114910461F4CE0101960E94B714C1
:10B0A000882331F0CE0101960E946758892B79F6EA
:10B0B000CE0101960E94ED14F301628073806CCF83
:10B0C0008091110781508093110780E0CACFDF92F1
:10B0D000EF92FF920F931F93CF93DF9300D000D096
:10B0E0001F921F92CDB7DEB77C0119821A821B8294
:10B0F0001C821D821E821F8218868A818F708A831D
:10B10000D701ED91FC916081718187E39AE00E9403
:10B11000638567E67AE087E39AE00E94C985C70104
:10B120000E94B71481111BC06EE57AE087E39AE0B4
:10B130000E94C98587E39AE00E94DA830FEF1FEF30
:10B14000C80128960FB6F894DEBF0FBECDBFDF91C1
:10B15000CF911F910F91FF90EF90DF900895C7015D
:10B160000E94E11CD82EF70181859285009791F00D
:10B17000DC01ED91FC91008CF18DE02D19958C0195
:10B1800097FD08C081E00115110509F480E00E94D7
:10B19000F119D6CFF7018085873009F42EC0EFEF83
:10B1A000ED0DE43150F5F0E08827E652F74A8F4F75
:10B1B0000C94CBD2EE58F758FD58FD58F758EE587E
:10B1C000FD58FD58FD58FD58FD58FD58FD58EE58E6
:10B1D000FD58FD58FD58FD58EE58EE586FE37AE0E3
:10B1E00087E39AE00E94C98501E010E0A9CF80E0E2
:10B1F0000E94F11910E000E0A3CF40E052E0B70157
:10B20000CE0101960E94C633D70118968C911897EB
:10B21000873071F160F4833009F454C0843061F0F8
:10B220006FE47AE087E39AE00E94C985E3CF883033
:10B2300009F448C08930A1F7CE0101960E94B19768
:10B240008C0164E47AE087E39AE00E94C985B80142
:10B2500087E39AE00E94D19B87E39AE00E94DA8319
:10B2600091E080E0012B09F490E0092F182F68CFBE
:10B270001296ED91FC9180858F7010E000E0853092
:10B2800001F76CE57AE087E39AE00E94C98520E047
:10B2900050E040E070E060E0F701828193810E941D
:10B2A000A057F82E082F10E069E57AE087E39AE0CE
:10B2B0000E94C9858F2D0E94F11987E39AE00E94B0
:10B2C000DA833ECFCE0101960E94D5348B01B9CFEF
:10B2D0002F923F924F925F926F927F928F929F92A6
:10B2E000AF92BF92CF92DF92EF92FF920F931F9394
:10B2F000CF93DF93CDB7DEB760970FB6F894DEBF7C
:10B300000FBECDBF6130710509F494C0DC01129607
:10B310006D917C916115710509F48CC04C01198205
:10B320001A821B821C821D821E821F8218868A81BD
:10B330008F708A8340E052E0CE0101960E94C633AE
:10B34000CE0101960E94B1971C01F4018281938184
:10B350000E94501C2B013C01D40117962D913D9168
:10B360004D915C911A97D1010E948CD22FEF30E061
:10B3700040E050E00E9440D229873A874B875C87A3
:10B380000E94ECA49B01AC0189859A85AB85BC85A4
:10B390000097A105B10509F468C0A12CB12C650185
:10B3A0007C018D01C301B2010E94D8298987411413
:10B3B000510461047104F1F1D40117968D919D91AE
:10B3C0000D90BC91A02D8D879E87AF87B88B0E9472
:10B3D000ECA49B01AC018D859E85AF85B889009753
:10B3E000A105B10561F0A12CB12C65017C018D0195
:10B3F000C301B2010E94D829882309F451C0D401A5
:10B4000012966D907C9080E00E940E19AB01BC01F9
:10B41000C3010E943D1F232869F0F40184810E942A
:10B42000EC12D40116969C91891304C061E0C4010A
:10B430000E94EE1C90E080E060960FB6F894DEBFAC
:10B440000FBECDBFDF91CF911F910F91FF90EF9075
:10B45000DF90CF90BF90AF909F908F907F906F9034
:10B460005F904F903F902F90089591E099879FCFE4
:10B47000B985BB23F1F060E0C4010E94EE1CF40129
:10B48000828193810E946758892BA1F640E050E0A9
:10B49000BA01D40112968D919C910E943D1FCACF92
:10B4A000F40184810E94EC12D40116969C918913B8
:10B4B000DFCF232809F4BECFF40184810E94EC126F
:10B4C000D40116969C918913B5CFB985B111B2CF2D
:10B4D000ADCFCF93DF93EC0169E377E187E39AE0A7
:10B4E0000E94C9856C817D8187E39AE00E94D19B8F
:10B4F00063E377E187E39AE00E94C98587E39AE0F6
:10B500000E94DA8361E08C810E9448A36E818C8165
:10B510000E941AA38A819B81009729F040E050E0A5
:10B52000BA010E943D1FE881F9810684F785E02D6C
:10B5300062E0CE0119958A819B810E946758181696
:10B5400019065CF40A80DB81C02D80E00E940E1990
:10B55000AB01BC01CE010E943D1F81E090E0DF9174
:10B56000CF9108952F923F924F925F926F927F9268
:10B570008F929F92AF92BF92CF92DF92EF92FF9203
:10B580000F931F93CF93DF93CDB7DEB7C955D10982
:10B590000FB6F894DEBF0FBECDBF0E94ECA49B0196
:10B5A000AC0160913B0670913C0680913D06909104
:10B5B0003E06A12CB12C650110E3E12E15E7F12E1A
:10B5C00000E010E00E94D829882309F426C2E09107
:10B5D0001707F0911807309709F41FC280911107DF
:10B5E0008F5F809311072680378010E0211431048B
:10B5F00009F438C1F10180858F708530F9F460E07D
:10B60000C1010E94A297FC0181859285A385B48522
:10B610000597A105B10591F4B101CE0101960E94F3
:10B620009520CE0101960E94B71466968FAF66975B
:10B63000811108C0CE0101960E94ED14F101228013
:10B640003380D4CF25961CAE1DAE1EAE1FAE2597FF
:10B6500029961CAE1DAE1EAE1FAE299740E052E0EB
:10B66000BE016F5F7F4FCE018F5B9F4F0E94C6333D
:10B67000CE0101960E94501C6B017C0169966FAF50
:10B6800069976A96DFAE6A97CE0101960E943E9C4A
:10B690004C01CE018F5B9F4F0E94021465966CAFE8
:10B6A0007DAF8EAF9FAF6597CE0101960E94E11CE2
:10B6B000182FB601DD0C880B990B0E94FDD020E0FD
:10B6C00030E048EC52E40E9456D32B013C01CE01FD
:10B6D00001960E94675868969FAF8EAF689766E79D
:10B6E00076E187E39AE00E94C98522E065964CAD39
:10B6F0005DAD6EAD7FAD659787E39AE00E94F783FD
:10B7000060E776E187E39AE00E94C98522E0B30111
:10B71000A20187E39AE00E94F7836AE676E187E375
:10B720009AE00E94C985612F70E087E39AE00E9449
:10B73000D19BE114F10409F48EC088E00E940E1937
:10B740009B01AC0144275527B70190E080E0AA2473
:10B75000AA94BA2CC12CD12C17E2E12E19E0F12EBB
:10B7600000E010E00E94D829882371F1F101608186
:10B77000718180E999E00E9463856AE576E180E95C
:10B7800099E00E94C985F1016081718182EE94E0A7
:10B790000E94BAA890E080E0BC0169964FAD69971D
:10B7A0006A965FAD6A97CE0101960E943D1F62E0E6
:10B7B00070E0C4010E949C19CE0101960E94ED1414
:10B7C00066961FAD66973ACF20E030E048E152E43C
:10B7D000C301B2010E94FED318163CF4F10160814E
:10B7E00071818EEE94E00E94BAA868968EAD9FADEE
:10B7F0006897892B19F461E070E0DBCF20E030E03E
:10B8000040E85FE365966CAD7DAD8EAD9FAD65970D
:10B810000E94E9D29B01AC01C301B2010E94F6D0A3
:10B8200070E060E087FDC5CFA301920165966CAD25
:10B830007DAD8EAD9FAD65970E94F6D01816DCF6F3
:10B840006BE476E187E39AE00E94C98587E39AE09A
:10B850000E94DA83B1CF61E476E187E39AE00E9447
:10B86000C985AACF809111078150809311070E944A
:10B87000ECA460933B0670933C0680933D06909346
:10B880003E060E94A32B2B013C010E94ECA46B01FD
:10B890007C010E944897882309F489C08091CA08D6
:10B8A000811185C030E020E041E050E060E4CE014D
:10B8B00001960E943A2A4FE350E065ED7CE1CE010B
:10B8C00001960E941ACB65EF73E0CE0101960E94AB
:10B8D00016D74FE350E068E176E1CE0101960E9471
:10B8E0001ACB2AE0AE014F5B5F4FC301B2010E9449
:10B8F000A5CBBE016F5B7F4FCE0101960E94BAA51A
:10B9000030E020E041E050E060E4CE0101960E948A
:10B910003A2A4FE350E065ED7CE1CE0101960E94AA
:10B920001ACB65EF73E0CE0101960E9416D74FE364
:10B9300050E061E176E1CE0101960E941ACBC70189
:10B94000B60128EE33E040E050E00E9440D2CA0148
:10B95000B9012AE0AE014F5B5F4F0E94A5CBBE014B
:10B960006F5B7F4FCE0101960E94BAA530E020E0C8
:10B9700041E050E060E4CE0101960E943A2A4FE394
:10B9800050E065E07DE1CE0101960E941ACB4FE0C8
:10B9900050E06FEF7CE1CE018F5B9F4F0E9438CB70
:10B9A000BE016F5B7F4FCE0101960E94BAA51123A5
:10B9B00009F44DC06BE376E187E39AE00E94C98504
:10B9C0000E94A32BAB01BC0187E39AE00E94C79BB6
:10B9D00063E376E187E39AE00E94C98560911107ED
:10B9E000062E000C770B87E39AE00E94D19B61E260
:10B9F00076E187E39AE00E94C9854091370650912D
:10BA000038066091390670913A0687E39AE00E9401
:10BA1000C79B87E39AE00E94DA83C75ADF4F0FB6CD
:10BA2000F894DEBF0FBECDBFDF91CF911F910F9174
:10BA3000FF90EF90DF90CF90BF90AF909F908F904E
:10BA40007F906F905F904F903F902F90089561E3AB
:10BA500076E187E39AE00E94C9850E94A32BAB019F
:10BA6000BC0187E39AE00E94C79B69E276E1B2CF0E
:10BA70002F923F924F925F926F927F928F929F92FE
:10BA8000AF92BF92CF92DF92EF92FF920F931F93EC
:10BA9000CF93DF93CDB7DEB7C556D1090FB6F89473
:10BAA000DEBF0FBECDBFDC0114962D913C91232B40
:10BAB00009F43DC73B014C01FC0182819B012250EE
:10BAC00031092230310508F0F8C5803409F4F7C295
:10BAD00008F04AC0843008F085C28091FB058F5F72
:10BAE0008093FB05A3016FEFC4010E942A53D40188
:10BAF00012960C9112970695017013961C9113974C
:10BB00008AEC810F803108F043C06BEF74E08D91B7
:10BB10009C910E942A977C010097D1F1FC018085BD
:10BB20008F708530A9F58091760A181324C0809112
:10BB3000770A803401F58091780A9091790A5C0146
:10BB4000990FCC08DD0860E0C7010E94A297FC01B4
:10BB500081859285A385B485A816B906CA06DB0639
:10BB60000CF065C0512C3EC0823409F4A8C208F420
:10BB700039C28058AFCF1093760A80E48093770A59
:10BB8000812F0E9484A39093790A8093780AD7CF5B
:10BB9000212F30E0F901ED50F14E8491F901E35588
:10BBA000F14E1491F901E959F14EF490FF2009F496
:10BBB0003BC081110E94B3A2EF2DF0E0EE0FFF1FFA
:10BBC000ED53F94FA591B491EC911E2331E020E0A3
:10BBD00009F430E0832F922F552453940817190647
:10BBE00009F0C0CFF3E06F16710409F488C0D401E6
:10BBF0001496ED91FC91E181EF70E150EC3008F08A
:10BC00007EC0F0E08827E85FF14A8F4F0C94CBD2DA
:10BC1000295EA55F5F5E955EA55FAE5EA55FE25E95
:10BC20000F5F285F6A5F8C5F90E080E0D5CF61E0B6
:10BC3000C7010E94A29755245394FC0181859285E7
:10BC4000A385B4858A159B05AC05BD050CF0CACF4C
:10BC500089CF0E94ECA49B01AC0144275527D40155
:10BC60001496ED91FC916281738190E080E0AA24AA
:10BC7000AA94BA2CC12CD12C18EEE12E13E0F12E8F
:10BC800000E010E00E94D8298823C9F1F401008166
:10BC900011816DEB74E0C8010E942A97892B41F451
:10BCA00062EC74E0C8010E942A97892B09F40EC146
:10BCB00042E050E063E0C4010E942A5320C00E9489
:10BCC000ECA49B01AC0144275527D4011496ED91B7
:10BCD000FC916281738190E080E0AA24AA94BA2C3E
:10BCE000C12CD12C1CE2E12EFF24F39400E010E0E3
:10BCF0000E94D82942E050E064E0811184C0D40160
:10BD00001496ED91FC91808183FB992790F995150C
:10BD100009F4D2C1982F907E09F439C1982F907EF2
:10BD200090528F71892B808358C10E94ECA49B0193
:10BD3000AC0144275527D4011496ED91FC91628102
:10BD4000738190E080E0AA24AA94BA2CC12CD12C53
:10BD500016E9E12EF12C00E010E0CACF0E94ECA41D
:10BD60009B01AC0144275527D4011496ED91FC9119
:10BD70006281738190E080E0AA24AA94BA2CC12C3D
:10BD8000D12C18EEE12E13E0F12E00E010E00E941D
:10BD9000D829882309F4B3CFF4010081118168EC1C
:10BDA00074E0C8010E942A97892B41F46EEC74E07C
:10BDB000C8010E942A97892B09F488C042E050E00C
:10BDC00068E079CF0E94ECA49B01AC014427552781
:10BDD000D4011496ED91FC916281738190E080E032
:10BDE000AA24AA94BA2CC12CD12C1CE2E12EFF2447
:10BDF000F39400E010E00E94D82942E050E069E0AE
:10BE0000882309F47CCFC4010E942A530E94ECA429
:10BE1000D4011496ED91FC917383628370CF0E94DC
:10BE2000ECA49B01AC0144275527D4011496ED9155
:10BE3000FC916281738190E080E0AA24AA94BA2CDC
:10BE4000C12CD12C16E9E12EF12C00E010E0D3CF6B
:10BE50000E94ECA49B01AC0144275527D401149601
:10BE6000ED91FC916281738190E080E0AA24AA9414
:10BE7000BA2CC12CD12C18EEE12E13E0F12E00E0EB
:10BE800010E00E94D829882309F439CFF4010081F9
:10BE9000118165ED74E0C8010E942A97892B39F45D
:10BEA0006BED74E0C8010E942A97892B21F042E0D3
:10BEB00050E06BE000CF67EB74E0C8010E942A9766
:10BEC00042E050E066E0892B09F4F5CE42E050E014
:10BED0006DE0F1CE0E94ECA49B01AC0144275527F4
:10BEE000D4011496ED91FC916281738190E080E021
:10BEF000AA24AA94BA2CC12CD12C1CE2E12EFF2436
:10BF0000F39400E010E00E94D829882309F4F7CECA
:10BF100042E050E06CE077CF0E94ECA49B01AC01C2
:10BF200044275527D4011496ED91FC9162817381C9
:10BF300090E080E0AA24AA94BA2CC12CD12C16E956
:10BF4000E12EF12C00E010E0DECF0E94ECA49B017A
:10BF5000AC0144275527D4011496ED91FC916281E0
:10BF6000738190E080E0AA24AA94BA2CC12CD12C31
:10BF700018E5E12E12E0F12E00E010E00E94D82931
:10BF8000882309F4BCCE42E050E060E094CE0E94E9
:10BF9000ECA4D4011496ED91FC9115977383628300
:10BFA000E181EF70552009F445C0E230F1F050F422
:10BFB000EE23E9F1D4011496ED91FC91808150FAC1
:10BFC00083F9B1CEE53089F0A3016AE0E73091F75B
:10BFD000C4010E942A538111EDCF8091FB0581504D
:10BFE0008093FB0590E080E0A4C4F40100811181FE
:10BFF00061EB74E0C8010E942A97892BA9F468ECD0
:10C0000074E0C8010E942A97892B71F46EEC74E0E9
:10C01000C8010E942A97892B39F469E974E0C801A4
:10C020000E942A97892B19F0A30166E0D1CFA301C2
:10C0300061E0CECFE150ED3008F0BCCFF0E08827D2
:10C04000EB5DFF498F4F0C94CBD23260DA5F3560E5
:10C050003560DA5F3860DA5F59605960596059605D
:10C0600059603560A30162E0B3CFA30165E0B0CFB2
:10C070000D911C9161EB74E0C8010E942A97892BF5
:10C08000A9F468EC74E0C8010E942A97892B71F426
:10C090006EEC74E0C8010E942A97892B39F469E993
:10C0A00074E0C8010E942A97892B19F0A30167E068
:10C0B0008FCFA30160E08CCF8F71806434CEB3E06A
:10C0C0006B16710409F48ECF6BEF74E0F40180817C
:10C0D00091810E942A978C01D40113968C919091A2
:10C0E000760A8913CEC09091770A903409F0C9C0BE
:10C0F0008091780A9091790A3C010115110509F4A3
:10C10000F0C0F80120852F70253009F0EAC0C80181
:10C110000E942E9CA4968FAFA497843008F4BDC0D3
:10C1200063E0C8010E94A297DC0119968D919C9151
:10C130006AE0D62ED89EF001D99EF00D1124A39668
:10C14000FFAFEEAFA39762E0C8010E94A297DC01A7
:10C1500019968D919C91D89E7001D99EF00C112456
:10C1600057010F2C000CCC08DD0861E0C8010E94CB
:10C17000A297A6969FAF8EAFA69760E0C8010E94D7
:10C18000A297FC0121843284438454849301072CB8
:10C19000000C440B550B2219330944095509A39689
:10C1A000AEADBFADA397BD01BB0F880B990B6A194C
:10C1B0007B098C099D090E9430D2A696EEADFFAD99
:10C1C000A697218532854385548522193309440970
:10C1D00055090E9462D2A20EB31EC41ED51EA4969B
:10C1E000FFADA497F53009F46BC081E090E0A39611
:10C1F000EEADFFADA3971F01FF0F440855082A14A9
:10C200003B044C045D040CF464C015012601970145
:10C210000F2C000C440B550B221633064406550612
:10C220000CF45CC0A2019101A496FFADA497F2307A
:10C2300009F06BC06301770CEE08FF0860E0C801ED
:10C240000E94A297FC0181859285A385B485C816BA
:10C25000D906EA06FB060CF486C361E0C8010E9419
:10C26000A297FC0181859285A385B4858C159D05D7
:10C27000AE05BF050CF0B6CE81E090E0A0E0B0E0E6
:10C2800075C38093760A90E49093770A0E9484A302
:10C290009093790A8093780A2FCF8AE0869D500187
:10C2A000879DB00C11240B2C000CCC08DD08F12C60
:10C2B000E12C20E038E2A3963FAF2EAFA39795CFB5
:10C2C00064E0C8010E94A297DC0119968D919C91AF
:10C2D0008ECF66246A9453E0752E99CF712C612C11
:10C2E000A3CF2AE0289F5001299FB00C112495016B
:10C2F000BB0C440B550BF12CE12C80E098E2A3968B
:10C300009FAF8EAFA39781E090E0D4011496ED919A
:10C31000FC9162817381D301A61BB70BB7FF03C0E9
:10C32000B195A195B1098A179B070CF4C1C0808112
:10C33000982F929596959770963008F0BCC09F5FA5
:10C340009295990F907E8F71892BB4C0F70161850A
:10C350007285DB018C91811196C3A114B10409F49B
:10C3600073C0D50118968C9118978F70843009F09E
:10C370006BC019966D917C91CE0101960E94EC3AAA
:10C38000CE0101960E94B714882309F459C06114A4
:10C39000710409F460C0E114F10431F0F701808503
:10C3A0008F70843009F442C025961CAE1DAE1EAEBF
:10C3B0001FAE259729961CAE1DAE1EAE1FAE299747
:10C3C00023961FAD23971F7023961FAF239781E0FD
:10C3D00022968FAF2297A12CCC24C394F12CE12C70
:10C3E00001E024962FAD249725963FAD259740E098
:10C3F00027965FAD279728966FAD289729967FAD32
:10C400002997CE0101960E9475401AC001151105A9
:10C4100029F0F80180858F70843019F062E075E0B2
:10C4200032C361857285FB01808195CF61857285FC
:10C43000FB018081882321F0CE0101960E94F39CAC
:10C44000CE0101960E94ED14D4011496ED91FC9159
:10C4500073826282C7CD0115110531F0D80118969B
:10C460008C918F708430F1F025961CAE1DAE1EAEFF
:10C470001FAE259729961CAE1DAE1EAE1FAE299786
:10C4800023961FAD23971F7023961FAF239782E03B
:10C4900022968FAF2297A12CCC24C394F12CE12CAF
:10C4A00002E09FCFF80161857285DB018C91C2CFDC
:10C4B00080818F7180838081803AB8F0C701FF0C42
:10C4C000AA0BBB0B82179307A407B50771F0A396BD
:10C4D000EEADFFADA397CF01FF0FAA0BBB0B8217E9
:10C4E0009307A407B50709F07DCD6615770509F414
:10C4F00079CD6D961CAE1DAE1EAE1FAE6D976B96C0
:10C500008FAD6B978F7080666B968FAF6B976D96C4
:10C510008CAD9DADAEADBFAD6D9765968CAF9DAF4B
:10C52000AEAFBFAF6597AAE0B0E00E9481D2699636
:10C530006CAF7DAF8EAF9FAF699762EB76E087E31C
:10C540009AE00E94C985D40113966C9187E39AE022
:10C550000E94CA9B60EB76E087E39AE00E94C9855F
:10C56000CE018F5A9F4F0E94323267E774E0F40188
:10C57000808191810E942A97B12CA12CD12CC12CB1
:10C580006296EFAC62976396FFAC639764960FADCB
:10C59000649765961FAD659766962FAD669767960B
:10C5A0003FAD679768964FAD689769965FAD69979D
:10C5B0006FEF0E94A44ED4010D911C916BE774E0C3
:10C5C000C8010E942A977C0160E874E0C8010E94BB
:10C5D0002A978C010097E1F1FC0180858F708430EF
:10C5E000B9F56185728540E450E0CE0101960E9464
:10C5F0005AD76FE270E0CE0101960E9421D7892BB5
:10C6000059F4D80119962D913C9143E050E060E433
:10C61000CE0101960E943A2A00E020E032E040E19B
:10C6200050E0BE016F5B7F4FCE018F5A9F4F0E943B
:10C6300011300E944897882359F08091CA088111CF
:10C6400007C0BE016F5B7F4FCE0101960E94BAA565
:10C65000E114F10409F4F8CEF70180858F7084307D
:10C6600009F0F2CE61857285CE0101960E94EC3A06
:10C67000CE0101960E94B714882309F4E1CEA12CC3
:10C68000CC24C394F12CE12C62960FAD6297639693
:10C690001FAD639764962FAD649765963FAD659720
:10C6A00066964FAD669767965FAD679768966FAD74
:10C6B000689769967FAD6997A4CE883009F444C025
:10C6C000803109F08FCC0E94ECA42B013C01C40105
:10C6D0000E942215A12CB12C650110E3E12E15E773
:10C6E000F12E00E010E0A30192010E94D8298823D6
:10C6F00009F478CC60E874E0D4018D919C910E949B
:10C700002A978C01009709F407C1FC0180858F707E
:10C71000843009F001C10E94ECA42AE0AE014F5F11
:10C720005F4F0E94A5CB0E944897882309F4F4C06C
:10C730008091CA088111F0C0BE016F5F7F4FD801A0
:10C7400019968D919C91E6C00E94ECA42B013C01AE
:10C75000C4010E942215A12CB12C650118E9E12E1B
:10C760001AE3F12E00E010E0A30192010E94D82903
:10C77000882309F437CCD4011496ED91FC911597D8
:10C78000818113961C91811153C01630F0F58CE015
:10C79000EEE1F2E0DE01119601900D928A95E1F74B
:10C7A000E12FF0E0EE0FFF1F21E030E02C0F3D1FE6
:10C7B000E20FF31F60E080810E9448A362E775E109
:10C7C00083E01330C9F070F46AE775E181E011305D
:10C7D00099F066E775E182E0123071F06EE775E17D
:10C7E00080E00AC06EE675E184E0143029F06AE664
:10C7F00075E185E0153091F70E94D99BD40114961C
:10C80000ED91FC9181E08183EDCB61E377E087E3FB
:10C810009AE00E94C985F401638187E39AE00E944F
:10C82000CA9B64E077E087E39AE00E94C985DACB8F
:10C8300024E0129FF0011124E450FA4FC080D1800F
:10C84000E280F38060E077E087E39AE00E94C985A8
:10C85000D40113966C9187E39AE00E94CA9B6CEE18
:10C8600076E087E39AE00E94C9852AE030E0B701CC
:10C87000A60187E39AE00E94DD8460E874E0F40199
:10C88000808191810E942A978C01009709F44CC005
:10C89000DC0118968C9118978F70843009F044C091
:10C8A00019966D917C9140E450E0CE0101960E9472
:10C8B0005AD76FE270E0CE0101960E9421D7892BF2
:10C8C00051F4F8012185328543E050E060E4CE0167
:10C8D00001960E943A2AFF92EF92DF92CF928DE169
:10C8E00094E09F938F938E010F5B1F4F1F930F93C5
:10C8F0000E94B1D70E9448970FB6F894DEBF0FBED2
:10C90000CDBF882349F08091CA08811105C0B801C4
:10C91000CE0101960E94BAA80E94ECA4AB01BC0112
:10C92000C4010E94FB145ECB6DED76E07CCF8FEFEF
:10C930009FEFCB59DF4F0FB6F894DEBF0FBECDBFD0
:10C94000DF91CF911F910F91FF90EF90DF90CF90EB
:10C95000BF90AF909F908F907F906F905F904F901F
:10C960003F902F90089580E090E0DC01F401248155
:10C970003581F90142815381052E000C660B770B3E
:10C9800084179507A607B70709F42CCB3C01D401FF
:10C990000D911C916BE774E0C8010E942A975C011D
:10C9A00060E874E0C8010E942A976C01A114B104E8
:10C9B00019F4892B09F448CD6CEA74E0C8010E948F
:10C9C0002A977C0167EA74E0C8010E942A978C01CB
:10C9D00068EB76E087E39AE00E94C985F401638101
:10C9E00087E39AE00E94CA9B66EB76E087E39AE0D1
:10C9F0000E94C985B30187E39AE00E94D19B87E337
:10CA00009AE00E94DA83C114D10409F4A6CCD601BD
:10CA100018968C9118978F70843009F09ECC1996D7
:10CA20006D917C9140E450E0CE0101960E945AD76E
:10CA30000E944897882309F490CC8091CA088111FC
:10CA40008CCC6FE270E0CE0101960E9421D7892B39
:10CA500051F4F6012185328543E050E060E4CE01D7
:10CA600001960E943A2A6114710409F4CFCCE114B2
:10CA7000F10439F0D70118968C918F70843009F445
:10CA800065CC6FEF74E0CE0101960E94BAA565CC2B
:10CA9000EF92FF920F931F93CF93DF93EC018B01E3
:10CAA0001D821C821A821B82E880F980E114F10445
:10CAB00009F470C08091450690914606892B09F4CF
:10CAC00069C0672B09F48701F80180858F70863073
:10CAD000A9F466E075E0C8010E942A97009719F052
:10CAE000FC0181858A8363EF75E0C8010E942A9763
:10CAF000009709F456C0FC0181858B8368E075E0DE
:10CB0000C7010E942A97009709F041C06BEA76E0BE
:10CB100087E39AE00E94C9856B8187E39AE00E94CF
:10CB2000CA9B69EA76E087E39AE00E94C9856A8138
:10CB300087E39AE00E94CA9B87E39AE00E94DA8327
:10CB4000E880F9800E94FF8C8C01892BC1F082E083
:10CB5000F801808711861286138614868081918160
:10CB6000009711F00E947F8A88E095E00E94AE8ACB
:10CB7000F80191838083B801C7010E94A99B68E0F6
:10CB800075E0888199810E942A97009719F009968B
:10CB90009D838C83DF91CF911F910F91FF90EF9038
:10CBA0000895F801808191810E9495CAA6CF8F9245
:10CBB0009F92AF92BF92CF92DF92EF92FF920F932C
:10CBC0001F93CF93DF9300D000D0CDB7DEB7209175
:10CBD000130730911407232B09F484C02091120706
:10CBE000211180C04C01809112078F5F8093120742
:10CBF000809111078F5F809311070E94ECA49B0125
:10CC0000AC016091330670913406809135069091A5
:10CC10003606A12CB12C65011BE0E12EF12C00E0C1
:10CC200010E00E94D829882309F452C0E09113072C
:10CC3000F09114070681178101151105B9F1F8016A
:10CC400080858F70863071F567E774E0C8010E94B7
:10CC50002A970097D1F0FC0120852F702530A9F488
:10CC6000E680F780E114F104E9F0FA82E982B80184
:10CC7000CE0101960E944865B401CE0101960E9442
:10CC8000385DF701E280F380EDCF1A83098370E00D
:10CC900060E0CE0101960E944865B401CE01019684
:10CCA0000E94385DF80102811381C6CFF3E08F1630
:10CCB000910451F00E94ECA4609333067093340603
:10CCC00080933506909336061092760A1092770A72
:10CCD0008091110781508093110780911207815034
:10CCE0008093120726960FB6F894DEBF0FBECDBF15
:10CCF000DF91CF911F910F91FF90EF90DF90CF9038
:10CD0000BF90AF909F908F900895A89582E090E09B
:10CD10000C94D7658091CA088F5F8093CA08A89544
:10CD200083E090E00E94D7650E94398A8091CA080A
:10CD300081508093CA080895CF92DF92EF92FF92BC
:10CD4000CF93DF93EC018C85883068F40E94B09219
:10CD50000E94ECA46B017C018C850E94CC92811115
:10CD600009C088E08C87DF91CF91FF90EF90DF9032
:10CD7000CF9008950E948A6661E070E080E090E0C4
:10CD80000E94B9A40E94ECA4AB01BC014C195D093E
:10CD90006E097F098D859E85B0E0A0E04817590790
:10CDA0006A077B07C8F28C850E94BE92DACFCF92C9
:10CDB000DF92EF92FF921F93CF93DF93EC017B0101
:10CDC0006A018C85883048F40E94CC92882319F03F
:10CDD0008C850E94B09288E08C87F70182819381D4
:10CDE000A481B5810097A105B10551F490E080E0E0
:10CDF000DF91CF911F91FF90EF90DF90CF9008953A
:10CE00008F3F9F4FAF4FBF4F89F370E060E081E2EB
:10CE10000E940793182F8C87883040F780E591E0B7
:10CE20000E941EA0A7014E5F5F4F24E030E06CE03F
:10CE300070E0812F0E947821B601812F0E94DB9241
:10CE400064E070E0812F0E94E88D0E94ECA46B01E9
:10CE50007C018C850E94CC92873121F18C3111F1BB
:10CE6000882321F20E94ECA4AB01BC014C195D099E
:10CE70006E097F098D859E85B0E0A0E08417950737
:10CE8000A607B70748F00E948A6661E070E080E07C
:10CE900090E00E94B9A4DDCF8C850E94BE9288E00C
:10CEA0008C87A4CF81E090E0A3CF4F925F926F92E6
:10CEB0007F92AF92BF92CF92DF92EF92FF920F9349
:10CEC0001F93CF93DF93CDB7DEB76D970FB6F8946E
:10CED000DEBF0FBECDBF2091450630914606FF2430
:10CEE000F394232B09F412C1811149C0FF24F39458
:10CEF0006BE77CE087E39AE00E94C98587E39AE0CC
:10CF00000E94DA83809132068F5F80933206E0912F
:10CF10001707F0911807309709F48BC00681178125
:10CF20000115110509F48FC0D80118968C918F70E6
:10CF3000853009F5C8010E942E9C8823E1F0F80194
:10CF400060817181CE0101960E94EC3ACE0101967A
:10CF50000E94B714882359F08A859B85009739F081
:10CF6000DC01ED91FC910284F385E02D1995CE0151
:10CF700001960E94ED14F80102811381D1CF64EB78
:10CF80007CE087E39AE00E94C98587E39AE00E94EB
:10CF9000DA830E94ECA42B013C01809111078823C5
:10CFA00071F10E94ECA49B01AC01A12CB12C650194
:10CFB00010E1E12E17E2F12E00E010E0C301B20112
:10CFC0000E94D82981111BC00E94398A80911B07B9
:10CFD000811126C08091150790911607059741F0A1
:10CFE0008091170790911807892B11F00E94D45651
:10CFF0000E94B25A82E090E00E94D765CECF809125
:10D000001107882309F472CF61E97CE080E999E097
:10D010000E94C98580E999E00E94DA83F12C68CFEB
:10D020008091190790911A07892BA1F20E94FD5057
:10D03000D1CF6BE67CE087E39AE00E94C98587E365
:10D040009AE00E94DA831092400610923F0663E64F
:10D050007CE087E39AE00E94C98587E39AE00E941A
:10D06000DA8364E670E080E090E00E94B9A4109258
:10D07000A106109210076BE47CE087E39AE00E941F
:10D08000C9850E94A32BAB01BC0187E39AE00E94F3
:10D09000C79B8091450690914606009711F00E942B
:10D0A000BD9F1092460610924506109214071092EA
:10D0B000130710921807109217071092A3061092E8
:10D0C000A20610920E0710920D0710920C071092F4
:10D0D0000B0710921A071092190766E47CE087E3A9
:10D0E0009AE00E94C9850E94A32BAB01BC0187E393
:10D0F0009AE00E94C79B87E39AE00E94DA8310922D
:10D100000F07809132068150809332068F2D6D96E5
:10D110000FB6F894DEBF0FBECDBFDF91CF911F9148
:10D120000F91FF90EF90DF90CF90BF90AF907F90E6
:10D130006F905F904F9008958F929F92BF92CF9281
:10D14000DF92EF92FF920F931F93CF93DF93CDB7B0
:10D15000DEB7A5970FB6F894DEBF0FBECDBF8091A6
:10D16000450690914606892B09F48FC480911107DA
:10D1700081118BC4809111078F5F809311076BE041
:10D1800072E186E899E00E94C98586E899E00E94EC
:10D19000DA8300914506109146066BE075E0C80100
:10D1A0000E942A97909318078093170761E175E012
:10D1B000C8010E942A979093A3068093A20666E373
:10D1C00075E0C8010E942A97909314078093130773
:10D1D00068E175E0C8010E942A9790930E0780933A
:10D1E0000D070E946A2E6DE175E0809145069091D1
:10D1F00046060E942A9790931A0780931907892B55
:10D20000A1F080911B07811110C08091A40690911C
:10D21000A506892B09F47CC081E080931B076BEF86
:10D2200071E186E899E00E94C9851092400610924B
:10D230003F06E0911707F0911807309709F406C3ED
:10D24000E680F78000911707109118070115110566
:10D2500009F4F5C2E114F10409F4F1C2F701808583
:10D260008F70853099F7C7010E942E9C823070F331
:10D27000B701CE0101960E949520CE0101960E9431
:10D28000B7148823E1F18A859B85009709F450C281
:10D29000DC01ED91FC910484F585E02D1995892B35
:10D2A00049F08A859B85DC01ED91FC910284F38530
:10D2B000E02D19958A859B85DC01ED91FC91068016
:10D2C000F781E02D1995892BD1F0CE0101960E94AE
:10D2D000E11C882341F040E051E060E070E0CE01C5
:10D2E00001960E94EA3C8D819E81892B41F040E0AD
:10D2F00052E060E070E0CE0101960E94EA3CD70166
:10D300001296ED90FC90CE0101960E94ED149ACFFA
:10D3100062EC71E187E39AE00E94C98587E39AE0B5
:10D320000E94DA836CEB71E187E39AE00E94C98581
:10D330000E94A32BAB01BC0187E39AE00E94C79B2C
:10D3400087E39AE00E94DA838FE090E00E94C8C8E9
:10D350008C0188E1D80111968C93119712961C923A
:10D3600012971C921E961C921E921D970E94E99F76
:10D370001093A5060093A406012B69F46DEA71E1F0
:10D3800080E999E00E94C98580E999E00E94DA83EA
:10D3900010921B074ACF0E94E99F8091A4069091AA
:10D3A000A5060E945B19882309F48EC065E971E126
:10D3B00086E899E00E94ED858091A4069091A506EB
:10D3C0000E94F725E091A406F091A50681E08083F4
:10D3D00065E771E187E39AE00E94ED858091A406FC
:10D3E0009091A5060E94052669E671E1811102C0AF
:10D3F00065E571E187E39AE00E94ED858091190768
:10D4000090911A07892B21F28091490690914A0642
:10D41000892B09F0DFC083E190E00E94C8C88C012D
:10D420008091A4069091A50625EA38E7F801328B91
:10D43000218B968385831482108289E0818381E029
:10D440008283838310934A06009349060E94ECA4CA
:10D450006B017C01F0E1CF0EF7E2DF1EE11CF11C55
:10D46000D8011596ED91FC9116978FEF838714865E
:10D4700013821482158216821782108611861286F4
:10D4800014961C92BB24B394BE01625E7F4FF801D8
:10D49000858196810E94DF2618160CF096C00E94A6
:10D4A000ECA46C157D058E059F0508F08EC0DE018D
:10D4B0005E9698E080E0915019F1ED91E827F0E058
:10D4C000E352F74E8491F7CF0E942C288091A40656
:10D4D0009091A5060E945B19882359F068E371E1D9
:10D4E00086E899E00E94C98586E899E00E94DA837F
:10D4F00085CF6CE171E180E999E00E94ED8548CF2C
:10D500009DA19813C1CFD8018C91811138C0159677
:10D510008D919C910E940526BE01625E7F4FF801AD
:10D52000858196810E94D82540E064EBD80115964C
:10D530008D919C910E94B225F80185809680C4014E
:10D540000E943E25C4010E94321267E887EF98E0EE
:10D550000E94BD1260E887EF98E00E94BD120E9411
:10D56000B6A4C4010E943E25982ED80115968D912F
:10D570009C910E94052695FC02C0F801B082AE0184
:10D580004F5F5F4FBE01625E7F4FC8010E9446261B
:10D59000D80111969C908E8D803109F488C2BE010D
:10D5A000625E7F4FC8010E94B526891508F0B4C09D
:10D5B000F8018181D80111968C93119714968C9162
:10D5C00014978F5F14968C935FCFE0914906F0918A
:10D5D0004A061282E0911907F0911A07E680F78057
:10D5E0009FE7D92E8091190790911A07892B09F48A
:10D5F00013CEE114F10409F40FCEBE01625E7F4F39
:10D60000F701808191810E944113882309F404CE9F
:10D6100065E071E187E39AE00E94C985D7016D91C9
:10D620007C9187E39AE00E94638587E39AE00E94F9
:10D63000DA830091490610914A06AE014F5F5F4FB1
:10D64000BE01625E7F4FC8010E949B26882309F4B9
:10D650005EC08E8D803109F45AC0DD82F80185816B
:10D6600096810E940526BE01625E7F4FD801159605
:10D670008D919C910E94D82540E06EE4F80185814F
:10D6800096810E94B22540E06B81D80115968D915C
:10D690009C910E94B22540E06C81F80185819681C1
:10D6A0000E94B2258E8D803141F040E06D81D8011D
:10D6B00015968D919C910E94B225F80185819681E5
:10D6C0000E940526BE01625E7F4FD80115968D919E
:10D6D0009C910E94D825F801408168E4858196815B
:10D6E0000E94B22564E170E080E090E00E94B9A45D
:10D6F000D8018C91882331F06AE070E080E090E0FE
:10D700000E94B9A4F801858196810E940526D7015F
:10D710001296ED90FC9066CF8E8D803111F48CE0E6
:10D7200049CFBE01625E7F4FC8010E94B52642CF3D
:10D73000CE0101960E943E9C8C01912C812C97FF7A
:10D7400006C011950195110988248394912CCE016E
:10D7500001960E94E11CC82ED12C8985853091F05C
:10D76000863009F0CCCDB02E61E0802F0E9448A316
:10D7700061E0892809F441C0CA94CD2809F041C06C
:10D7800060E03FC0CD2829F462E0CE0101960E94FE
:10D79000B21C40E051E060E070E0CE0101960E94D2
:10D7A000EA3C8D819E81892B41F040E052E060E0AF
:10D7B00070E0CE0101960E94EA3C61E0802F0E9459
:10D7C00048A360E0802F0E941AA363EF71E187E312
:10D7D0009AE00E94C985B80187E39AE00E94D19B34
:10D7E0006EEE71E187E39AE00E94C9856CEE71E10B
:10D7F00087E39AE00E94C98582CDCA94CD2809F0BA
:10D80000BFCFC62ED12C8B2D0E941AA367EE71E1DB
:10D8100087E39AE00E94C985B80187E39AE00E94F5
:10D82000D19B65EE71E187E39AE00E94C985B6015C
:10D8300087E39AE00E94D19B63EE71E1D9CFF801B2
:10D84000868197819093400680933F0687E39AE014
:10D850000E94DA83E0911307F0911407309709F4DE
:10D860008AC0809111078F5F80931107068117810D
:10D870000115110509F47AC0D80118968C918F70A2
:10D88000863009F069C01F8F0E8F70E060E0CE0116
:10D890004E960E9448658AA19BA1892B09F45CC021
:10D8A0008091450690914606892B09F455C0EE8C6F
:10D8B000FF8CF70180858F70863099F567E774E0FB
:10D8C000C7010E942A970097F1F0DC0118962C916D
:10D8D00018972F702530B9F41696CD90DC90C114AE
:10D8E000D104F9F0DA82C982B701CE0101960E9413
:10D8F0004865ED81FE811082118212821382F60149
:10D90000C280D380ECCFFA82E98270E060E0CE0181
:10D9100001960E94486562E070E0CE0101960E9487
:10D92000385DEAA1FBA1108211821282138288A1C4
:10D93000843068F462E0823008F060E089A10E94DF
:10D9400048A3EAA1FBA18181807F818305C0803447
:10D9500041F060E0823431F0D80112960D911C91B3
:10D9600087CF62E089A10E9448A3F6CF809111077A
:10D9700081508093110768EF70E186E899E00E947A
:10D98000C98560EF70E186E899E00E94C98581E071
:10D990002091170730911807232B09F480E00E948B
:10D9A000DB1967EE70E186E899E00E94C98581E0A5
:10D9B0002091130730911407232B09F480E00E9473
:10D9C000DB1960EE70E186E899E00E94C98581E08C
:10D9D00020910D0730910E07232B09F480E00E945F
:10D9E000DB1967ED70E186E899E00E94C98581E066
:10D9F0002091190730911A07232B09F480E00E9427
:10DA0000DB196EEC70E186E899E00E94C98580918F
:10DA1000A1060E94DB1986E899E00E94DA8369EC8E
:10DA200070E186E899E00E94C9850E94A32BAB01B2
:10DA3000BC0186E899E00E94C79B86E899E00E94B5
:10DA4000DA8381E08093100783E599E00E946118F2
:10DA5000882351F083E599E00E949C6684E090E081
:10DA600090931607809315078091150790911607DC
:10DA7000079731F484E090E09093160780931507A0
:10DA800080911107815080931107A5960FB6F894E5
:10DA9000DEBF0FBECDBFDF91CF911F910F91FF90E1
:10DAA000EF90DF90CF90BF909F908F900895BCE053
:10DAB000B91508F47DCD33CEAF92BF92DF92EF92CD
:10DAC000FF920F931F93CF93DF9300D000D0CDB779
:10DAD000DEB78C017B01D42EFB0184819581892BDB
:10DAE000F9F0A080B1806FE370E0C5010E9421D7FA
:10DAF0000097B1F09C012A193B0937FD11C050E095
:10DB000040E0B701CE0101960E949A81BE016F5F8D
:10DB10007F4FC7010E945080CE0101960E944A812A
:10DB200060E275E0C7010E94CB7F882321F1F801F4
:10DB3000128A118A80E090E19587848784E890E0DA
:10DB4000948B838B81E0868780E090E2908B87873F
:10DB5000D58A81E090E026960FB6F894DEBF0FBE1E
:10DB6000CDBFDF91CF911F910F91FF90EF90DF908C
:10DB7000BF90AF9008956DE275E0C7010E94CB7F22
:10DB8000882369F0F801128A118A148A138A84E8BA
:10DB900090E095878487168680E090E3D7CF90E069
:10DBA00080E0D9CFEF92FF920F931F93CF93DF9333
:10DBB00000D01F92CDB7DEB78C017B01FB018485BD
:10DBC0008830A8F08BED93E0F80191838083128276
:10DBD000138214821582C8010F900F900F900F903E
:10DBE000DF91CF911F910F91FF90EF90089580E505
:10DBF00091E00E941EA024E030E0AE014F5F5F4F35
:10DC00006CE070E0F70184850E94A722BE016F5F7F
:10DC10007F4FC8010E940986DECFCF93DF93CDB737
:10DC2000DEB72E970FB6F894DEBF0FBECDBF809142
:10DC300011078F5F8093110761EF76E186E899E025
:10DC40000E94C98586E899E00E94DA8310928209D1
:10DC50001092810980E090E190937D0980937C0986
:10DC600084E890E0909384098093830981E0809315
:10DC70007E0980E090E29093800980937F0982E79B
:10DC80008093850980E799E00E9465218B37910593
:10DC900009F0BEC063EE76E187E39AE00E94C98591
:10DCA00087E39AE00E94DA831C821B8281EA92E079
:10DCB0009A83898380E799E09E838D838FEF9FEF1E
:10DCC00098878F8380E00E945567CE0101960E945D
:10DCD00000A0909346068093450680E799E00E9455
:10DCE000FB198091450690914606892B01F567ED59
:10DCF00076E180E999E00E94C98580E999E00E9477
:10DD0000DA8366E875E0CE0109960E948981CE012A
:10DD100009960E9473ADCE0109960E944A818091B6
:10DD2000110781508093110790E080E019C064ECE6
:10DD300076E186E899E00E94C98586E899E00E942C
:10DD4000DA83809111078150809311070E949C68AB
:10DD50008091620990916309892B59F481E090E0E8
:10DD60002E960FB6F894DEBF0FBECDBFDF91CF91D8
:10DD700008950E948C98882389F382E70E947798FF
:10DD80008091620990916309DC01ED91FC9100881A
:10DD9000F189E02D60E670E019956091620970915B
:10DDA000630940E0CE0109960E946683BE01675F69
:10DDB0007F4F84E699E00E945080CE0109960E9430
:10DDC0004A818091620990916309DC01ED91FC9197
:10DDD0000488F589E02D199566EA76E187E39AE0F3
:10DDE0000E94C98564E679E0CE0109960E9480818F
:10DDF000BE01675F7F4F87E39AE00E94BB8587E3A0
:10DE00009AE00E94DA83CE0109960E944A81A6CF49
:10DE100080E799E00E949415892BA1F080E799E0B2
:10DE20000E94BE1566E875E0CE0101960E948981C8
:10DE3000CE0101960E9473ADCE0101960E944A81E7
:10DE40000E94E2AD80E799E00E94FB1963EB76E166
:10DE500086E899E00E94C98586E899E00E94DA8305
:10DE60005ECFEF92FF920F931F93CF93DF9300D07B
:10DE700000D0CDB7DEB78091620990916309892BFC
:10DE800009F46CC087E70E947798809162099091AD
:10DE90006309DC01ED91FC910088F189E02D70E0CF
:10DEA00060E0199510E000E08091620990916309AB
:10DEB000DC01ED91FC9111971C962D913C9102177C
:10DEC000130740F40190F081E02D60E019950F5F99
:10DED0001F4FEACF0088F189E02D70E060E01995CE
:10DEE00008EE12E08CEEE82E82E0F82E80916209B6
:10DEF00090916309F80161918F01DC01ED91FC9132
:10DF00000190F081E02D1995E016F10679F78091E6
:10DF1000620990916309DC01ED91FC910488F58917
:10DF2000E02D199566E875E0CE0101960E94898181
:10DF3000CE0101960E9473ADCE0101960E944A81E6
:10DF400087E090E00E94939B87E090E00E949D9B79
:10DF50006CE672E186E899E00E94C9851092820918
:10DF60001092810980E090E190937D0980937C0973
:10DF700084E890E0909384098093830981E0809302
:10DF80007E0980E090E29093800980937F0982E788
:10DF90008093850980E799E00E94BE1580E799E0AB
:10DFA0000E94FB1988EC90E026960FB6F894DEBF2D
:10DFB0000FBECDBFDF91CF911F910F91FF90EF90DA
:10DFC0000895FF920F931F93CF93DF9300D000D05B
:10DFD000CDB7DEB78C01BC01CE0101960E948081D5
:10DFE000BE016F5F7F4F87E39AE00E94BB8587E3A6
:10DFF0009AE00E94DA83CE0101960E944A816EE186
:10E0000073E1CE0101960E945281BE016F5F7F4F86
:10E01000C8010E94B07FF82ECE0101960E944A816D
:10E02000FF2069F0B801CE0101960E948081CE01E7
:10E0300001960E9473ADCE0101960E944A812696F8
:10E040000FB6F894DEBF0FBECDBFDF91CF911F9109
:10E050000F91FF9008954F925F926F927F928F92EF
:10E060009F92AF92BF92CF92DF92EF92FF920F9367
:10E070001F93CF93DF93CDB7DEB7C859D1090FB641
:10E08000F894DEBF0FBECDBF8E010F5B1F4FD801CE
:10E090001D921C92FE01ED5BFF4F8EE1DF011D9290
:10E0A0008A95E9F78091620990916309892B09F4B7
:10E0B000CEC10E948C98882309F4C9C182E70E94CE
:10E0C00077988091620990916309DC01ED91FC9150
:10E0D0000088F189E02D60E270E019954FE150E091
:10E0E000B80180916209909163090E94D1987C01E6
:10E0F0008091620990916309DC01ED91FC910488A3
:10E10000F589E02D1995E114F10409F4A0C1F80195
:10E11000EE0DFF1D108280916F091F928F938091E9
:10E120006E091F928F9380916D091F928F9380913A
:10E130006C091F928F9380916B091F928F9380912E
:10E140006A091F928F9389E395E09F938F931F92A3
:10E1500080E48F93FE0131966F01FF93EF930E944D
:10E1600074D761E074E186E899E00E94C985B8013E
:10E1700086E899E00E946385B60186E899E00E94EE
:10E18000638586E899E00E94DA837E01F1E6EF0E6E
:10E19000F11CD70113961C921E92129788EE93E001
:10E1A000A0E0B0E0F70184839583A683B78388E07D
:10E1B000848788EE93E09687858789E593E091834D
:10E1C0008083108A1786128B018B148A138A80E54C
:10E1D00090E0968B858B118E65E273E187E39AE080
:10E1E0000E94C98564E679E0CE0185589F4F0E9460
:10E1F0008081BE0165587F4F87E39AE00E94BB850E
:10E2000087E39AE00E94DA83CE0185589F4F0E94EF
:10E210004A8168E675E0CE0183579F4F0E9489814D
:10E2200068E675E0CE0185589F4F0E948981BE0146
:10E2300065587F4FCE018B579F4F0E94808164E6C7
:10E2400079E0CE018B579F4F0E94E680BE01635755
:10E250007F4F0E94E680BC01CE018D569F4F0E94E9
:10E260008081CE018B579F4F0E944A81CE018558F5
:10E270009F4F0E944A81CE0183579F4F0E944A813F
:10E280008AE695E0CB57DF4F99838883C558D04005
:10E29000C757DF4F19821882C958D040C557DF4F82
:10E2A00019821882CB58D040CD56DF4F8881998192
:10E2B000C359D040C957DF4F99838883C758D0408E
:10E2C0006BEF73E187E39AE00E94C9850E94A32B5C
:10E2D000AB01BC0187E39AE00E94C79B87E39AE009
:10E2E0000E94DA8364E670E080E090E00E94B9A4C6
:10E2F00081EE9FE6D70150969C938E931F9762EB19
:10E300007CE782E39DE80E940BCC8C010FB6F89469
:10E31000DEBF0FBECDBF892B09F4F4C083E090E0CF
:10E320000E94C8C8D8011D969C938E931C97FC012F
:10E33000F182E0821282C7010E946118882319F0DD
:10E34000C7010E949C66D70153966D917C915497AA
:10E350005596AD90BC906115710509F48FC0CE0142
:10E3600085589F4F0E940986A501BE0165587F4FC1
:10E37000C7010E94D766181619060CF0C0C0D70155
:10E380005196BC9051975296AC90DF92CF9280E814
:10E3900093E19F938F931F930F930E9492CCDF92F0
:10E3A000CF928BE793E19F938F931F930F930E94DC
:10E3B00092CCD8011C96ED91FC9181E08283DF9292
:10E3C000CF9288E793E19F938F931F930F930E94BF
:10E3D00092CCD8011C96ED91FC911282AF92BF9223
:10E3E00082E493E19F938F931F930F930E9492CCAB
:10E3F0000FB6F894DEBF0FBECDBFB12C89E3C82E97
:10E4000083E1D82E8B2D94E08902F0011124A5E838
:10E41000B0E0AC0FBD1FEA0FFB1F80819181009718
:10E42000A9F12281338121153105C9F33F932F933F
:10E430009F938F93DF92CF921F930F930E9492CC62
:10E44000B3940FB6F894DEBF0FBECDBFDBCF40E272
:10E4500050E063E374E1C8010E9438CB65E174E1E8
:10E4600086E899E00E94C985B80186E899E00E9493
:10E47000638586E899E00E94DA834DCEF7016189D1
:10E480007289A501C7010E94831875CF8DE793E1BA
:10E490009F938F931F930F930E9492CCD70158960E
:10E4A0001C921E925797D8011C96ED91FC91C0804A
:10E4B000D1800F900F900F900F9033E3A32EB12CCB
:10E4C000D601ED91FC910084F185E02DC6011995EE
:10E4D00041975CF4B1E0AB1AB10839F064E170E047
:10E4E00080E090E00E94B9A4EBCFD601ED91FC91C1
:10E4F0000084F185E02DC6011995419734F4C801D7
:10E500000E940B8D10E000E05AC066E875E0CE0175
:10E5100083579F4F0E948981912CA12CD601ED91A8
:10E52000FC910688F789E02DC60119958823E1F151
:10E53000BDE0AB1201C0A92CD601ED91FC9106887B
:10E54000F789E02DC60119958111D4C0D601ED914E
:10E55000FC910084F185E02DC6011995892B09F401
:10E56000DBC0D601ED91FC910284F385E02DC6015C
:10E570001995B82EBAE08B1709F4D0C0EDE08E17CC
:10E5800009F4CCC0FFEF8F1709F4C6C0682FCE0185
:10E5900083579F4F0E943C809A2CAB2CBFCFBAE090
:10E5A000BB12FACFAB12F8CFCC24C394D12CCE013E
:10E5B00083579F4F0E944A81CD2809F4A3CFD701EA
:10E5C0005796ED90FC906DEE73E187E39AE00E9420
:10E5D000C985B70187E39AE00E94D19B87E39AE05F
:10E5E0000E94DA8364E670E080E090E00E94B9A4C3
:10E5F0000115110509F451C1B8ECEB16F10409F04D
:10E600002AC161EE73E186E899E00E94C98564EF52
:10E6100071E080E090E00E94B9A4EF961FAE1EAEBC
:10E62000EF97C158DF4F19821882CF57D0408FEF34
:10E630009FEFCF57DF4F99838883C158D0408BE835
:10E6400092E0ED969FAF8EAFED97CD57DF4F1983D8
:10E650000883C358D040F89481E00E945567CE01EA
:10E6600085589F4F0E9400A09093460680934506D0
:10E670007894C8010E940B8D8091450690914606C2
:10E68000892B09F0D6C066E875E0CE0183579F4F0D
:10E690000E948981CE0183579F4F0E9473ADCE01A6
:10E6A00083579F4F0E944A816AEC73E180E999E0A9
:10E6B0000E94C985F12CE12CCE018D569F4F0E94FE
:10E6C0004A81C701C856DF4F0FB6F894DEBF0FBEB0
:10E6D000CDBFDF91CF911F910F91FF90EF90DF9011
:10E6E000CF90BF90AF909F908F907F906F905F90F2
:10E6F0004F900895D601ED91FC910084F185E02DB5
:10E70000C6011995892B09F021CF64E670E080E0FD
:10E7100090E00E94B9A410CFBB24BA9468E775E0DA
:10E720008AE999E00E946385BE0163577F4F8AE9B9
:10E7300099E00E94BB858AE999E00E94DA8360E350
:10E7400073E1CE0185589F4F0E945281BE016558EA
:10E750007F4FCE0183579F4F0E94B07F982ECE01EE
:10E7600085589F4F0E944A81992099F1CF56DF4FDB
:10E7700028813981C159D04049E050E0BE0163573A
:10E780007F4FCE0185589F4F0E949A81ED968EADA6
:10E790009FADED97412C512C3201009719F00E944A
:10E7A000B3CA2B014201CE0185589F4F0E944A8176
:10E7B0004114510429F0D70158965C924E92579714
:10E7C000B4018AE999E00E94D19B8AE999E00E940C
:10E7D000DA83F7018784908881149104D1F0CF56B1
:10E7E000DF4F88819981C159D040892B91F0BE01BA
:10E7F00063577F4FCE0185589F4F0E948081CE0185
:10E8000085589F4FF4011995CE0185589F4F0E945E
:10E810004A8166E875E0CE0183579F4F0E941A81B6
:10E82000FFEFBF12BCCEC8010E940B8DD12CC12CB2
:10E83000BECE0E949C6880911007882329F00E9418
:10E84000EB9A67FF0E94ED1B63EC73E186E899E0A9
:10E850000E94C98531CFE0E3EE16E1E0FE0651F4F7
:10E860006FEA73E186E899E00E94C985C8010E94B9
:10E870000B8D22CF67E973E180E999E00E94C98599
:10E88000C8010E940B8DB70180E999E00E94D19BDD
:10E8900080E999E00E94DA830FCF64E873E187E3AF
:10E8A0009AE00E94C985EE24EA94FE2C05CF0F93CE
:10E8B0001F93CF93DF93EB0102970CF485C00A817D
:10E8C0001B8167E173E1C8010E94E3CA892B51F4FF
:10E8D00081E00E94899B88EC90E0DF91CF911F91AD
:10E8E0000F91089563E173E1C8010E94E3CA892B87
:10E8F00011F480E0EECF63EF72E186E899E00E94C8
:10E90000C9850E94EB9A63FB662760F981E068275E
:10E9100070E086E899E00E94D19B86E899E00E9429
:10E92000DA838091620990916309892BE9F10A8168
:10E930001B810E948C988823B9F1F8010190002076
:10E94000E9F73197E01BF10BB09770F582E70E9471
:10E9500077988091620990916309DC01ED91FC91B7
:10E960000088F189E02D60E270E01995B80180918E
:10E970006209909163090E94638580916209909178
:10E980006309DC01ED91FC910190F081E02D60E0E4
:10E9900019958091620990916309DC01ED91FC91D8
:10E9A0000488F589E02D19956A817B8186E899E0D4
:10E9B0000E9463856CEE72E186E899E00E94C98549
:10E9C00086E899E00E94DA838091150790911607F6
:10E9D00002977CF10E942B70883C910539F424E069
:10E9E00030E0309316072093150777CF8F3F9807B5
:10E9F000C9F461ED72E187E39AE00E94C98587E37B
:10EA00009AE00E94DA8310920F0783E090E09093DF
:10EA100016078093150783E599E00E949C6689ECB0
:10EA200090E05BCF209110072111D9CF2FE030E08B
:10EA3000D8CF64EC72E180E999E00E94C98580E951
:10EA400099E00E94DA8384EF91E047CF5F926F9262
:10EA50007F928F929F92AF92BF92CF92DF92EF926E
:10EA6000FF920F931F93CF93DF93CDB7DEB7CF56AF
:10EA7000D1090FB6F894DEBF0FBECDBF4C018B019C
:10EA8000F42E642F87E39AE00E94CA9B66E67DE03D
:10EA900087E39AE00E94C985B801CE0101965C0126
:10EAA0000E948081B50187E39AE00E94BB8587E3DD
:10EAB0009AE00E94DA83C5010E944A8192E0F9122D
:10EAC0006BC264E67DE0C5010E945281B501C801B8
:10EAD0000E94E07FF82EC5010E944A81FF2009F4C0
:10EAE000D0C220E04DE251E0B40181E399E00E9400
:10EAF0009A89E0900B07F0900C076DE57DE0CE0160
:10EB000086599F4F0E94528166E57DE0CE018C5967
:10EB10009F4F0E945281CE01885A9F4F0E94F62338
:10EB20006E961FAD6E976D960FAD6D976C96DFACC0
:10EB30006C976B96CFAC6B9766E875E0CE018196CB
:10EB40000E948981BE016F5D7F4FC5010E94808157
:10EB50006C2DC5010E949B806BE775E00E94CC8004
:10EB60006D2D0E949B806BE775E00E94CC80602F2A
:10EB70000E949B806BE775E00E94CC80612F0E9411
:10EB80009B80BC01CE01825A9F4F0E948081C501AB
:10EB90000E944A81CE0181960E944A8161E57DE012
:10EBA000CE018E5A9F4F0E94528166E875E0CE01D9
:10EBB000845B9F4F0E94898102E619E0D801189674
:10EBC0006C9170E084E0759567958A95E1F7C501D1
:10EBD0000E944B984D815E8169817A81CE01845B70
:10EBE0009F4F0E941080C5010E944A81F8016085F4
:10EBF0006F7070E0C5010E944B984D815E81698104
:10EC00007A81CE01845B9F4F0E941080C5010E94D3
:10EC10004A810F5F1F4FF9E008361F0779F66BE452
:10EC20007DE0CE018A5B9F4F0E9452816AE27DE0C7
:10EC3000CE0181960E945281BE016F5D7F4FCE0151
:10EC4000CE960E948081BE016A5B7F4FCE01CE9638
:10EC50000E94E680BE01645B7F4F0E94E680BE0199
:10EC60006E5A7F4F0E94E680BE01625A7F4F0E941B
:10EC7000E680BE016C597F4F0E94E6808C014AE01D
:10EC8000B50180E590E00E947DCBF5010190002068
:10EC9000E9F73197AF014A195B09B501C8010E9434
:10ECA0001080811103C0C8010E948980BE0166598D
:10ECB0007F4FC8010E94E680B7010E94CC80BC0152
:10ECC000C4010E94BB85C4010E94DA83CE01CE96A6
:10ECD0000E944A81CE0181960E944A81CE018A5BC0
:10ECE0009F4F0E944A81CE01845B9F4F0E944A81C0
:10ECF000CE018E5A9F4F0E944A81CE01825A9F4F69
:10ED00000E944A81CE018C599F4F0E944A81CE01B8
:10ED100086599F4F0E944A81C4010E94DA8364E6AB
:10ED200070E080E090E00E94B9A4D401ED91FC91E4
:10ED30000488F589E02DC401199501E010E088C030
:10ED400028966EAD7FAD2897CE0181960E94F39CE8
:10ED5000892B09F450C122961CAE1DAE1EAE1FAE0B
:10ED6000229726961CAE1DAE1EAE1FAE26978FAD07
:10ED70008F708FAF40E053E0BE016F5D7F4FCE01DB
:10ED8000CE960E94C63300E020E033E040E250E03F
:10ED9000B501CE01CE960E941130BC01C6010E9481
:10EDA000248108EC10E129C1EE2009F4F3C046E00B
:10EDB00050E070E060E0C8010E944D7FD8016D9185
:10EDC0007C91CE0181960E94EC3ACE0181960E9400
:10EDD000B71400E911E08823B9F189A5873061F4FF
:10EDE000CE0181960E94675861E0892B09F462E0A8
:10EDF000CE0181960E94B21C22961CAE1DAE1EAEA4
:10EE00001FAE229726961CAE1DAE1EAE1FAE2697D5
:10EE10008FAD8F708FAF40E053E0BE016F5D7F4FCD
:10EE2000CE01CE960E94C63300E020E033E040E2FF
:10EE300050E0B501CE01CE960E941130BC01C60152
:10EE40000E94248108EC10E1CE0181960E94ED140D
:10EE5000C801C159DF4F0FB6F894DEBF0FBECDBF5A
:10EE6000DF91CF911F910F91FF90EF90DF90CF90A6
:10EE7000BF90AF909F908F907F906F905F9008951C
:10EE8000F801608171810E942A977C01892B09F029
:10EE900040C104E911E0DCCFEE2009F47BC049E079
:10EEA00050E070E060E0C8010E944D7F4AE0B4018C
:10EEB000C5010E94668341E050E061E574E0C8014D
:10EEC0000E9410804D815E8169817A81C8010E9413
:10EED000108066E07DE087E39AE00E94C985B80172
:10EEE000CE0181960E948081BE016F5D7F4F87E3D6
:10EEF0009AE00E94BB8587E39AE00E94DA83CE0104
:10EF000081960E944A816EEF7CE0CE0181960E943C
:10EF10005281F801848195812DA13EA1821793072A
:10EF2000E1F4892BA1F1E080F18069A07AA0D701FA
:10EF30008D917D01882359F1082E000C990B0E94B8
:10EF4000B1D66C01F30181913F01082E000C990BA1
:10EF50000E94B1D6C816D90651F3CE0181960E94FF
:10EF60004A81552041F021E048EC50E0B40181E3B2
:10EF700099E00E949A89D8018D919C910E94C8893C
:10EF8000009711F484E991E08C01C5013DC055243E
:10EF90005394E3CF01E97ECFB1E0FB1270C063E28E
:10EFA0007DE0C5010E945281B501C8010E94B07F79
:10EFB000582EC5010E944A81552049F1EE2051F397
:10EFC00046E050E070E060E0C8010E944D7F4AE0FA
:10EFD000B401CE018A5B9F4F0E946683F801608175
:10EFE0007181CE0181960E94EC3ACE0181960E94F9
:10EFF000B7148111A5CE00E911E0CE0181960E94DF
:10F00000ED14CE018A5B9F4F0E944A8121CF6CE0B4
:10F010007DE0C5010E945281B501C8010E94B07F08
:10F02000F82EC5010E944A81F11036CF61EF7CE0D5
:10F03000C5010E945281B501C8010E94B07F182FFE
:10F04000C5010E944A8100E0112309F401CF80E04C
:10F050000E94899B69EC7CE086E899E00E94C98562
:10F0600086E899E00E94DA8366E875E0C5010E94AF
:10F070008981C5010E9473ADC5010E944A8100E0EB
:10F080005DCE6CE17DE0C5010E945281B501C801F1
:10F090000E94B07FF82EC5010E944A81F11084CEF3
:10F0A00066E17DE0C5010E945281B501C8010E9460
:10F0B000B07FF82EC5010E944A81FF2001F3EE20A7
:10F0C00009F468CF45E050E070E060E0C8010E94BC
:10F0D0004D7F6BE775E0C8010E94CB7F882339F034
:10F0E000E0901707F0901807E114F10491F466E836
:10F0F00075E0C8010E94CB7F811107C0809117077E
:10F1000090911807009709F0BBCEE0904506F0906B
:10F11000460620E048EC50E2B40181E399E00E9409
:10F120009A89C4010E94DA831C821B8281EA92E0E0
:10F130009A8389839E828D828FEF9FEF98878F833A
:10F14000B701C5010E94F18AEACD0895FC0124812E
:10F1500035816217730748F480819181009729F007
:10F16000860F971FFC018081089580E0089508951F
:10F170000895AF92BF92CF92DF92EF92FF920F93DA
:10F180001F93CF93DF936C017B018B01040F151F3D
:10F19000EB015E01AE18BF08C017D10759F06991A5
:10F1A000D601ED91FC910190F081E02DC6011995F9
:10F1B000892B79F7C501DF91CF911F910F91FF90B6
:10F1C000EF90DF90CF90BF90AF900895FC01538DEA
:10F1D000448D252F30E0842F90E0821B930B541731
:10F1E00010F0CF96089501970895FC01918D828DBE
:10F1F000981761F0A28DAE0FBF2FB11D5D968C9157
:10F20000928D9F5F9F73928F90E008958FEF9FEF95
:10F210000895FC01918D828D981731F0828DE80F51
:10F22000F11D858D90E008958FEF9FEF0895FC010B
:10F23000918D228D892F90E0805C9F4F821B9109D8
:10F240008F73992708958AE999E00E94177921E040
:10F25000892B09F420E0822F0895FC01A48DA80FCA
:10F26000B92FB11DA35ABF4F2C91848D90E0019608
:10F270008F739927848FA689B7892C93A089B18928
:10F280008C91837080648C93938D848D981306C0C9
:10F290000288F389E02D80818F7D80830895EF922D
:10F2A000FF920F931F93CF93DF93EC0181E0888F40
:10F2B0009B8D8C8D98131AC0E889F989808185FF10
:10F2C00015C09FB7F894EE89FF896083E889F989B2
:10F2D00080818370806480839FBF81E090E0DF91B4
:10F2E000CF911F910F91FF90EF900895F62E0B8D07
:10F2F00010E00F5F1F4F0F731127E02E8C8D8E11C2
:10F300000CC00FB607FCFACFE889F989808185FF28
:10F31000F5CFCE010E942D79F1CFEB8DEC0FFD2FB3
:10F32000F11DE35AFF4FF0829FB7F8940B8FEA89E3
:10F33000FB8980818062CFCFCF93DF93EC01888DF2
:10F340008823B9F0AA89BB89E889F9898C9185FD60
:10F3500003C0808186FD0DC00FB607FCF7CF8C91EE
:10F3600085FFF2CF808185FFEDCFCE010E942D7900
:10F37000E9CFDF91CF91089580E090E0892B29F0CB
:10F380000E94237981110E94000080E090E0892B87
:10F3900049F080E090E0892B29F00E940000811163
:10F3A0000E94000080E090E0892B49F080E090E02E
:10F3B000892B29F00E94000081110E94000080E04A
:10F3C00090E0892B49F080E090E0892B29F00E94A1
:10F3D000000081110C94000008950F931F93FC010D
:10F3E00062857385848595850281138124813581A9
:10F3F000601B710B820B930B068517852089318961
:10F40000601B710B820B930B1F910F910895DC0110
:10F41000ED91FC910190F081E02D19948FEF9FEF19
:10F420000895FC0162897389848995890895EF9212
:10F430000F931F93CF93DF93FC01248D222341F080
:10F44000213051F1DF91CF911F910F91EF900895ED
:10F45000228933894489558986899789A08DB18D00
:10F46000821B930BA40BB50B892F9A2FAB2FBB27B5
:10F470008C010F5F1F4F6281738184819581CFB7AB
:10F48000F894DCB7E1E0ECBFEE24E394E2E0FEEFB9
:10F490001995DCBFCFBFD6CFF0E0E0E0DF91CF9190
:10F4A0001F910F91EF901994FC01138E128E411150
:10F4B0000CC082899389A489B589868B978BA08F8C
:10F4C000B18F148E81E090E0089590E080E008957F
:10F4D000CF92DF92EF92FF92CF93DF93DC01CB01CB
:10F4E000642FCFB7F8946D01EE24FF24CBBEDCB7B8
:10F4F00041E04CBFA901E1E0FEEF1995DCBFCFBFB1
:10F50000DF91CF91FF90EF90DF90CF900895CF9350
:10F51000DF93FC01248D211110C0EC01828D938DAD
:10F52000892B49F066897789808D918D30E020E0C4
:10F5300045E00E94687A1B8E1A8EDF91CF91089564
:10F540001F93CF93DF93FC01248D211145C0162F0B
:10F55000EC01828D938D892B49F466897789808DA2
:10F56000918D30E020E043E00E94687A4A8D5B8D07
:10F57000CA0181709927FE01E80FF91F158F892BA9
:10F5800069F02D8D3E8D6E897F89888D998D640FF0
:10F59000751F811D911D41E00E94687A8A8D9B8DA7
:10F5A00001969B8F8A8F81159140B1F46E897F8976
:10F5B000888D998D30E020E045E00E94687A1B8EAE
:10F5C0001A8E8E899F89A88DB98D9F5FAF4FBF4FCF
:10F5D0008E8B9F8BA88FB98F81E090E0DF91CF91C8
:10F5E0001F910895DC01ED91FC910280F381E02DE3
:10F5F00040E01994FB0144815581228133812150DF
:10F6000031094217530750F4A081B181A40FB51FEF
:10F610008C938481958101969583848380E00895FD
:10F62000CF93DF93EC01E881F9810284F385E02D2B
:10F63000CE0119950196B9F7DF91CF910895CF9238
:10F64000DF92EF92FF920F931F93CF93DF937C0192
:10F650006A018B01D0E0C0E0CC15DD0581F0D70157
:10F66000ED91FC910284F385E02DC70119958F3F40
:10F67000980729F0F80181938F012196EDCFCE01F3
:10F68000DF91CF911F910F91FF90EF90DF90CF907E
:10F690000895CF93C62FDC01ED91FC910088F1898C
:10F6A000E02D1995DC01ED91FC910190F081E02DA8
:10F6B0006C2FCF911994062E000C770BFC017783E9
:10F6C00066830895CF93DF93EC018E819F8101962D
:10F6D00011F5E881F9810088F189E02DCE011995B5
:10F6E000DC01ED91FC910084F185E02D1995892BC9
:10F6F000B1F0E881F9810284F385E02DCE011995FE
:10F700008132910534F3E881F9810684F785E02D93
:10F71000682FCE01199581E0DF91CF91089580E0A7
:10F72000FBCFFC0120812EBD9B012150310941F00E
:10F7300051810DB407FEFDCF4EB55EBD4193F5CFAF
:10F7400061507109860F971F0DB407FEFDCF2EB5CE
:10F75000FC0120830895E0911D07F0911E07808130
:10F7600090911C07892B80830895E0911D07F091EB
:10F770001E07908180911C078095892380830895BE
:10F780008EBD00000DB407FEFDCF8EB5089590E04C
:10F7900020916208233339F40C96982F990F990F12
:10F7A000990F80E008954896F8CFEF92FF920F935B
:10F7B0001F93CF93DF93EC018B017A010E94ECA49D
:10F7C000688B798B8A8B9B8B8C819D81DC01ED9181
:10F7D000FC910280F381E02DA701B801DF91CF9168
:10F7E0001F910F91FF90EF9019941F93CF93DF9388
:10F7F000EC01162F0E94ECA4688B798B8A8B9B8B73
:10F800008C819D81DC01ED91FC910190F081E02DD6
:10F81000612FDF91CF911F911994CF92DF92EF92D8
:10F82000FF92CF93DF93EC018E819F818F3F9807EA
:10F8300059F02FEF3FEF3F832E83DF91CF91FF9061
:10F84000EF90DF90CF9008950E94ECA46B017C01B3
:10F85000A4EFCA0EA1E0DA1EE11CF11CE881F981D7
:10F860000088F189E02DCE011995DC01ED91FC9124
:10F870000084F185E02D1995892B39F40E94ECA4C0
:10F880006C157D058E059F0548F3E881F981008898
:10F89000F189E02DCE011995DC01ED91FC910284F6
:10F8A000F385E02DDF91CF91FF90EF90DF90CF9027
:10F8B0001994FB0101900020E9F73197AF01461B35
:10F8C000570BDC01ED91FC910280F381E02D19943E
:10F8D0000E94ACD60F931F93CF93DF93D0E0C0E08C
:10F8E000009791F08C01C1E6D7E0688179816115BC
:10F8F000710529F0C8010E942CD7892B29F00B80B3
:10F90000DC81C02D209789F7CE01DF91CF911F9127
:10F910000F9108950F931F93CF93DF93EC0188818C
:10F920009981009759F02A813B812617370730F0DB
:10F9300081E0DF91CF911F910F9108958B016F5F4F
:10F940007F4F0E94CBD5009759F0998388831B8302
:10F950000A832C813D81232B59F7FC011082E8CFCB
:10F9600080E0E7CFEF92FF920F931F93CF93DF9347
:10F97000009751F4CFEFDFEFCE01DF91CF911F91D0
:10F980000F91FF90EF900895DC011C96ED90FC9094
:10F99000F70100811181D801ED91FC910688F7896A
:10F9A000E02DC8011995882329F3D801ED91FC9128
:10F9B0000084F185E02DC8011995D801ED91FC91E5
:10F9C000892B61F30284F385E02DC8011995EC01C0
:10F9D000019681F2F801818D882329F06C2F8AE944
:10F9E00099E00E94CA9BD70112968C91882321F23C
:10F9F000C532D10509F6D801ED91FC910084F1855D
:10FA0000E02DC801199502975CF0D801ED91FC91A9
:10FA10000688F789E02DC80119958111ECCFAACF8E
:10FA2000D1E0C0E0D801ED91FC910284F385E02D96
:10FA3000C80119958F3F980709F49CCF9C01215468
:10FA400031092A31310570F48D2F8295807F829F94
:10FA5000C00D1124D11104C00C2E000CDD0B8CCF75
:10FA6000D0E0E0CF9C01215631092A31310560F305
:10FA7000C0978A30910570F79D2F9295907F989F3F
:10FA8000C00D1124E7CFCF92DF92EF92FF920F9338
:10FA90001F93CF93DF936C018B0186E090E00E946F
:10FAA000C8C8EC019093A3078093A207F6010190C8
:10FAB0000020E9F7CF018C199D090E94C8C87C017C
:10FAC000B6010E9435D7F60101900020E9F7319781
:10FAD000EC19FD09EE0DFF1D1082F982E8821B83EF
:10FAE0000A838091A4079091A5079D838C83D0936E
:10FAF000A507C093A407DF91CF911F910F91FF90AD
:10FB0000EF90DF90CF900895FC01868197818F3F21
:10FB1000980729F02FEF3FEF3783268308958085DC
:10FB200091850C9456CC7F928F929F92AF92BF9208
:10FB3000CF92DF92EF92FF920F931F93CF93DF93B9
:10FB4000CDB7DEB7A6970FB6F894DEBF0FBECDBF18
:10FB50008C01762E942E852E20E2A22ECE010196C7
:10FB60007C01DC01EA2D1D92EA95E9F76801F3E4D6
:10FB7000CF0ED11C8BED93E09AA389A38FEF8BA3BB
:10FB80008CA38DA38EA343E450E0BE016F5D7F4F35
:10FB9000C6010E943923019609F4BFC081E0898320
:10FBA0008A8386E0B82EBB821C82D80114966D91A0
:10FBB0007D918D919C9117970E94D3D26D837E8306
:10FBC0008F83988789869A8680E890E09C878B87C8
:10FBD0004CE150E0B701C6010E94CE22FE013796EB
:10FBE0008AE1DF011D928A95E9F74801B8E08B0EA2
:10FBF000911CF401D70101900D92BA94E1F740E114
:10FC000050E0B701C6010E94CE22F7011192AA94DA
:10FC1000E9F796E0A92EB12C40E250E0B701C60109
:10FC20000E94CE22F1E0AF1AB108B1F783E68983D2
:10FC300092E89A8393E59B838C8385E38D8381E0AF
:10FC40008E837F829DE3988797E099878A8786E0F5
:10FC5000F401DE011B9601900D928A95E1F78CE08C
:10FC6000898B8A8B6DE775E0CE0143960E9435D76C
:10FC7000D8011B966C91CE0149960E945FA0F801B5
:10FC80006485CE014B960E945FA0D8011D966C91B1
:10FC9000CE014D960E945FA04EE150E0B701C60133
:10FCA0000E94CE22B3E07B121EC082E3898384E0EF
:10FCB0008A83F80196859B8397859C8390899D8391
:10FCC00091899E8396E39F838887828D8987838D20
:10FCD0008A87848D8B87858D8C874CE050E0B701B7
:10FCE000C6010E94CE2287E3898386E08A8391E061
:10FCF0009B8393E09C838D838FE08E838AE38F8345
:10FD00008BE388878FEF898749E050E0B701C60110
:10FD10000E94CE22C6010E940823A6960FB6F89430
:10FD2000DEBF0FBECDBFDF91CF911F910F91FF902E
:10FD3000EF90DF90CF90BF90AF909F908F907F908B
:10FD4000089590E080E00C94A621CF93DF93C4E166
:10FD5000D0E00E94A17E882361F061E070E080E045
:10FD600090E00E94B9A42197A1F780E0DF91CF91A4
:10FD7000089581E0FBCFFF920F931F93CF93DF9302
:10FD80001F921F92CDB7DEB7F82E22E030E0AE0111
:10FD90004F5F5F4F66E270E00E94A72209811A81DF
:10FDA00010270127102722E030E0AE014F5F5F4FA0
:10FDB00066E270E08F2D0E94A72289819A819827A0
:10FDC000892798270817190749F4C8010F900F9041
:10FDD000DF91CF911F910F91FF9008958C01E3CF98
:10FDE000AF92BF92CF92DF92EF92FF920F931F9349
:10FDF000CF93DF93DC01CD90DC901197C114D10437
:10FE000039F01496CD91DC918C017601209761F444
:10FE1000DF91CF911F910F91FF90EF90DF90CF90E6
:10FE2000BF90AF90089575015701BFEFAB1ABB0AA1
:10FE3000F7018081082E000C990B0E94DACA892BE9
:10FE400091F72197CC0DDD1D8881082E000C990BB0
:10FE50000E94DACA892B29F0CE15DF0510F0219710
:10FE6000F3CFAE014F5F5F4F4E195F09D801159672
:10FE70005C934E931497CE14DF0420F4B701C601AF
:10FE80000E94E8D6D801ED91FC91119714968D91BE
:10FE90009C91E80FF91F1082BBCFCF93DF93DC0159
:10FEA0001496ED91FC916E177F0728F541155105C9
:10FEB00011F19F01261B370B4217530708F49A01D3
:10FEC000DB01EC0188819981E21BF30BFD83EC835C
:10FED000AF01461B570B260F371FBC01620F731F64
:10FEE0008A0F9B1F0E945AD7E881F9818C819D81DE
:10FEF000E80FF91F1082DF91CF910895DF92EF9202
:10FF0000FF920F931F93CF93DF93FC01E480F58062
:10FF1000E114F10451F48FEF9FEFDF91CF911F9126
:10FF20000F91FF90EF90DF900895EC010190F08128
:10FF3000E02DEE0DFF1DD080108208811981062E64
:10FF4000000C770BC8010E9469D70E0D1F1DF80128
:10FF5000D082009701F328813981821B930BDDCF7A
:10FF6000FB0144815581FC0124813581241735072B
:10FF700078F080819181009759F0FB016081718157
:10FF80006115710529F00E944CD721E0892B09F0F9
:10FF900020E0822F0895FC0124813581232B39F440
:10FFA00021E0FB018081882349F020E007C08081A7
:10FFB00091810E942CD721E0892BB9F7822F0895D7
:10FFC000FC0124813581FB014481558124173507CB
:10FFD000E1F4FC0180819181FB01608171810097D6
:10FFE000D1F061157105A1F4232BC1F0FC018081D2
:10FFF00090E008C0232B91F0FB01808190E0919567
:020000021000EC
:100000008195910921E0892B09F020E0822F089544
:100010000E942CD7F7CF6115710561F721E0F6CF6B
:10002000EF92FF920F931F93CF93DF9361157105AA
:1000300041F480E0DF91CF911F910F91FF90EF90FD
:10004000089541155105B1F07B01EC010C811D8132
:10005000040F151FB8010E948A7C882351F3288160
:1000600039818C819D81B701820F931F0E9435D702
:100070001D830C8381E0DECFCF93DF931F921F920D
:10008000CDB7DEB769831A8241E050E0BE016F5FF1
:100090007F4F0E9410800F900F90DF91CF910895B5
:1000A0000F931F93CF93DF938C01EB01FC018081B1
:1000B00091810097E1F06881798161157105A9F05E
:1000C000428153812C813D814217530770F00E9479
:1000D00035D78C819D81F801958384831D821C8294
:1000E000DF91CF911F910F9108950E9464C988817B
:1000F0009981F801918380838A819B819383828394
:100100008C819D8195838483198218821B821A8237
:10011000E5CFCF93DF93EC0188819981009711F0AF
:100120000E9464C9198218821D821C821B821A8255
:10013000DF91CF910895EF92FF920F931F93CF938A
:10014000DF9300D01F92CDB7DEB77C01862F4AE047
:100150008E010F5F1F4FB80190E00E947DCBF80128
:1001600001900020E9F73197AF01401B510BB80116
:10017000C7010E941080811103C0C7010E948980BD
:10018000C7010F900F900F900F90DF91CF911F91AB
:100190000F91FF90EF900895CF93DF93EC016115DD
:1001A000710539F4CE010E948980CE01DF91CF9193
:1001B0000895FB0101900020E9F73197AF01461B3C
:1001C000570B0E941080882369F3EFCFCF93DF9302
:1001D000EC01FB0144815581608171810E94108096
:1001E000811103C0CE010E948980CE01DF91CF91A1
:1001F0000895EF92FF920F931F93CF93DF93EC013B
:100200007B018A01BA010E948A7C81110BC0CE0158
:100210000E948980CE01DF91CF911F910F91FF90B5
:10022000EF9008951D830C83B701888199810E9406
:1002300035D7F0CFFB0101900020E9F73197AF01EE
:10024000461B570B0C94F980CF93DF93EC0161159B
:10025000710531F00E941A81CE01DF91CF9108958E
:100260000E948980F9CFCF93DF93EC01FB018617C1
:10027000970749F0608171816115710541F04481F2
:1002800055810E94F980CE01DF91CF9108950E949F
:100290008980F9CFFC0180819181009711F00C9445
:1002A00064C90895EF92FF920F931F93CF93DF934A
:1002B000EC018B01198218821B821A821D821C821A
:1002C000CB010E9411CB7C01BC01CE010E948A7C33
:1002D000811109C0CE01DF91CF911F910F91FF9045
:1002E000EF900C948980FD82EC82B801888199811D
:1002F000DF91CF911F910F91FF90EF900C940ACB5B
:10030000FC011182108213821282158214820C94D5
:100310003381FC01118210821382128215821482B1
:10032000FB0101900020E9F73197AF01461B570B05
:100330000C94F980AF92BF92CF92DF92EF92FF922E
:100340000F931F93CF93DF935C016B017A018901B7
:100350002417350720F48F2D7901042F182F66E814
:1003600075E0C5010E948981D6011496CD91DC917A
:10037000EC16FD06C8F40C171D0708F4E801D601B9
:10038000ED91FC911197EC0FFD1F108110826D9182
:100390007C916E0D7F1DC5010E942481F601808134
:1003A0009181C80FD91F1883C501DF91CF911F918B
:1003B0000F91FF90EF90DF90CF90BF90AF90089596
:1003C0001F920F920FB60F9211240BB60F922F931C
:1003D0003F934F935F936F937F938F939F93AF93CD
:1003E000BF93EF93FF93E0911202F09113021995DE
:1003F000FF91EF91BF91AF919F918F917F916F91FD
:100400005F914F913F912F910F900BBE0F900FBEB8
:100410000F901F9018951F920F920FB60F921124F4
:100420000BB60F922F933F934F935F936F937F93EE
:100430008F939F93AF93BF93EF93FF93E09110023D
:10044000F09111021995FF91EF91BF91AF919F919A
:100450008F917F916F915F914F913F912F910F906D
:100460000BBE0F900FBE0F901F9018951F920F920A
:100470000FB60F9211240BB60F922F933F934F9309
:100480005F936F937F938F939F93AF93BF93EF93FC
:10049000FF93E0910602F09107021995FF91EF9109
:1004A000BF91AF919F918F917F916F915F914F918C
:1004B0003F912F910F900BBE0F900FBE0F901F908A
:1004C00018951F920F920FB60F9211240BB60F9230
:1004D0002F933F934F935F936F937F938F939F934C
:1004E000AF93BF93EF93FF93E0910402F091050265
:1004F0001995FF91EF91BF91AF919F918F917F914E
:100500006F915F914F913F912F910F900BBE0F9084
:100510000FBE0F901F9018951F920F920FB60F925B
:1005200011240BB60F922F933F934F935F936F93CA
:100530007F938F939F93AF93BF93EF93FF93E0913C
:100540000E02F0910F021995FF91EF91BF91AF91BB
:100550009F918F917F916F915F914F913F912F91DB
:100560000F900BBE0F900FBE0F901F9018951F920B
:100570000F920FB60F9211240BB60F922F933F9349
:100580004F935F936F937F938F939F93AF93BF939B
:10059000EF93FF93E0910C02F0910D021995FF91FA
:1005A000EF91BF91AF919F918F917F916F915F91EB
:1005B0004F913F912F910F900BBE0F900FBE0F9058
:1005C0001F9018951F920F920FB60F9211240BB621
:1005D0000F922F933F934F935F936F937F938F93DC
:1005E0009F93AF93BF93EF93FF93E0910A02F09133
:1005F0000B021995FF91EF91BF91AF919F918F9150
:100600007F916F915F914F913F912F910F900BBE12
:100610000F900FBE0F901F9018951F920F920FB65C
:100620000F9211240BB60F922F933F934F935F932A
:100630006F937F938F939F93AF93BF93EF93FF93AA
:10064000E0910802F09109021995FF91EF91BF9195
:10065000AF919F918F917F916F915F914F913F915A
:100660002F910F900BBE0F900FBE0F901F901895FB
:100670000F931F93CF93DF93EC010E94ECA4688744
:1006800079878A879B87E881F9810284F385E02D49
:10069000CE01199597FF15C00E94ECA40885198515
:1006A0002A853B85601B710B820B930B0C811D818E
:1006B0002E813F81601771078207930720F38FEF28
:1006C0009FEFDF91CF911F910F910895EF92FF92CD
:1006D0000F931F93CF93DF93EC017B01042F66E808
:1006E00075E00E948981C7010E943883002E000CAA
:1006F000110B97FD0BC00817190741F0682FCE01A9
:100700000E943C80C7010E943883F3CFCE01DF9165
:10071000CF911F910F91FF90EF9008958F929F922C
:10072000AF92BF92EF92FF920F931F93CF93DF93FD
:10073000CDB7DEB7A1970FB6F894DEBF0FBECDBF21
:100740007C01FA01CB0119A2223008F42AE08E01C3
:100750000F5D1F4F822E912CB12CA12CBF01A50142
:1007600094010E9440D2F901CA016A300CF5605D23
:10077000D8016E938D01232B242B252B79F790E044
:1007800080E0109721F0BD01C7010E94597CA1961D
:100790000FB6F894DEBF0FBECDBFDF91CF911F9192
:1007A0000F91FF90EF90BF90AF909F908F90089522
:1007B000695CDECF64E875E00C94597C0F931F935D
:1007C000CF93DF93EC010E94597C8C01CE010E94F3
:1007D000DA83800F911FDF91CF911F910F910895C0
:1007E000DC01ED91FC910190F081E02D19942F92A4
:1007F0003F924F925F926F927F928F929F92AF92B1
:10080000BF92CF92DF92EF92FF921F93CF93DF932D
:10081000EC016A017B01722EAB019601CB01B6019E
:100820000E945ED467E875E0811126C04601570139
:10083000E894B7F82FEF3FEF4FE75FE7C501B4014A
:100840000E945ED481110CC02FEF3FEF4FE75FE7AE
:10085000C501B4010E94F6D06BE875E0181664F08B
:100860002FEF3FEF4FE75FE4C701B6010E94FED3D1
:100870001816B4F46FE875E0CE01DF91CF911F91A7
:10088000FF90EF90DF90CF90BF90AF909F908F90B0
:100890007F906F905F904F903F902F900C94597C79
:1008A0002FEF3FEF4FE75FECC701B6010E94F6D094
:1008B00087FDE0CF20E030E0A901C701B6010E942A
:1008C000F6D0312C212C87FF09C06DE2CE010E94A9
:1008D000F0831C01F7FAF094F7F8F09410E060E070
:1008E00070E080E09FE3711641F020E030E040E2EC
:1008F00051E40E9456D31F5FF6CFA70196010E94D4
:10090000EAD22B013C010E94CFD34B015C012AE0CB
:10091000BC01A401CE010E948E837C01E20CF31C79
:100920001123C1F1C501B4010E94FBD09B01AC01B0
:10093000C301B2010E94E9D24B015C016EE2CE011B
:100940000E94F083E80EF91E115020F120E030E003
:1009500040E251E4C501B4010E945CD12B013C018D
:100960000E94CFD34B01B12CA12C2AE0B501A401E8
:10097000CE010E948E83E80EF91EC501B4010E94CB
:10098000FBD09B01AC01C301B2010E94E9D24B0133
:100990005C01DACFC701DF91CF911F91FF90EF90FB
:1009A000DF90CF90BF90AF909F908F907F906F908F
:1009B0005F904F903F902F900895CF92DF92EF92EB
:1009C000FF920F931F93CF93DF932115310581F48D
:1009D000DC01ED91FC910190F081E02D642FDF911D
:1009E000CF911F910F91FF90EF90DF90CF901994CE
:1009F0002A30310501F52AE077FF1DC06A017B012D
:100A0000EC016DE20E94F0838C0144275527BA0166
:100A10004C195D096E097F092AE0CE010E948E8380
:100A2000800F911FDF91CF911F910F91FF90EF9059
:100A3000DF90CF900895DF91CF911F910F91FF909C
:100A4000EF90DF90CF900C948E838F929F92AF9215
:100A5000BF92CF92DF92EF92FF920F931F93CF93AB
:100A6000DF937C018B014C0182E0880E911C5701C1
:100A7000E5E0AE0EB11CD0E0C0E0F40161914F01A1
:100A8000C8010E94CA9B6C016EE2C8010E94F083FB
:100A90008C0D9D1DC80FD91F8A149B0471F7F70197
:100AA0006581C8010E94CA9B8C0F9D1FDF91CF9169
:100AB0001F910F91FF90EF90DF90CF90BF90AF907C
:100AC0009F908F9008956115710511F00C94597CD9
:100AD00090E080E008950F931F93CF93DF93EC0194
:100AE0008B0168E675E00E94638501151105C1F16F
:100AF000F80161918F01662399F1603240F0623212
:100B000031F06C3521F0CE010E94F083F1CF6CE51D
:100B1000CE010E94F083F801319780818C30D1F0B2
:100B200044F48930D9F08A30B9F0883009F762E6A8
:100B3000EACF823259F024F462E78D3021F3D8CF26
:100B40008F3231F06CE58C35F1F2D2CF62E2DBCF3F
:100B50006FE2D9CF66E6D7CF6EE6D5CF64E7D3CFC5
:100B600062E2CE010E94F08390E080E0DF91CF91BD
:100B70001F910F910895DB0114964D915C9115978B
:100B80006D917C91DC01ED91FC910280F381E02D6F
:100B90001994EF92FF920F931F93CF93DF938C01E1
:100BA0007B01D0E0C0E0F701EC0FFD1F64916623EC
:100BB00061F0D801ED91FC910190F081E02DC80128
:100BC0001995892B11F02196EECFCE01DF91CF91AF
:100BD0001F910F91FF90EF9008950F931F93CF9364
:100BE000DF93EC010E94C9858C01CE010E94DA835B
:100BF000800F911FDF91CF911F910F9108958AE986
:100C000099E00E94DA836DED79E18AE999E00C942C
:100C1000C985DC018BED93E08D939D9384E0FB010E
:100C200001900D928A95E1F708953F924F925F925D
:100C30006F927F928F929F92AF92BF92CF92DF92EC
:100C4000EF92FF920F931F93CF93DF93CDB7DEB751
:100C5000EA970FB6F894DEBF0FBECDBF7C012A0124
:100C60003B0169010E94ECA44B015C0187010D5B13
:100C70001F4FC8010E942D1718161906ACF00E94CC
:100C8000ECA4681979098A099B0946165706680673
:100C9000790608F468C10E948A6661E070E080E02D
:100CA00090E00E94B9A4E5CF42E250E0BE016F5F40
:100CB0007F4FC8010E94B81689818230D1F0312C53
:100CC000832DEA960FB6F894DEBF0FBECDBFDF913D
:100CD000CF911F910F91FF90EF90DF90CF90BF9039
:100CE000AF909F908F907F906F905F904F903F90CC
:100CF0000895F801848995898334910501F76D8100
:100D00007E818F8198850E94D3D24B015C01F601D0
:100D100080829182A282B38246E050E0B701685F90
:100D20007F4FCE014D960E94DBD6892B41F6F7010D
:100D300080819181A281B38188169906AA06BB069B
:100D400008F4BDCF84819581A681B7818815990566
:100D5000AA05BB0508F4B3CF89899A89AB89BC89F8
:100D600086879787A08BB18B4EEC50E070E060E0F7
:100D7000C8010E94B816312CC701829698AB8FA784
:100D8000F701B696FAABE9AB08969CAB8BAB670163
:100D90009AE1C90ED11CBD96FEABEDABC7014296E0
:100DA00098AF8FABFD97FAAFE9AF4701FEE18F0E29
:100DB000911CF801818D928D181619060CF080CFC8
:100DC000C8010E94D7168333910509F4B2C014F507
:100DD0008130910509F464C044F4892B51F3C801B2
:100DE0000E94D716AC01552775C08330910509F4D0
:100DF00062C00697A1F7C8010E94D716B82E44E03A
:100E000050E0B401C8010E94B816EB2DE450FF0B6E
:100E1000AF0160C08A33910509F45FC084F5853362
:100E20009105B1F1C697D9F6C8010E94D7165C01A9
:100E3000B601CE0189960E9409868BA59CA5ADA519
:100E4000BEA5892B8A2B8B2BB1F0EDA9FEA9408082
:100E5000518062807380B601CE0183960E9409861C
:100E60008DA19EA1AFA1B8A5A501481659066A0695
:100E70007B0609F0B8CF44E050E0B60118C08B33D0
:100E8000910509F440C08F3F910509F492CFA7CF97
:100E9000C8010E94D716C8010E94D716382E89CFE4
:100EA000C8010E94D71644E050E06FA978ADC80190
:100EB0000E94B8167ECFC8010E94D716B82E44E013
:100EC00050E069AD7AADC8010E94B8168B2D8450F0
:100ED000990BAC0170E060E0EACFC8010E94D71620
:100EE00044E050E069A97AA9C8010E94B816F70148
:100EF00066A177A180A591A50E94D3D266A377A30E
:100F000080A791A756CFC8010E94D71644E050E0B1
:100F10006BA97CA9C8010E94B816F70162A573A548
:100F200084A595A50E94D3D262A773A784A795A78D
:100F300040CFC8010E94D71644E050E06FA578A9C1
:100F4000C8010E94B816F70162A173A184A195A1FE
:100F50000E94D3D262A373A384A395A366A777A7A5
:100F600080AB91AB26CF33243A94AACE2F923F92F6
:100F70004F925F926F927F928F929F92AF92BF92A9
:100F8000CF92DF92EF92FF920F931F93CF93DF9355
:100F900000D000D0CDB7DEB78C010E9439CA2FEC4B
:100FA00037E040E050E00E9462D2DC01CB010196C4
:100FB000A11DB11DF80184839583A683B783808327
:100FC0009183A283B3835801F3E4AF0EB11CC50132
:100FD0000E94821664E470E0C5010E94FC17882319
:100FE00009F445C10E94ECA42B013C01480182E4B4
:100FF000880E911C48EEC42E43E0D42EE12CF12C37
:1010000052E0252E1E821D82D4018C918330B1F1D5
:10101000811166C0F80184819581A681B78101960E
:10102000A11DB11D84839583A683B7830E94ECA480
:101030006419750986099709A70196010E9440D293
:10104000A90161E0C8010E94937D81E0D4018C93E5
:101050008D819E810197C1F20E94ECA464197509EB
:1010600086099709D801D6962D913D914D915C91B5
:10107000D997261737074807590720F6C5010E9458
:101080008216F80184819581A681B7810196A11D00
:10109000B11D84839583A683B7830E94ECA4F801D5
:1010A000FE9660837183828393838D819E812696D1
:1010B0000FB6F894DEBF0FBECDBFDF91CF911F9169
:1010C0000F91FF90EF90DF90CF90BF90AF909F90E7
:1010D0008F907F906F905F904F903F902F900895EA
:1010E0008430F1F4F80184819581A681B78101965D
:1010F000A11DB11D84839583A683B7830E94ECA4B0
:101100006419750986099709A70196010E9440D2C2
:10111000A90163E0C8010E94937DD4012C9298CF6D
:10112000813051F5F80142AD53AD64AD75AD9E010E
:101130002F5F3F4FC8010E941586382EF2E08F13B3
:1011400090C089819A81AB81BC81F80184839583A9
:10115000A683B7830E94ECA46419750986099709D0
:10116000A70196010E9440D2A90163E0C8010E9434
:10117000937DD4013C926CCF823009F069CFF801A5
:1011800042AD53AD64AD75AD9E012F5F3F4FC801B9
:101190000E941586382EF5E08F135DC0E3E0D40180
:1011A000EC93F80182A193A1A4A1B5A1892B8A2B6C
:1011B0008B2B41F484E893E0A0E0B0E082A393A3FA
:1011C000A4A3B5A3F80186A197A1A0A5B1A5892BD9
:1011D0008A2B8B2B61F482A193A1A4A1B5A1B69512
:1011E000A7959795879586A397A3A0A7B1A7F80180
:1011F00082A593A5A4A5B5A5892B8A2B8B2BA9F431
:1012000082A193A1A4A1B5A1AC01BD0123E0769573
:101210006795579547952A95D1F7841B950BA60B93
:10122000B70B82A793A7A4A7B5A7F80186A197A19A
:10123000A0A5B1A586A797A7A0ABB1AB82A593A5A2
:10124000A4A5B5A582AB93ABA4ABB5AB81E090E010
:101250009E838D83FDCE96E0891303C0D4011C923A
:10126000F7CEBFEF3B12F4CEF4011082F1CE1E8216
:101270001D821BCF1F920F920FB60F9211240BB637
:101280000F922F933F934F935F936F937F938F931F
:101290009F93AF93BF93EF93FF938AE999E00E94E6
:1012A0002D79FF91EF91BF91AF919F918F917F9198
:1012B0006F915F914F913F912F910F900BBE0F90C7
:1012C0000FBE0F901F9018951F920F920FB60F929E
:1012D00011240BB60F922F938F939F93EF93FF934D
:1012E000E091AA09F091AB098081E091B009F091F9
:1012F000B10982FD1DC090818091B3098F5F8F730A
:101300002091B409821741F0E091B309F0E0E6566C
:10131000F64F958F8093B309FF91EF919F918F9135
:101320002F910F900BBE0F900FBE0F901F9018952E
:101330008081F2CFDF92EF92FF920F931F93CF93B2
:10134000DF9300D000D0CDB7DEB78B017A01D22E6B
:1013500066E875E0CE0101960E9489819E012F5FAB
:101360003F4F4D2DB701C8010E9459AECE010196E5
:101370000E944A8126960FB6F894DEBF0FBECDBFFD
:10138000DF91CF911F910F91FF90EF90DF90089523
:10139000CF92DF92EF92FF920F931F93CF93DF9341
:1013A000CDB7DEB7EC970FB6F894DEBF0FBECDBF5A
:1013B000DC012C91222309F459C061E574E00E94FC
:1013C00047CB9A8389837E01B3E0EB0EF11C01E0E9
:1013D00010E0D02EC12E61E574E090E080E00E9424
:1013E00047CBF701819391937F010E31110521F0D5
:1013F0000F5F1F4F892B69F70091A2071091A30778
:10140000E980FA800115110549F1D8016D917C91AF
:10141000C7010E942CD7892BE9F4D8011296ED91CF
:10142000FC91BE016F5F7F4F8D2D9C2D19958C0116
:101430000E94FF85C801EC960FB6F894DEBF0FBE80
:10144000CDBFDF91CF911F910F91FF90EF90DF9073
:10145000CF900895F80104811581D4CF61EE79E130
:101460008AE999E00E94ED850E94FF8510E000E086
:10147000E1CFCF938AE999E00E941779892BE9F1AE
:101480008AE999E00E94F578C82F8A3089F08D307A
:1014900079F0883001F568E08AE999E00E94F083EC
:1014A0008091A607882331F381508093A607E2CF6D
:1014B000E091A607F0E0EA59F84F108264E875E081
:1014C0008AE999E00E94638586E697E00E94C889D0
:1014D0001092A607CFCF682F8AE999E00E94F08387
:1014E000E091A607EB3330F681E08E0F8093A607DC
:1014F000F0E0EA59F84FC083BDCFCF910895CF9364
:10150000DF930E946A7CEC01892B99F08A818150DB
:101510008A8381110EC0888199810E9464C91982D1
:101520001882E0916407F0916507C1E6D7E0309733
:1015300019F4DF91CF9108959381848120813181C5
:10154000232B41F49B838C83CF010E9464C99B8130
:101550008C81FE01EF01E92FF82FE9CFEF92FF9286
:101560000F931F93CF93DF937C010E946A7CFC0151
:10157000892B61F082818F5F828380819181DF91ED
:10158000CF911F910F91FF90EF900895C1E6D7E0A2
:1015900088819981892B51F4C7010E94C1D6998312
:1015A000888321E02A83EBCFEC01F2CF8B819C81F1
:1015B0000097D1F785E090E00E94C8C88C0190E0C8
:1015C00080E001151105D9F21C830B83C7010E942D
:1015D000C1D6F8019183808321E022831482138293
:1015E000CECF8F929F92AF92BF92CF92DF92EF9227
:1015F000FF920F931F93CF93DF936115710509F449
:101600008FC0DB011896EC911897EF70E73008F067
:1016100087C0EC01F0E08827EF5EF4478F4F0C9411
:10162000CBD2188B298B328B498B938BA58BDE8B7E
:1016300063E975E0CE01DF91CF911F910F91FF908B
:10164000EF90DF90CF90BF90AF909F908F900C94D1
:10165000597C19968C916DE975E0882359F368E9F6
:1016600075E0E8CF19964D915D916D917C911C9735
:101670002AE030E0CE01DF91CF911F910F91FF90D2
:10168000EF90DF90CF90BF90AF909F908F900C9491
:10169000DD841996CD90DD90ED90FC901C9720E0B4
:1016A00030E0A901C701B6010E94F6D087FF09C04A
:1016B00067EF73E0CE010E946385F7FAF094F7F8C4
:1016C000F094C701B6010E94CFD34B015C01BC016D
:1016D000A401CE010E94C79B6BE775E0CE010E947A
:1016E0006385C501B4010E94FBD09B01AC01C70119
:1016F000B6010E94E9D22DEC3CEC4CE45DE30E9483
:10170000EAD220E030E040E251E40E945CD10E9445
:10171000CFD3AB0170E060E02AE0CE010E948E835F
:1017200090E080E01DC019966D917C91CE01DF9113
:10173000CF911F910F91FF90EF90DF90CF90BF90CE
:10174000AF909F908F900C946B8516960D911C9185
:101750006BE5CE010E94F083019679F48FEF9FEF45
:10176000DF91CF911F910F91FF90EF90DF90CF907D
:10177000BF90AF909F908F9008950115110579F05B
:10178000B801CE010E94F18A019641F3D801129668
:101790000D911C910115110511F06CE2DACF6DE588
:1017A000CE010E94F08321E030E0019611F030E09C
:1017B00020E088279927821B930BD2CF16960D9194
:1017C0001C916BE7CE010E94F083019639F201155E
:1017D000110529F1D8016D917C91CE010E946B8594
:1017E000019609F4BBCF6AE3CE010E94F083019613
:1017F00009F4B4CFB801CE010E94F18A019609F430
:10180000ADCFD80112960D911C910115110539F03B
:101810006CE2CE010E94F0830196C9F69FCF6DE77E
:10182000BFCF0F931F93CF93DF93EC01E881F98132
:101830000284F385E02D199500E011E08F3F9807B1
:10184000D1F081329105E4F401501109E881F98168
:101850000F3F100731F00284F385E02DCE0119957A
:10186000EDCFE881F9810684F785E02D682FCE0160
:10187000199590E080E0DF91CF911F910F9108952D
:10188000012B79F78FEF9FEFF6CFCF92DF92EF9298
:10189000FF920F931F93CF93DF937C016B01DC01C9
:1018A000ED91FC910284F385E02D1995829761F00A
:1018B000CFEFDFEFCE01DF91CF911F910F91FF901E
:1018C000EF90DF90CF90089584E0F601808786E066
:1018D00090E00E94C8C88C01009751F3E1E2F7E064
:1018E000DC01ED93FC9380E4DF011D928A95E9F71A
:1018F00080E490E0F8019383828315821482D701FB
:10190000ED91FC910284F385E02DC7011995EC015E
:101910000196C9F0C232D10509F44DC0C032D105DB
:101920000CF449C0B8018C2FCC35D10549F5D7014D
:10193000ED91FC910284F385E02DC7011995EC012E
:101940008F3F980721F4C8010E9464C9B3CF823643
:10195000910541F15CF48F32910509F18C359105C7
:10196000D9F0829761F6B80182E20AC08E369105FD
:10197000E1F04CF4B8018CE0C636D10509F0BFCFD8
:101980000E94FA7ABCCF8237910591F0B80189E0C4
:10199000C437D105A9F3B3CFB8018CE5F1CFB801B5
:1019A0008FE2EECFB80188E0EBCFB8018AE0E8CF54
:1019B000B8018DE0E5CFF80184819581009749F069
:1019C0000190F081E02DE80FF91F31978081882385
:1019D00021F0B80180E00E94FA7A81E297E00E944B
:1019E000AE8AEC01892B19F0C8010E9464C9D601A6
:1019F0001A96DC93CE931997D0E0C0E05BCF8DE0D0
:101A000090E00E94C8C8009729F02DE0FC011192D7
:101A10002A95E9F708950F931F93CF93DF930097CB
:101A2000E1F0EC010C851D850115110579F0D80157
:101A30008D919C91009739F0DC01ED91FC91048827
:101A4000F589E02D1995C8010E9464C9CE01DF9186
:101A5000CF911F910F910C94E1CBDF91CF911F910A
:101A60000F910895AF92BF92CF92DF92EF92FF92C3
:101A70000F931F93CF93DF9300D01F92CDB7DEB7A4
:101A800061157105B1F06B01182FDB011C96AD904B
:101A9000BC90F501E080F180D701ED91FC910688C2
:101AA000F789E02DC7011995811106C0C6010E9472
:101AB0000B8D8FEF9FEF13C0F5019281911124C020
:101AC000D701ED91FC910190F081E02D612FC701CC
:101AD0001995F701818D811111C090E080E00F9080
:101AE0000F900F900F90DF91CF911F910F91FF906A
:101AF000EF90DF90CF90BF90AF900895612F8AE96B
:101B000099E00E94F083E9CF812F8F7D81548A3143
:101B1000B8F280ED810F8A3098F283ED810F823028
:101B200078F21F3569F21E3759F21132B1F086ECA6
:101B3000810F823090F08AED810F873070F01D3375
:101B400061F0812F8F7E8F3241F08DED810F8230D9
:101B500020F01B3511F01D3511F491FFB1CF198222
:101B60001A821B821C82812F012E000C990B9F93DD
:101B70001F9383EA95E09F938F938E010F5F1F4F12
:101B80001F930F930E94B1D76E01F4E0CF0ED11CCA
:101B90000F900F900F900F900F900F90D8016D91B4
:101BA0008D01D701ED91FC910190F081E02DC701ED
:101BB0001995F701818D882339F0F80131976081FB
:101BC0008AE999E00E94F0830C151D0539F785CF4D
:101BD000CF93C82F462F61E070E00E94892161E019
:101BE00070E08C2F0E94B7218111F9CFCF91089519
:101BF000AF92BF92CF92DF92EF92FF920F931F931B
:101C0000CF93DF9300D01F92CDB7DEB78C016B016D
